:1000000000000320F5620100D96201009162010045
:100010009162010091620100916201009162010010
:10002000916201009162010091620100D9620100B8
:10003000D962010091620100AD570100255A01000B
:10004000D9620100D9620100D9620100D9620100C0
:10005000D9620100D9620100D9620100D9620100B0
:10006000D9620100D9620100D9620100D9620100A0
:10007000D9620100D9620100D9620100D962010090
:10008000D9620100D9620100D9620100D962010080
:10009000D9620100D9620100D9620100D962010070
:1000A000A9180100051A0100D9620100D9620100F6
:1000B000D9620100D9620100D962010049750100CD
:1000C000D962010071970100D9620100CD98010049
:1000D000D9620100FD990100D9620100D9620100D5
:1000E000D9620100D9620100D9620100D962010020
:1000F000D9620100D9620100D9620100D962010010
:10010000D9620100D9620100D9620100D9620100FF
:10011000D962010035780100D9620100D96201007D
:10012000D9620100D9620100D9620100D9620100DF
:10013000D9620100D9620100D9620100D9620100CF
:10014000F9540100D96201002D9B0100D962010020
:10015000D9620100D9620100D9620100D9620100AF
:10016000D9620100D9620100611B0100D96201005E
:10017000D9620100D9620100D9620100D96201008F
:10018000D9620100B9FE0000D9620100D962010004
:10019000D9620100D96201005D9C0100D9620100B1
:1001A000D9620100D9620100D9620100D96201005F
:1001B000D9620100D9620100D9620100D96201004F
:1001C000D9620100D9620100D9620100D96201003F
:1001D000FFFFFFFFFFFFFFFFFFFFFFFFFFFFFFFF2F
:10040000FFFFFFFFFFFFFFFFFFFFFFFFDEF9FFFF23
:1004100010B5054C237833B9044B13B10448AFF33E
:1004200000800123237010BD00B0FF1F00000000FA
:10043000940E0F00084B10B51BB108490848AFF3E4
:1004400000800848036803B910BD074B002BFBD0A0
:10045000BDE81040184700BF0000000004B0FF1FB7
:10046000940E0F0058A2FF1F0000000049F2FC2369
:10047000C1F6FF731B7C022B9DBF41F6E062C0F208
:10048000020252F823000020704700BF49F2FC230B
:10049000C1F6FF735B7C032B9DBF41F6EC62C0F29B
:1004A000020252F823000020704700BF49F2FC23EB
:1004B000C1F6FF7349F2B822987C49F2A423C1F631
:1004C000FF72C1F6FF7300280CBF10461846704734
:1004D00049F2FC23C1F6FF7393F822306BB149F265
:1004E0003033C1F6FF7346F64F62C0F2200249F284
:1004F00030301A60C1F6FF70704749F23033C1F6F0
:10050000FF7346F24F62C0F2660249F230301A6061
:10051000C1F6FF70704700BF4DF67833C2F200039A
:100520001B786BB149F2E023C1F6FF7346F25952D2
:10053000C0F2730249F2E0201A60C1F6FF70704702
:1005400049F2E023C1F6FF7346F64E72C0F2200274
:1005500049F2E0201A60C1F6FF707047704700BF93
:10056000704700BF704700BF704700BF08B549F231
:10057000FC23C1F6FF73DA7C72B140F2306149F2BC
:100580002430C0F20201C1F6FF701CF011FE49F2E6
:100590002430C1F6FF7008BD40F2246149F22430D6
:1005A000C0F20201C1F6FF701CF002FE49F22430D5
:1005B000C1F6FF7008BD00BF10B549F2FC23C1F6BB
:1005C000FF73B2EE047A1B7D07EE903AF8EE677A7D
:1005D00049F2B024C7EE876AC1F6FF7416EE900A9E
:1005E0001BF00EFB0B4640F23C610246C0F20201DA
:1005F00020461CF0DDFD204610BD00BF10B549F2BD
:10060000FC23C1F6FF73B2EE047A5B7D07EE903AED
:10061000F8EE677A49F23C34C7EE876AC1F6FF7498
:1006200016EE900A1BF0ECFA0B4640F23C610246D3
:10063000C0F2020120461CF0BBFD204610BD00BFE9
:1006400010B549F2FC23C1F6FF7349F24834C1F6F4
:10065000FF7440F2486193F90A202046C0F202017B
:100660001CF0A6FD204610BD10B5044614F0C6FED1
:10067000204610BD08B549F2FC23C1F6FF7393F87C
:10068000212072B140F25C6149F2DC20C0F202012B
:10069000C1F6FF701CF08CFD49F2DC20C1F6FF7042
:1006A00008BD40F25463C0F2020393E8030049F22C
:1006B000DC23C1F6FF731860197149F2DC20C1F622
:1006C000FF7008BD00F0F703F52B06D0F92804D021
:1006D000EF2803D800F0F00070470020704700BFFB
:1006E00038B549F2E864C1F6FF74014600230A22D6
:1006F000204615F09FFA0546204615F089FA284451
:1007000038BD00BF38B549F2E864C1F6FF74014650
:1007100000230A22204615F08DFA0546204615F0E2
:1007200077FA284438BD00BF10B504461CF068FDB8
:1007300001462046BDE8104018F01EBE10B5044624
:100740001CF05EFD0146204618F016FE044649F2F4
:10075000E860C1F6FF7015F05BFA204410BD00BFE1
:1007600040F2646038B52021C0F202004DF6FC343E
:1007700018F002FEC2F200044EF2B8112046C2F296
:10078000000112F0F3F943F2B441C2F2000149F260
:10079000FC224CF66C00C2F20000C1F6FF7244F27B
:1007A0009043C2F200034D688570127B4A600020BE
:1007B00063259D6383F83C00586372B6AA42A8BFC4
:1007C0002A469200DA6262B62046BDE8384012F04E
:1007D00019BA00BF40F2886008B5C0F202001021CB
:1007E00018F0CAFD49F2FC23C1F6FF7393F82230DA
:1007F000E3B144F2F413C2F20003F821986C0368E9
:100800001B68984740F29C60C0F20200FFF78CFF23
:100810004EF28070C2F200004FF60F0114F096F80D
:1008200040F2AC60C0F20200FFF77EFF49F2E860E0
:10083000C1F6FF70BDE8084015F0EAB940F2C460A7
:1008400008B5C0F20200132118F096FD49F2FC230E
:10085000C1F6FF7393F82230E3B144F2F413C2F20D
:100860000003FB21986C03681B68984740F29C606A
:10087000C0F20200FFF758FF4EF28070C2F2000093
:100880004FF60F3114F062F840F2AC60C0F2020093
:10089000FFF74AFF49F2E860C1F6FF70BDE8084083
:1008A00015F0B6B940F2D86008B5C0F202001021C8
:1008B00018F062FD49F2FC23C1F6FF7393F8223071
:1008C000E3B144F2F413C2F20003FA21986C036816
:1008D0001B68984740F29C60C0F20200FFF724FFBB
:1008E0004EF28070C2F200004FF60F2114F02EF885
:1008F00040F2AC60C0F20200FFF716FF49F2E86078
:10090000C1F6FF70BDE8084015F082B940F2EC6016
:1009100008B5C0F202000F2118F02EFD49F2FC23A9
:10092000C1F6FF7393F82230E3B144F2F413C2F23C
:100930000003FC21986C03681B68984740F29C6098
:10094000C0F20200FFF7F0FE4EF28070C2F200002B
:100950004FF60F4113F0FAFF40F2AC60C0F2020014
:10096000FFF7E2FE49F2E860C1F6FF70BDE808401B
:1009700015F04EB940F2FC6008B5C0F202001B2130
:1009800018F0FAFC49F2FC23C1F6FF7393F8223009
:10099000C3B144F2F413C2F20003F621986C036869
:1009A000DB6C984740F29C60C0F20200FFF7BCFE8F
:1009B0004FF20F6017F056FE40F21870C0F20200BE
:1009C000FFF7B2FE49F2E860C1F6FF70BDE80840EB
:1009D00015F01EB940F2287008B5C0F202001621C9
:1009E00018F0CAFC49F2FC23C1F6FF7393F82230D9
:1009F000E3B144F2F413C2F20003FF21986C0368E0
:100A00001B68984740F29C60C0F20200FFF78CFE22
:100A10004EF28070C2F200004FF60F7113F096FF95
:100A200040F2AC60C0F20200FFF77EFE49F2E860DF
:100A3000C1F6FF70BDE8084015F0EAB82DE9F041B5
:100A4000804640F240700F46C0F20200102118F0BC
:100A500093FC49F2FC23C1F6FF7393F822303BB9B3
:100A600049F2E860C1F6FF70BDE8F04115F0D0B87A
:100A700044F2F415C2F20005F021A86C0368DB6CA7
:100A8000984757B1444608EB0706A86C14F8011BB9
:100A900003681B689847A642F7D1A86C0368F72142
:100AA000DB6C984740F29C60C0F20200FFF73CFE0E
:100AB0004EF280703A464146C2F20000002313F025
:100AC00083FF40F2AC60C0F20200FFF72DFE49F256
:100AD000E860C1F6FF70BDE8F04115F099B800BFBD
:100AE00038B5044640F25470C0F202001F2118F0DD
:100AF00043FC49F2FC23C1F6FF7393F82230EBB1BB
:100B000004F00F044FF202152404C0F2100525432F
:100B10004EF280702946C2F2000013F017FF40F237
:100B2000AC60C0F20200FFF7FFFD284617F09AFD07
:100B300040F21870C0F20200FFF7F6FD49F2E860DB
:100B4000C1F6FF70BDE8384015F062B840F274702D
:100B500008B5C0F20200182118F00EFC49F2FC237F
:100B6000C1F6FF7393F82230E3B144F2F413C2F2FA
:100B70000003FE21986C03681B68984740F29C6054
:100B8000C0F20200FFF7D0FD4EF28070C2F200000A
:100B90004FF60F6113F0DAFE40F2AC60C0F20200D3
:100BA000FFF7C2FD49F2E860C1F6FF70BDE80840FA
:100BB00015F02EB840F2907008B5C0F20200162170
:100BC00018F0DAFB49F2FC23C1F6FF7393F82230E8
:100BD000E3B144F2F413C2F20003F621986C036807
:100BE000DB6C984740F29C60C0F20200FFF79CFD6E
:100BF0004EF28070C2F200004FF20F6113F0A6FEB9
:100C000040F2AC60C0F20200FFF78EFD49F2E860EE
:100C1000C1F6FF70BDE8084014F0FABF40F2A870BA
:100C200010B51621C0F2020018F0A6FB49F2E860E8
:100C3000C1F6FF704DF6FC3414F0EAFFC2F2000476
:100C40004CF6E8412046C2F2000111F08FFF43F25A
:100C5000B442C2F200024CF66C03C2F200035268C6
:100C60001A702046BDE8104011F0CCBF38B50446DC
:100C700040F2C0700D46C0F202000D2118F07CFB5E
:100C800049F2FC23C1F6FF7393F822300BB32B0417
:100C900003F4FE03013C43F44043240243F00C03FD
:100CA00004F470641C434EF280702146C2F20000CE
:100CB00013F04CFE40F2AC60C0F20200FFF734FDCE
:100CC000204617F0CFFC40F21870C0F20200FFF788
:100CD0002BFD49F2E860C1F6FF70BDE8384014F022
:100CE00097BF00BF38B5044640F2D0700D46C0F241
:100CF00002000D2118F040FB49F2FC23C1F6FF73FE
:100D000093F822300BB32B0403F4FE03013C43F4AD
:100D10005043240243F00D0304F470641C434EF26C
:100D200080702146C2F2000013F010FE40F2AC6069
:100D3000C0F20200FFF7F8FC204617F093FC40F2E7
:100D40001870C0F20200FFF7EFFC49F2E860C1F64C
:100D5000FF70BDE8384014F05BBF00BF70B50646B9
:100D600040F2E0700C46C0F202001221154618F065
:100D700003FB49F2FC23C1F6FF7393F822303BB921
:100D800049F2E860C1F6FF70BDE8704014F040BF62
:100D90006B1E1B02240404F4FE0403F4706323435B
:100DA00043F45043340143F00D03E4B21C434EF2CC
:100DB0008070C2F20000214613F0C8FD40F2AC6022
:100DC000C0F20200FFF7B0FC6EB140F21870C0F242
:100DD0000200FFF7A9FC49F2E860C1F6FF70BDE828
:100DE000704014F015BF204617F03CFCEDE700BF43
:100DF00038B5044640F2F470C0F202001A2118F02F
:100E0000BBFA49F2FC23C1F6FF7393F822301BB3FF
:100E100044F2F415C2F20005F321A86C03681B68C4
:100E20009847A86C036804F07F01DB6C984740F298
:100E30009C60C0F20200FFF777FC200400F4FE0083
:100E400040F4734040F0020017F00CFC40F21870C0
:100E5000C0F20200FFF768FC49F2E860C1F6FF70DB
:100E6000BDE8384014F0D4BE38B5044640F6100052
:100E7000C0F20200242118F07FFA49F2FC23C1F6E7
:100E8000FF7393F822301BB344F2F415C2F200054D
:100E9000F121A86C03681B689847A86C0368214679
:100EA0001B68984740F29C60C0F20200FFF73CFCD0
:100EB00004F00F044FF202102404C0F2100020438B
:100EC00017F0D0FB40F21870C0F20200FFF72CFCC4
:100ED00049F2E860C1F6FF70BDE8384014F098BEF2
:100EE00038B5044640F63800C0F20200152118F06B
:100EF00043FA49F2FC23C1F6FF7393F822303BB367
:100F000044F2F415C2F20005F321A86C03681B68D3
:100F10009847A86C036804F07F01DB6C984740F2A7
:100F20009C60C0F20200FFF7FFFB210401F4FE0108
:100F300041F473414EF28070C2F2000041F00201B0
:100F400013F004FD40F2AC60C0F20200FFF7ECFBCE
:100F500049F2E860C1F6FF70BDE8384014F058BEB1
:100F600038B5054640F650000C46C0F202000D218F
:100F700018F002FA49F2FC23C1F6FF7393F822300D
:100F80004BB304F30D0404F500536C1E1A04240241
:100F900002F4FE0204F47064144344F460445B04FD
:100FA00003F0FE4344F00E041C434EF280702146D1
:100FB000C2F2000013F0CAFC40F2AC60C0F20200C2
:100FC000FFF7B2FB204617F04DFB40F21870C0F25D
:100FD0000200FFF7A9FB49F2E860C1F6FF70BDE827
:100FE000384014F015BE00BF38B5044640F6600026
:100FF000C0F202001F2118F0BFF949F2FC23C1F62C
:10100000FF7393F822303BB344F2F415C2F20005AB
:10101000F121A86C03681B689847A86C03682146F7
:101020001B68984740F29C60C0F20200FFF77CFB0F
:1010300004F00F044FF202112404C0F210014EF22A
:101040008070C2F20000214313F080FC40F2AC60DB
:10105000C0F20200FFF768FB49F2E860C1F6FF70DA
:10106000BDE8384014F0D4BD10B540F680004CF611
:101070006C04C2F200042921C0F2020018F07CF9CD
:1010800049F2E86094F90310C1F6FF7014F062FDB4
:1010900049F2E860C1F6FF7014F0BAFD4FF2B801F2
:1010A0004DF6FC30C2F20001C2F2000011F05EFD0C
:1010B0004DF6FC300221C2F2000011F07FFD43F238
:1010C000B441C2F2000194F903204B682370002A56
:1010D00044F29043C2F2000315DB12240020A24226
:1010E0004A609C6383F83C005863D4BF9200482256
:1010F00072B6DA6262B64DF6FC30C2F20000BDE8AC
:10110000104011F07FBD00221220986383F83C202C
:101110005A63E2704A6072B6DA6262B64DF6FC302B
:10112000C2F20000012111F043FDE4E710B540F6E2
:10113000AC004CF66C04C2F200042921C0F202009B
:1011400018F01AF949F2E86094F90510C1F6FF7039
:1011500014F000FD49F2E860C1F6FF7014F058FD8C
:101160004CF2F8214DF6FC30C2F20001C2F2000050
:1011700011F0FCFC4DF6FC300221C2F2000011F02F
:101180001DFD43F2B441C2F2000194F905204B6801
:101190002370002A44F29043C2F2000315DB0324BB
:1011A0000020A2424A609C6383F83C005863D4BF8D
:1011B00092000C2272B6DA6262B64DF6FC30C2F2D0
:1011C0000000BDE8104011F01DBD0022032098630F
:1011D00083F83C205A6362714A6072B6DA6262B682
:1011E0004DF6FC30C2F20000012111F0E1FCE4E711
:1011F00010B540F6D8004CF66C04C2F200042D2164
:10120000C0F2020018F0B8F849F2E86094F9021050
:10121000C1F6FF7014F09EFC49F2E860C1F6FF7061
:1012200014F0F6FC42F6A0114DF6FC30C2F20001BB
:10123000C2F2000011F09AFC4DF6FC300221C2F21D
:10124000000011F0BBFC43F2B441C2F2000194F97A
:1012500002204B682370002A44F29043C2F200033C
:1012600015DB08240020A2424A609C6383F83C00FE
:101270005863D4BF9200202272B6DA6262B64DF68D
:10128000FC30C2F20000BDE8104011F0BBBC0022EF
:101290000820986383F83C205A63A2704A6072B6B3
:1012A000DA6262B64DF6FC30C2F20000012111F0A4
:1012B0007FFCE4E738B5054649F2E86440F60810DB
:1012C000C1F6FF741E21C0F2020018F055F829463D
:1012D00000230A22204614F0ADFC40F628100E210F
:1012E000C0F2020018F048F849F2FC23C1F6FF737F
:1012F0000A2293F821102046002314F09BFC40F6AC
:1013000038100121C0F2020018F036F8204614F01F
:101310007FFC002038BD00BFF8B549F2FC24C1F6BF
:10132000FF740F4694F821301646054623B19842C3
:1013300002D0FFF7BFFF50B14BF20063C2F20003CF
:1013400094F909101868394400220BF0EBFD40F6BF
:101350003C10C0F20200122118F00EF894F822306E
:101360002BB3330603F0FE4343F400433F04013D37
:1013700043F0080307F4FE072D023B4305F47065B4
:101380001D434EF280702946C2F2000013F0DEFACF
:1013900040F2AC60C0F20200FFF7C6F9284617F031
:1013A00061F940F21870C0F20200FFF7BDF949F28E
:1013B000E860C1F6FF70BDE8F84014F029BC00BF3A
:1013C000F8B549F2FC24C1F6FF740F4694F82130B9
:1013D0001646054623B1984202D0FFF76BFF50B185
:1013E0004BF20063C2F2000394F909101868394403
:1013F00032460BF097FD40F65010C0F2020011216A
:1014000017F0BAFF94F822302BB3360606F0FE46EA
:1014100046F410463F04013D46F0090607F4FE0776
:101420002D023E4305F4706535434EF28070294627
:10143000C2F2000013F08AFA40F2AC60C0F202007F
:10144000FFF772F9284617F00DF940F21870C0F254
:101450000200FFF769F949F2E860C1F6FF70BDE8E4
:10146000F84014F0D5BB00BFF8B549F2FC26C1F630
:10147000FF760F4696F821301546044623B1984270
:1014800002D0FFF717FF48B14BF20063C2F200032E
:101490002A461868036839465B68984740F6641026
:1014A000C0F202000D2117F067FF96F822302BB32F
:1014B0002D0605F0FE4545F430453F04013C45F05E
:1014C0000B0507F4FE0724023D4304F470642C432B
:1014D0004EF280702146C2F2000013F037FA40F25B
:1014E000AC60C0F20200FFF71FF9204617F0BAF80F
:1014F00040F21870C0F20200FFF716F949F2E860F6
:10150000C1F6FF70BDE8F84014F082BB40F67410DD
:1015100010B52021C0F2020017F02EFF49F2E8605A
:10152000C1F6FF704DF6FC3414F072FBC2F20004F9
:101530004EF228112046C2F2000111F017FB4DF6C1
:101540007832C2F2000243F2B441C2F2000144F226
:101550009043C2F2000312784A6001200021986390
:1015600083F83C10596372B69200DA6262B6204684
:10157000BDE8104011F046BB40F6981038B51C216C
:10158000C0F2020017F0F8FE49F2E860C1F6FF7001
:101590004DF6FC3414F03CFBC2F200044BF2CC11CB
:1015A0002046C1F6FF7111F0E1FA43F2B441C2F2F4
:1015B000000149F2FC224CF66C00C2F20000C1F6B8
:1015C000FF7244F29043C2F200034D68C570527D31
:1015D0004A60002063259D6383F83C00586372B61F
:1015E000AA42A8BF2A469200DA6262B62046BDE847
:1015F000384011F007BB00BF40F6B81038B51F21C6
:10160000C0F2020017F0B8FE49F2E860C1F6FF70C0
:101610004DF6FC3414F0FCFAC2F2000444F21C0152
:101620002046C2F2000111F0A1FA43F2B441C2F225
:10163000000149F2FC224CF66C00C2F20000C1F637
:10164000FF7244F29043C2F200034D68C570527CB1
:101650004A60002003259D6383F83C00586372B6FE
:10166000AA42A8BF2A469200DA6262B62046BDE8C6
:10167000384011F0C7BA00BF40F6D81038B5202165
:10168000C0F2020017F078FE49F2E860C1F6FF7080
:101690004DF6FC3414F0BCFAC2F2000443F6F861D3
:1016A0002046C2F2000111F061FA43F2B441C2F2E5
:1016B000000149F2FC224CF66C00C2F20000C1F6B7
:1016C000FF7244F29043C2F200034D68C570D27CB1
:1016D0004A60002060259D6383F83C00586372B621
:1016E000AA42A8BF2A469200DA6262B62046BDE846
:1016F000384011F087BA00BF40F6FC1038B5182109
:10170000C0F2020017F038FE49F2E860C1F6FF703F
:101710004DF6FC3414F07CFAC2F200044BF2C071B6
:101720002046C2F2000111F021FA43F2B441C2F2A4
:10173000000149F2FC224CF66C00C2F20000C1F636
:10174000FF7244F29043C2F200034D688570D27973
:101750004A60002063259D6383F83C00586372B69D
:10176000AA42A8BF2A469200DA6262B62046BDE8C5
:10177000384011F047BA00BF40F6182038B517219D
:10178000C0F2020017F0F8FD49F2E860C1F6FF7000
:101790004DF6FC3414F03CFAC2F200044CF24C1149
:1017A0002046C2F2000111F0E1F943F2B441C2F265
:1017B000000149F2FC224CF66C00C2F20000C1F6B6
:1017C000FF7244F29043C2F200034D6885701279B3
:1017D0004A60002063259D6383F83C00586372B61D
:1017E000AA42A8BF2A469200DA6262B62046BDE845
:1017F000384011F007BA00BF40F6302038B5182144
:10180000C0F2020017F0B8FD49F2E860C1F6FF70BF
:101810004DF6FC3414F0FCF9C2F2000443F6085112
:101820002046C2F2000111F0A1F943F2B441C2F224
:10183000000149F2FC224CF66C00C2F20000C1F635
:10184000FF7244F29043C2F200034D688570D27A71
:101850004A60002063259D6383F83C00586372B69C
:10186000AA42A8BF2A469200DA6262B62046BDE8C4
:10187000384011F0C7B900BF40F64C2070B51821B0
:10188000C0F2020017F078FD49F2E860C1F6FF707F
:101890004DF6FC3414F0BCF9C2F200044CF6980189
:1018A0002046C2F2000111F061F949F2FC23C1F6B1
:1018B000FF7343F2B441C2F200014CF66C0044F2F3
:1018C0009042C2F2000293F908304E684B60C2F2B7
:1018D00000000021632523EAE3738670956382F894
:1018E0003C10516372B6AB42A8BF2B469B00D3623B
:1018F00062B62046BDE8704011F084B940F6682019
:1019000038B51E21C0F2020017F036FD49F2E8603A
:10191000C1F6FF704DF6FC3414F07AF9C2F20004FF
:101920004DF67C312046C2F2000111F01FF943F25E
:10193000B441C2F2000149F2FC224CF66C00C2F242
:101940000000C1F6FF7244F29043C2F200034D68FA
:10195000457192F821204A60002010259D6383F88C
:101960003C00586372B6AA42A8BF2A469200DA62C7
:1019700062B62046BDE8384011F044B940F68820F0
:10198000F8B51621C0F2020017F0F6FC49F2E86043
:10199000C1F6FF704DF6FC3414F03AF9C2F20004BF
:1019A0004BF258412046C1F6FF7111F0DFF849F2C1
:1019B000FC23C1F6FF7343F2B441C2F2000193F974
:1019C0000A304F684B604CF66C0044F29042C2F211
:1019D00000026FF03101C2F20000002632258B4276
:1019E0008770B8BF0B46516382F83C60956372B64E
:1019F000AB42A8BF2B469B00D36262B62046BDE82F
:101A0000F84011F0FFB800BF40F6A02038B52421FF
:101A1000C0F2020017F0B0FC49F2E860C1F6FF70B6
:101A20004DF6FC3414F0F4F8C2F200044BF6140145
:101A30002046C2F2000111F099F843F2B441C2F21B
:101A4000000149F2FC224CF66C00C2F20000C1F623
:101A5000FF7244F29043C2F200034D68C570527B9E
:101A60004A60002063259D6383F83C00586372B68A
:101A7000AA42A8BF2A469200DA6262B62046BDE8B2
:101A8000384011F0BFB800BF40F6C82038B520215B
:101A9000C0F2020017F070FC49F2E860C1F6FF7076
:101AA0004DF6FC3414F0B4F8C2F200044DF2F471B7
:101AB0002046C2F2000111F059F843F2B441C2F2DB
:101AC000000149F2FC224CF66C00C2F20000C1F6A3
:101AD000FF7244F29043C2F200034D68C570927BDE
:101AE0004A60002063259D6383F83C00586372B60A
:101AF000AA42A8BF2A469200DA6262B62046BDE832
:101B0000384011F07FB800BF40F6EC2038B51B21FB
:101B1000C0F2020017F030FC49F2E860C1F6FF7035
:101B20004DF6FC3414F074F8C2F200044CF6103197
:101B30002046C2F2000111F019F843F2B441C2F29A
:101B4000000149F2FC224CF66C00C2F20000C1F622
:101B5000FF7244F29043C2F200034D68C570D27B1D
:101B60004A60002063259D6383F83C00586372B689
:101B7000AA42A8BF2A469200DA6262B62046BDE8B1
:101B8000384011F03FB800BF40F6083038B51C218E
:101B9000C0F2020017F0F0FB49F2E860C1F6FF70F6
:101BA0004DF6FC3414F034F8C2F200044BF6203148
:101BB0002046C1F6FF7110F0D9FF43F2B441C2F2E2
:101BC000000149F2FC224CF66C00C2F20000C1F6A2
:101BD000FF7244F29043C2F200034D68C570927CDC
:101BE0004A60002001259D6383F83C00586372B66B
:101BF0009200DA6262B62046BDE8384011F002B8C1
:101C000040F6283070B51A21C0F2020017F0B4FB7C
:101C100049F2E860C1F6FF7013F0FAFF4DF6BC31EF
:101C20004DF6FC30C2F20001C2F2000010F09EFF3F
:101C300049F2FC22C1F6FF7243F2B441C2F2000144
:101C400092F823204E684A604CF66C0044F29043B0
:101C5000C2F200033021C2F20000002501248A42B2
:101C6000467183F83C505C6399630EDC5AB1920074
:101C700072B6DA6262B64DF6FC30C2F20000BDE820
:101C8000704010F0BFBF0422F2E7C022F0E700BFAF
:101C900040F6443038B52021C0F2020017F06CFB4A
:101CA00049F2E860C1F6FF704DF6FC3413F0B0FF66
:101CB000C2F200044DF634012046C2F2000110F0D9
:101CC00055FF43F2B441C2F2000149F2FC224CF646
:101CD0006C00C2F20000C1F6FF7244F29043C2F2FF
:101CE00000034D68C570D27D4A60002063259D6366
:101CF00083F83C00586372B6AA42A8BF2A469200F5
:101D0000DA6262B62046BDE8384010F07BBF00BF03
:101D100040F6683038B52221C0F2020017F02CFBE3
:101D200049F2E860C1F6FF704DF6FC3413F070FF25
:101D3000C2F200044DF228312046C2F2000110F038
:101D400015FF43F2B441C2F2000149F2FC224CF605
:101D50006C00C2F20000C1F6FF7244F29043C2F27E
:101D600000034D68C570527E4A60002014259D63B3
:101D700083F83C00586372B6AA42A8BF2A46920074
:101D8000DA6262B62046BDE8384010F03BBF00BFC3
:101D900040F68C3038B51E21C0F2020017F0ECFA84
:101DA00049F2E860C1F6FF704DF6FC3413F030FFE5
:101DB000C2F200044CF628512046C2F2000110F095
:101DC000D5FE43F2B441C2F2000149F2FC224CF6C6
:101DD0006C00C2F20000C1F6FF7244F29043C2F2FE
:101DE00000034D68C570D27E4A60002063259D6364
:101DF00083F83C00586372B6AA42A8BF2A469200F4
:101E0000DA6262B62046BDE8384010F0FBBE00BF83
:101E100040F6AC3038B52021C0F2020017F0ACFA21
:101E200049F2E860C1F6FF704DF6FC3413F0F0FEA5
:101E3000C2F200044BF28C112046C1F6FF7110F083
:101E400095FE43F2B441C2F2000149F2FC224CF685
:101E50006C00C2F20000C1F6FF7244F29043C2F27D
:101E600000034D68457192F822204A600020012548
:101E70009D6383F83C00586372B69200DA6262B6E2
:101E80002046BDE8384010F0BDBE00BF40F6D0305F
:101E900038B51E21C0F2020017F06EFA49F2E86070
:101EA000C1F6FF704DF6FC3413F0B2FEC2F200042E
:101EB0004BF650412046C2F2000110F057FE43F2AB
:101EC000B441C2F2000149F2FC224CF66C00C2F2AD
:101ED0000000C1F6FF7244F29043C2F200034D6865
:101EE000C570127E4A60002063259D6383F83C0024
:101EF000586372B6AA42A8BF2A469200DA6262B656
:101F00002046BDE8384010F07DBE00BF40F6F030FE
:101F1000F8B51B21C0F2020017F02EFA49F2E86072
:101F2000C1F6FF704DF6FC3413F072FEC2F20004ED
:101F30004AF64C712046C2F2000110F017FE49F239
:101F4000FC23C1F6FF7343F2B441C2F2000193F9DE
:101F50001F304F684B604CF66C0044F29042C2F266
:101F600000026FF03101C2F20000002632258B42E0
:101F7000C770B8BF0B46516382F83C60956372B678
:101F8000AB42A8BF2B469B00D36262B62046BDE899
:101F9000F84010F037BE00BF40F60C4038B51F21A6
:101FA000C0F2020017F0E8F949F2E860C1F6FF70EC
:101FB0004DF6FC3413F02CFEC2F200044FF2C411B3
:101FC0002046C2F2000110F0D1FD43F2B441C2F24A
:101FD000000149F2FC224CF66C00C2F20000C1F68E
:101FE000FF7244F29043C2F200034D68C570127F45
:101FF0004A60002063259D6383F83C00586372B6F5
:10200000AA42A8BF2A469200DA6262B62046BDE81C
:10201000384010F0F7BD00BF40F62C4038B51A210B
:10202000C0F2020017F0A8F949F2E860C1F6FF70AB
:102030004DF6FC3413F0ECFDC2F200044DF65C7179
:102040002046C2F2000110F091FD43F2B441C2F209
:10205000000149F2FC224CF66C00C2F20000C1F60D
:10206000FF7244F29043C2F200034D68457192F84A
:1020700020204A60002063259D6383F83C0058635C
:1020800072B6AA42A8BF2A469200DA6262B6204619
:10209000BDE8384010F0B6BD40F6484038B51E21C6
:1020A000C0F2020017F068F949F2E860C1F6FF706B
:1020B0004DF6FC3413F0ACFDC2F200044EF2E80120
:1020C0002046C2F2000110F051FD43F2B441C2F2C9
:1020D000000149F2FC224CF66C00C2F20000C1F68D
:1020E000FF7244F29043C2F200034D68C570927EC5
:1020F0004A60002014259D6383F83C00586372B643
:10210000AA42A8BF2A469200DA6262B62046BDE81B
:10211000384010F077BD00BF40F66840F8B519218F
:10212000C0F2020017F028F949F2E860C1F6FF702A
:102130004DF6FC3413F06CFDC2F2000444F2303171
:102140002046C2F2000110F011FD49F2FC23C1F655
:10215000FF7343F2B441C2F2000193F91E304F689D
:102160004B604CF66C0044F29042C2F200026FF0F9
:102170003101C2F20000002632258B42C770B8BF81
:102180000B46516382F83C60956372B6AB42A8BFC0
:102190002B469B00D36262B62046BDE8F84010F0A3
:1021A00031BD00BF40F6844038B51B21C0F20200AB
:1021B00017F0E2F849F2E860C1F6FF704DF6FC3422
:1021C00013F026FDC2F200044CF638112046C2F28C
:1021D000000110F0CBFC43F2B441C2F2000149F21D
:1021E000FC224CF66C00C2F20000C1F6FF7244F211
:1021F0009043C2F200034D68C570127C4A60002013
:1022000002259D6383F83C00586372B6AA42A8BFBA
:102210002A46AA40DA6262B62046BDE8384010F08D
:10222000F1BC00BF40F6A04038B51921C0F2020051
:1022300017F0A2F849F2E860C1F6FF704DF6FC34E1
:1022400013F0E6FCC2F2000442F648512046C2F206
:10225000000110F08BFC43F2B441C2F2000149F2DC
:10226000FC224CF66C00C2F20000C1F6FF7244F290
:102270009043C2F200034D68857052794A60002095
:1022800063259D6383F83C00586372B6AA42A8BFD9
:102290002A469200DA6262B62046BDE8384010F065
:1022A000B1BC00BF40F6BC4038B51A21C0F20200F4
:1022B00017F062F849F2E860C1F6FF704DF6FC34A1
:1022C00013F0A6FCC2F2000444F284312046C2F2AC
:1022D000000110F04BFC43F2B441C2F2000149F29C
:1022E000FC224CF66C00C2F20000C1F6FF7244F210
:1022F0009043C2F200034D68857092794A600020D5
:1023000063259D6383F83C00586372B6AA42A8BF58
:102310002A469200DA6262B62046BDE8384010F0E4
:1023200071BC00BF40F6D84038B52121C0F2020090
:1023300017F022F849F2E860C1F6FF704DF6FC3460
:1023400013F066FCC2F200044DF21C612046C2F29A
:10235000000110F00BFC43F2B441C2F2000149F25B
:10236000FC224CF66C00C2F20000C1F6FF7244F28F
:102370009043C2F200034D68C570527F4A6000204E
:1023800063259D6383F83C00586372B6AA42A8BFD8
:102390002A469200DA6262B62046BDE8384010F064
:1023A00031BC00BF40F6FC40F8B51B21C0F2020072
:1023B00016F0E2FF49F2E860C1F6FF704DF6FC341A
:1023C00013F026FCC2F200044EF270012046C2F265
:1023D000000110F0CBFB49F2FC23C1F6FF7343F27E
:1023E000B441C2F2000193F909304F684B604CF6DA
:1023F0006C0044F29042C2F200026FF01701C2F288
:102400000000002618258B428770B8BF0B46516329
:1024100082F83C60956372B6AB42A8BF2B469B0026
:10242000D36262B62046BDE8F84010F0EBBB00BFB7
:1024300040F6185038B52121C0F2020016F09CFF7A
:1024400049F2E860C1F6FF704DF6FC3413F0E0FB92
:10245000C2F200044EF21C312046C2F2000110F01C
:1024600085FB43F2B441C2F2000149F2FC224CF672
:102470006C00C2F20000C1F6FF7244F29043C2F257
:1024800000034D68C570927D4A60002063259D63FE
:1024900083F83C00586372B6AA42A8BF2A4692004D
:1024A000DA6262B62046BDE8384010F0ABBB00BF30
:1024B00040F63C5038B51D21C0F2020016F05CFF1A
:1024C00049F2E860C1F6FF704DF6FC3413F0A0FB52
:1024D000C2F200044AF68C712046C2F2000110F0EC
:1024E00045FB43F2B441C2F2000149F2FC224CF632
:1024F0006C00C2F20000C1F6FF7244F29043C2F2D7
:1025000000034D68C570127D4A60002063259D63FD
:1025100083F83C00586372B6AA42A8BF2A469200CC
:10252000DA6262B62046BDE8384010F06BBB00BFEF
:1025300040F65C5070B51C21C0F2020016F01CFF82
:1025400049F2E860C1F6FF7013F062FB4BF634719C
:102550004DF6FC30C2F20001C2F2000010F006FBA2
:1025600049F24432C1F6FF7243F2B441C2F20001B3
:1025700012784E684A604CF66C0044F29043C2F206
:1025800000036321C2F20000002501248A42067084
:1025900083F83C505C6399630EDC5AB1920072B6CA
:1025A000DA6262B64DF6FC30C2F20000BDE870405F
:1025B00010F028BB0422F2E74FF4C672EFE700BF29
:1025C00040F67C5070B51C21C0F2020016F0D4FE1B
:1025D00049F2E860C1F6FF7013F01AFB4AF6406159
:1025E0004DF6FC30C2F20001C2F2000010F0BEFA5B
:1025F00049F24432C1F6FF7243F2B441C2F2000123
:1026000012784E684A604CF66C0044F29043C2F275
:1026100000036321C2F20000002501248A420670F3
:1026200083F83C505C6399630EDC5AB1920072B639
:10263000DA6262B64DF6FC30C2F20000BDE87040CE
:1026400010F0E0BA0422F2E74FF4C672EFE700BFE1
:1026500040F69C5008B5C0F202001D2116F08CFE19
:1026600049F2FC23C1F6FF7393F82230D3B144F250
:10267000F413C2F20003FE21986C03681B689847AC
:1026800040F29C600F21C0F2020016F075FE4FF67A
:102690000F6015F0E7FF40F21870C0F202000F2142
:1026A00016F06AFE49F2E860C1F6FF70BDE8084026
:1026B00013F0AEBA40F6BC5008B5C0F202001B21C0
:1026C00016F05AFE49F2FC23C1F6FF7393F822304C
:1026D000D3B144F2F413C2F20003FF21986C0368F3
:1026E0001B68984740F29C600F21C0F2020016F070
:1026F00043FE4FF60F7015F0B5FF40F21870C0F2B0
:1027000002000F2116F038FE49F2E860C1F6FF70B2
:10271000BDE8084013F07CBA40F6D85008B5C0F2C6
:102720000200142116F028FE49F2FC23C1F6FF73C3
:1027300093F82230D3B144F2F413C2F20003FC2127
:10274000986C03681B68984740F29C600F21C0F2A8
:10275000020016F011FE4FF60F4015F083FF40F215
:102760001870C0F202000F2116F006FE49F2E86070
:10277000C1F6FF70BDE8084013F04ABA40F6F050C9
:1027800008B5C0F20200152116F0F6FD49F2FC234F
:10279000C1F6FF7393F82230D3B144F2F413C2F2BE
:1027A0000003F821986C03681B68984740F29C600E
:1027B0000F21C0F2020016F0DFFD4FF60F0015F0FA
:1027C00051FF40F21870C0F202000F2116F0D4FD44
:1027D00049F2E860C1F6FF70BDE8084013F018BA8E
:1027E00040F6086008B5C0F20200182116F0C4FDDA
:1027F00049F2FC23C1F6FF7393F82230D3B144F2BF
:10280000F413C2F20003FB21986C03681B6898471D
:1028100040F29C600F21C0F2020016F0ADFD4FF6B1
:102820000F3015F01FFF40F21870C0F202000F21A8
:1028300016F0A2FD49F2E860C1F6FF70BDE808405D
:1028400013F0E6B940F6246008B5C0F20200152185
:1028500016F092FD49F2FC23C1F6FF7393F8223083
:10286000D3B144F2F413C2F20003FA21986C036866
:102870001B68984740F29C600F21C0F2020016F0DE
:102880007BFD4FF60F2015F0EDFE40F21870C0F200
:1028900002000F2116F070FD49F2E860C1F6FF70EA
:1028A000BDE8084013F0B4B940F63C6008B5C0F28A
:1028B0000200162116F060FD49F2FC23C1F6FF73F9
:1028C00093F82230CBB14EF28070C2F200004FF28A
:1028D0000F6112F03BF840F2AC601421C0F202002C
:1028E00016F04AFD4FF20F6015F0BCFE40F2187072
:1028F000C0F202000F2116F03FFD49F2E860C1F678
:10290000FF70BDE8084013F083B900BF10B504465E
:1029100040F65460C0F20200152116F02DFD49F278
:10292000FC23C1F6FF7393F82230F3B1240404F4BE
:10293000FE0444F4734444F002044EF280702146D5
:10294000C2F2000012F002F840F2AC601421C0F2B2
:10295000020016F011FD204615F084FE40F21870BA
:10296000C0F202000F2116F007FD49F2E860C1F63F
:10297000FF70BDE8104013F04BB900BF2DE9F041E6
:10298000804640F66C600F46C0F20200152116F03A
:10299000F3FC49F2FC23C1F6FF7393F822303BB9F4
:1029A00049F2E860C1F6FF70BDE8F04113F030B9BC
:1029B00044F2F415C2F20005F021A86C0368DB6C48
:1029C000984757B1444608EB0706A86C14F8011B5A
:1029D00003681B689847A642F7D1A86C0368F721E3
:1029E000DB6C984740F29C600F21C0F2020016F0A9
:1029F000C3FC39464046002215F088FE40F21870AC
:102A0000C0F202000F2116F0B7FC49F2E860C1F6EF
:102A1000FF70BDE8F04113F0FBB800BF40F68460E2
:102A200008B5C0F20200102116F0A6FC49F2FC2302
:102A3000C1F6FF7393F82230CBB14EF28070C2F230
:102A400000004FF60F2111F081FF40F2AC6014211D
:102A5000C0F2020016F090FC4FF60F2015F002FEB7
:102A600040F21870C0F202000F2116F085FC49F206
:102A7000E860C1F6FF70BDE8084013F0C9B800BFB8
:102A800040F6986008B5C0F20200162116F074FCFA
:102A900049F2FC23C1F6FF7393F82230CBB14EF21A
:102AA0008070C2F200004FF60F7111F04FFF40F23C
:102AB000AC601421C0F2020016F05EFC4FF60F70FD
:102AC00015F0D0FD40F21870C0F202000F2116F090
:102AD00053FC49F2E860C1F6FF70BDE8084013F00E
:102AE00097B800BF40F6B06008B5C0F202000F21F1
:102AF00016F042FC49F2FC23C1F6FF7393F8223032
:102B0000CBB14EF28070C2F200004FF60F4111F0CF
:102B10001DFF40F2AC601421C0F2020016F02CFC44
:102B20004FF60F4015F09EFD40F21870C0F2020003
:102B30000F2116F021FC49F2E860C1F6FF70BDE8F4
:102B4000084013F065B800BF40F6C06008B5C0F299
:102B50000200102116F010FC49F2FC23C1F6FF73AD
:102B600093F82230CBB14EF28070C2F200004FF6E3
:102B70000F0111F0EBFE40F2AC601421C0F2020034
:102B800016F0FAFB4FF60F0015F06CFD40F21870CE
:102B9000C0F202000F2116F0EFFB49F2E860C1F627
:102BA000FF70BDE8084013F033B800BF40F6D460B2
:102BB00008B5C0F20200182116F0DEFB49F2FC2332
:102BC000C1F6FF7393F82230CBB14EF28070C2F29F
:102BD00000004FF60F6111F0B9FE40F2AC60142115
:102BE000C0F2020016F0C8FB4FF60F6015F03AFD78
:102BF00040F21870C0F202000F2116F0BDFB49F23E
:102C0000E860C1F6FF70BDE8084013F001B800BFEE
:102C100038B5044640F6F0600D46C0F202001021BF
:102C200016F0AAFB49F2FC23C1F6FF7393F8223099
:102C3000DBB14EF2807000232A46C2F2000021462A
:102C400011F0C2FE40F2AC601421C0F2020016F096
:102C500093FB29462046002215F058FD40F21870DB
:102C6000C0F202000F2116F087FB49F2E860C1F6BE
:102C7000FF70BDE8384012F0CBBF00BF40F60470D3
:102C800008B5C0F20200132116F076FB49F2FC23CE
:102C9000C1F6FF7393F82230CBB14EF28070C2F2CE
:102CA00000004FF60F3111F051FE40F2AC601421DC
:102CB000C0F2020016F060FB4FF60F3015F0D2FCA8
:102CC00040F21870C0F202000F2116F055FB49F2D5
:102CD000E860C1F6FF70BDE8084012F099BF00BF80
:102CE00038B5054612F036FF0446284612F090FF2C
:102CF000204438BD10B440F21C540023C0F202043A
:102D00004172026104600372C36041B1194600E080
:102D1000026942F82310427A01339A42F8DC40F209
:102D20008853C2F201031A680AB90CE01A465369C3
:102D3000002BFBD15061002343618380C3808372E9
:102D40005DF8044B70471860F5E700BF10B40368E6
:102D500041681A780C78417A037A0C4202EA03023D
:102D60001AD0837A03F003030AB143F0040343F05B
:102D700008039A10082B82722AD8072B22D2032B21
:102D80002ED011D9042B13D0062B14D1C3685DF8B3
:102D9000044B023BC3607047837A03F00303002AAD
:102DA000E7D043F00403E4E7012B0BD0022B02D160
:102DB000C368013BC3605DF8044B70470D2BF7D02F
:102DC0000E2BF8D1C3685DF8044B0133C360704724
:102DD0000C2B05D0F2D8092BD8D00B2BE8D0EAE782
:102DE000C3685DF8044B0233C360704708B54FF207
:102DF0007453C2F20003D3F8EC00FFF7A7FF08BD3D
:102E000008B54FF27453C2F20003D3F8E800FFF79D
:102E10009DFF08BD08B54FF27453C2F20003D3F80A
:102E2000E400FFF793FF08BD08B54FF27453C2F2F8
:102E30000003D3F8E000FFF789FF08BD08B54FF2A3
:102E40007453C2F20003D3F8DC00FFF77FFF08BD24
:102E500008B54FF27453C2F20003D3F8D800FFF75D
:102E600075FF08BD08B54FF27453C2F20003D3F8E2
:102E7000D400FFF76BFF08BD08B54FF27453C2F2E0
:102E80000003D3F8D000FFF761FF08BD08B54FF28B
:102E90007453C2F20003D3F8CC00FFF757FF08BD0C
:102EA00008B54FF27453C2F20003D3F8C800FFF71D
:102EB0004DFF08BD08B54FF27453C2F20003D3F8BA
:102EC000C400FFF743FF08BD08B54FF27453C2F2C8
:102ED0000003D3F8C000FFF739FF08BD08B54FF273
:102EE0007453C2F20003D3F8BC00FFF72FFF08BDF4
:102EF00008B54FF27453C2F20003D3F8B800FFF7DD
:102F000025FF08BD08B54FF27453C2F20003D3F891
:102F1000B400FFF71BFF08BD08B54FF27453C2F2AF
:102F20000003D3F8B000FFF711FF08BD08B54FF25A
:102F30007453C2F20003D3F8AC00FFF707FF08BDDB
:102F400008B54FF27453C2F20003D3F8A800FFF79C
:102F5000FDFE08BD08B54FF27453C2F20003D3F86A
:102F6000A400FFF7F3FE08BD08B54FF27453C2F298
:102F70000003D3F8A000FFF7E9FE08BD08B54FF243
:102F80007453C2F20003D3F89C00FFF7DFFE08BDC4
:102F900008B54FF27453C2F20003D3F89800FFF75C
:102FA000D5FE08BD08B54FF27453C2F20003D3F842
:102FB0009400FFF7CBFE08BD08B54FF27453C2F280
:102FC0000003D3F89000FFF7C1FE08BD08B54FF22B
:102FD0007453C2F20003D3F88C00FFF7B7FE08BDAC
:102FE00008B54FF27453C2F20003D3F88800FFF71C
:102FF000ADFE08BD08B54FF27453C2F20003D3F81A
:103000008400FFF7A3FE08BD08B54FF27453C2F267
:103010000003D3F88000FFF799FE08BD08B54FF212
:103020007453C2F20003D86FFFF790FE08BD00BFD3
:1030300008B54FF27453C2F20003986FFFF786FE93
:1030400008BD00BF08B54FF27453C2F20003586FB9
:10305000FFF77CFE08BD00BF08B54FF27453C2F203
:103060000003186FFFF772FE08BD00BF08B54FF2EE
:103070007453C2F20003D86EFFF768FE08BD00BFAC
:1030800008B54FF27453C2F20003986EFFF75EFE6C
:1030900008BD00BF08B54FF27453C2F20003586E6A
:1030A000FFF754FE08BD00BF08B54FF27453C2F2DB
:1030B0000003186EFFF74AFE08BD00BF08B54FF2C7
:1030C0007453C2F20003D86DFFF740FE08BD00BF85
:1030D00008B54FF27453C2F20003986DFFF736FE45
:1030E00008BD00BF08B54FF27453C2F20003586D1B
:1030F000FFF72CFE08BD00BF08B54FF27453C2F2B3
:103100000003186DFFF722FE08BD00BF08B54FF29F
:103110007453C2F20003D86CFFF718FE08BD00BF5D
:1031200008B54FF27453C2F20003986CFFF70EFE1D
:1031300008BD00BF08B54FF27453C2F20003586CCB
:10314000FFF704FE08BD00BF08B54FF27453C2F28A
:103150000003186CFFF7FAFD08BD00BF08B54FF279
:103160007453C2F20003D86BFFF7F0FD08BD00BF37
:1031700008B54FF27453C2F20003986BFFF7E6FDF7
:1031800008BD00BF08B54FF27453C2F20003586B7C
:10319000FFF7DCFD08BD00BF08B54FF27453C2F263
:1031A0000003186BFFF7D2FD08BD00BF08B54FF252
:1031B0007453C2F20003D86AFFF7C8FD08BD00BF10
:1031C00008B54FF27453C2F20003986AFFF7BEFDD0
:1031D00008BD00BF08B54FF27453C2F20003586A2D
:1031E000FFF7B4FD08BD00BF08B54FF27453C2F23B
:1031F0000003186AFFF7AAFD08BD00BF08B54FF22B
:103200007453C2F20003D869FFF7A0FD08BD00BFE8
:1032100008B54FF27453C2F200039869FFF796FDA8
:1032200008BD00BF08B54FF27453C2F200035869DD
:10323000FFF78CFD08BD00BF08B54FF27453C2F212
:1032400000031869FFF782FD08BD00BF08B54FF203
:103250007453C2F20003D868FFF778FD08BD00BFC1
:1032600008B54FF27453C2F200039868FFF76EFD81
:1032700008BD00BF08B54FF27453C2F2000358688E
:10328000FFF764FD08BD00BF08B54FF27453C2F2EA
:1032900000031868FFF75AFD08BD00BF1D2810B5D0
:1032A0000B4600F0E983024622D92C2800F0648105
:1032B0003FD8242800F0EE8340F2A880282800F0B0
:1032C000748300F2D680262800F0F58140F2D58282
:1032D0004FF27454C2F2000442F67D71C0F2000154
:1032E00004222720C4F89C3013F0FAF9012010BD05
:1032F0000E2800F097833AD8062800F0A1836CD9F5
:103300000A2800F0058300F20781082800F07E817A
:1033100040F275824FF27454C2F2000443F2D511A8
:10332000C0F2000104220920636213F0D9F90120E0
:1033300010BD342800F0BD8336D8302800F06383F8
:1033400000F2D6802E2800F0528140F201824FF226
:103350007454C2F2000442F6DD61C0F2000104229E
:103360002F20C4F8BC3013F0BBF9012010BD152884
:1033700000F0748364D9192800F0FA8100F2A58066
:10338000172800F08A8140F2D1824FF27454C2F2C1
:10339000000443F2A901C0F20001042218202366B0
:1033A00013F09EF9012010BD382800F0CE8275D8A8
:1033B000362800F0398140F27F824FF27454C2F215
:1033C000000442F63D61C0F2000104223720C4F837
:1033D000DC3013F085F9012010BD022800F00182D5
:1033E00040F27881042800F04B8140F2BD824FF218
:1033F0007454C2F2000443F22521C0F200010422F9
:103400000520636113F06CF9012010BD202800F045
:10341000448240F28981222800F0238140F2D48244
:103420004FF27454C2F2000442F6CD71C0F20001B2
:1034300004222320C4F88C3013F052F9012010BD6F
:10344000112800F0B18140F25A81132800F0FB806E
:1034500040F2B8814FF27454C2F2000443F2F90111
:10346000C0F2000104221420236513F039F9012071
:1034700010BD2A2800F0AC8040F2E0814FF2745475
:10348000C2F2000442F62D71C0F2000104222B208A
:10349000C4F8AC3013F024F9012010BD3A2800F034
:1034A0008880C0F072823B2840F06D824FF27454E5
:1034B000C2F2000442F6ED51C0F200010422C4F849
:1034C000EC3013F00DF9012010BD1B2863D040F241
:1034D0008B824FF27454C2F2000443F25901C0F2DD
:1034E000000104221C20236713F0FAF8012010BD0C
:1034F000322824D040F292814FF27454C2F2000478
:1035000042F68D61C0F2000104223320C4F8CC30B1
:1035100013F0E6F8012010BD0C281FD040F29E8168
:103520004FF27454C2F2000443F28511C0F200015C
:1035300004220D20636313F0D3F8012010BD4FF275
:103540007454C2F2000442F6A161C0F200010422E8
:10355000C4F8C83013F0C4F8012010BD4FF2745401
:10356000C2F2000443F29911C0F200010422236365
:1035700013F0B6F8012010BD4FF27454C2F20004EB
:1035800042F61971C0F200010422C4F8B03013F001
:10359000A7F8012010BD4FF27454C2F2000443F2A8
:1035A0006D01C0F200010422E36613F099F80120D6
:1035B00010BD4FF27454C2F2000442F60161C0F231
:1035C00000010422C4F8E83013F08AF8012010BD8D
:1035D0004FF27454C2F2000442F64171C0F200018D
:1035E0000422C4F8A83013F07BF8012010BD4FF27C
:1035F0007454C2F2000442F6F161C0F200010422E8
:10360000C4F8B83013F06CF8012010BD4FF27454B8
:10361000C2F2000443F2E911C0F200010422236265
:1036200013F05EF8012010BD4FF27454C2F2000492
:1036300042F65161C0F200010422C4F8D83013F000
:103640004FF8012010BD4FF27454C2F2000443F24F
:103650000D11C0F200010422E36413F041F80120CF
:1036600010BD4FF27454C2F2000442F6E171C0F290
:1036700000010422C4F8883013F032F8012010BD94
:103680004FF27454C2F2000443F23921C0F2000137
:10369000236113F025F8012010BD4FF27454C2F2DB
:1036A000000443F2BD01C0F200010422E36513F0FF
:1036B00017F8012010BD4FF27454C2F2000442F614
:1036C0009171C0F200010422C4F8983013F008F898
:1036D000012010BD002800F0FF80012840F0538138
:1036E0004FF27454C2F2000443F27521C0F200019B
:1036F00004220120636012F0F3FF012010BD0F28A7
:1037000000F0F880102840F03E814FF27454C2F26D
:10371000000443F24911C0F2000104221020236486
:1037200012F0DEFF012010BD1E282FD01F2840F010
:103730002A814FF27454C2F2000443F21D01C0F218
:10374000000104221F20E36712F0CAFF012010BD10
:103750004FF27454C2F2000442F60571C0F2000147
:1037600004222D20C4F8B43012F0BAFF012010BD9D
:103770004FF27454C2F2000443F29501C0F200010A
:103780000422636612F0ACFF012010BD4FF27454A6
:10379000C2F2000443F23101C0F200010422A36727
:1037A00012F09EFF012010BD4FF27454C2F20004CB
:1037B00043F23511C0F200010422636412F090FF5D
:1037C000012010BD4FF27454C2F2000443F22111E3
:1037D000C0F2000104221220A36412F081FF012034
:1037E00010BD4FF27454C2F2000443F26121C0F2E2
:1037F00000010422A36012F073FF012010BD4FF2FC
:103800007454C2F2000443F2FD11C0F2000104221C
:103810000720E36112F064FF012010BD4FF27454E1
:10382000C2F2000442F6B561C0F200010422312068
:10383000C4F8C43012F054FF012010BD4FF274548C
:10384000C2F2000442F65571C0F2000104222920A0
:10385000C4F8A43012F044FF012010BD4FF274549C
:10386000C2F2000443F2AD11C0F2000104220B20A9
:10387000E36212F035FF012010BD4FF27454C2F222
:10388000000442F6A571C0F2000104222520C4F80C
:10389000943012F025FF012010BD4FF27454C2F293
:1038A000000443F20901C0F200010422C4F8803090
:1038B00012F016FF012010BD4FF27454C2F2000442
:1038C00042F66561C0F2000104223520C4F8D4300C
:1038D00012F006FF012010BD4FF27454C2F2000432
:1038E00043F28921C0F200010422236012F0F8FEA5
:1038F000012010BD4FF27454C2F2000443F25D1176
:10390000C0F200010422E36312F0EAFE012010BDC0
:103910004FF27454C2F2000443F2C111C0F200012C
:103920000422A36212F0DCFE012010BD4FF2745499
:10393000C2F2000443F2D101C0F2000104221620B9
:10394000A36512F0CDFE012010BD4FF27454C2F2F7
:10395000000442F62961C0F200010422C4F8E030FC
:1039600012F0BEFE012010BD4FF27454C2F20004EA
:1039700043F24D21C0F2000104220320E36012F063
:10398000AFFE012010BD002010BD4FF27454C2F2F2
:10399000000442F61561C0F2000104223920C4F887
:1039A000E43012F09DFE012010BD4FF27454C2F2BB
:1039B000000442F66971C0F200010422C4F8A0308C
:1039C00012F08EFE012010BD4FF27454C2F20004BA
:1039D00042F6F571C0F2000104222120C4F88430BF
:1039E00012F07EFE012010BD4FF27454C2F20004AA
:1039F00043F28101C0F2000104221A20A36612F0F2
:103A00006FFE012010BD4FF27454C2F2000442F662
:103A1000C961C0F200010422C4F8C03012F060FE97
:103A2000012010BD4FF27454C2F2000443F2711130
:103A3000C0F200010422A36312F052FE012010BD67
:103A40004FF27454C2F2000443F21121C0F200019B
:103A50000422A36112F044FE012010BD4FF2745401
:103A6000C2F2000443F2E501C0F2000104226365E2
:103A700012F036FE012010BD4FF27454C2F2000461
:103A800043F24501C0F200010422636712F028FEF0
:103A9000012010BD4FF27454C2F2000442F6B97115
:103AA000C0F200010422C4F8903012F019FE012087
:103AB00010BD4FF27454C2F2000442F67961C0F2B4
:103AC00000010422C4F8D03012F00AFE012010BD1B
:103AD000F8B5044615460E460846022113F078F85C
:103AE0002846022113F074F840F6EC03C0F20F03ED
:103AF000012253F83600227200F50071216053F85C
:103B0000351062724DF2C04301F5007762F31F4336
:103B100000226760E260013BFDD190F8003291F82D
:103B2000002203F00103D20744BF43F00203DBB2DB
:103B3000A37221463046FFF7B1FB21462074284688
:103B4000FFF7ACFB237C184420742046F8BD00BF6F
:103B500010B5037C012B04462CD972B6E36862B61B
:103B6000002BB8BF033362699B1093420DDBA16940
:103B70008B4217DC237C012B20D972B6E06862B639
:103B80000028B8BF0330801010BD237F23B972B660
:103B90009200E26062B6EDE7A3699B0072B6E36053
:103BA00062B6E7E7237F002BF1D172B68900E160AE
:103BB00062B6DFE772B6FFF7C9F8CFE772B6204604
:103BC000FFF7C4F8DAE700BF091A49B238B581EA4D
:103BD000E175A5EBE175D5B100294FF000040BDBD1
:103BE0004DF6FC300134C2F200000021E4B20EF0C8
:103BF000DFFFAC42F4DB38BD4DF6FC300134C2F2DD
:103C000000000121E4B20EF0D3FFAC42F4DB38BD7A
:103C1000F8B544F29044C2F20004074604F12000D3
:103C2000FFF796FF4CF66C05C2F200054DF6FC3628
:103C3000C2F200064BF6F461E855C2F200013046CC
:103C40000EF094FF304602210EF0B8FF43F2B4426A
:103C500095F90030C2F20002002105205360A063F4
:103C600023EAE37384F83C10616372B68342A8BF11
:103C700003469B00E36262B6F8BD00BFF8B544F2AC
:103C80009044C2F20004074604F12000FFF760FFF1
:103C90004CF66C05C2F200054DF6FC36C2F2000689
:103CA00042F6A011E855C2F2000130460EF05EFF68
:103CB000304602210EF082FF43F2B44295F9023001
:103CC000C2F20002002108205360A06323EAE373DC
:103CD00084F83C10616372B68342A8BF03469B0020
:103CE000E36262B6F8BD00BFF8B544F29044C2F298
:103CF0000004074604F12000FFF72AFF4CF66C058C
:103D0000C2F200054DF6FC36C2F200064FF2B801D1
:103D1000E855C2F2000130460EF028FF304602217D
:103D20000EF04CFF43F2B44295F90330C2F20002A8
:103D3000002112205360A06323EAE37384F83C104F
:103D4000616372B68342A8BF03469B00E36262B61A
:103D5000F8BD00BFF8B544F29044C2F20004074633
:103D600004F12000FFF7F4FE4CF66C05C2F20005EA
:103D70004DF6FC36C2F200064CF2F821E855C2F2CC
:103D8000000130460EF0F2FE304602210EF016FF22
:103D900043F2B44295F90530C2F20002002103203B
:103DA0005360A06323EAE37384F83C10616372B646
:103DB0008342A8BF03469B00E36262B6F8BD00BF22
:103DC000F8B544F29044C2F20004074604F1200022
:103DD000FFF7BEFE4CF66C05C2F200054DF6FC3650
:103DE000C2F200064EF22811E855C2F20001304638
:103DF0000EF0BCFE304602210EF0E0FE95F92730B1
:103E00000022012123EAE373A16384F83C2062636A
:103E100072B68B42A8BF0B469B00E36262B6F8BD48
:103E200038B549F24434C1F6FF7440F6187049F2CF
:103E3000E8650B21C1F6FF75C0F2020015F09CFA8F
:103E4000217800230A22284611F0F4FE284611F0BA
:103E5000DFFE4BF63412C1F6FF724DF67833C2F234
:103E600000032178117000221A7038BD38B505465C
:103E700049F2E86440F624700A21C1F6FF74C0F2EA
:103E8000020015F079FA294600230A22204611F093
:103E9000D1FE204611F0BCFE07EE905A0023C4F27A
:103EA000C623F8EE676A07EE103A86EE870A00230B
:103EB00007EE903A4BF20063C2F2000330EE270A9D
:103EC000186807F009FE49F2FC23C1F6FF731D7163
:103ED00038BD00BF38B5054649F2E86440F6307099
:103EE0000C21C1F6FF74C0F2020015F045FA294614
:103EF00000230A22204611F09DFE204611F088FE84
:103F000007EE905A0023C4F2C623F8EE676A07EE64
:103F1000103A86EE870A002307EE903A4BF20063D0
:103F2000C2F2000330EE270A186807F0C1FE49F21A
:103F3000FC23C1F6FF735D7138BD00BF38B505467F
:103F400049F2E86440F640700D21C1F6FF74C0F2FA
:103F5000020015F011FA294600230A22204611F02A
:103F600069FE204611F054FE07EE905A0023C4F279
:103F7000C623F8EE676A07EE103A86EE870A00233A
:103F800007EE903A4BF20063C2F2000330EE270ACC
:103F9000186807F079FF49F2FC23C1F6FF739D71A1
:103FA00038BD00BF38B5054649F2E86440F65070A8
:103FB0000B21C1F6FF74C0F2020015F0DDF92946AD
:103FC00000230A22204611F035FE204611F020FE83
:103FD00007EE905A0023C4F2C623F8EE676A07EE94
:103FE000103A86EE870A002307EE903A4BF2006300
:103FF000C2F2000330EE270A186808F02FF849F2E1
:10400000FC23C1F6FF73DD7138BD00BF38B505462E
:1040100049F2E86440F65C700B21C1F6FF74C0F20F
:10402000020015F0A9F92946204611F093FD20461B
:1040300011F0EEFD07EE905A0023C4F2C623F8EE0D
:10404000E76A07EE103A86EE870A002307EE903AF9
:104050004BF20063C2F2000330EE270A186808F042
:10406000ABFB49F2FC23C1F6FF731D7238BD00BFE4
:1040700038B5054649F2E86440F668700E21C1F68D
:10408000FF74C0F2020015F077F92946204611F0BE
:1040900061FD204611F0BCFD49F2FC23C1F6FF731F
:1040A0005D7238BD38B5054649F2E86440F678706F
:1040B0000921C1F6FF74C0F2020015F05DF929462E
:1040C000204611F047FD204611F0A2FD07EE905A60
:1040D0000023C4F2482306EE103AF8EEE77A0023F4
:1040E000C4F2C82306EE903A77EE867A002387EE74
:1040F000A60A07EE103A4BF20063C2F2000330EE5C
:10410000070A186808F046FC49F2FC23C1F6FF7361
:104110009D7238BD38B5054649F2E86440F68470B2
:104120000B21C1F6FF74C0F2020015F025F92946F3
:1041300000230A22204611F07DFD204611F068FD83
:1041400007EE905A0023C4F2C623F8EE676A07EE22
:10415000103A86EE870A002307EE903A4BF200638E
:10416000C2F2000330EE270A186808F0FFFC49F29B
:10417000FC23C1F6FF73DD7238BD00BF38B50546BC
:1041800049F2E86440F690701321C1F6FF74C0F262
:10419000020015F0F1F8294600230A22204611F00A
:1041A00049FD204611F034FD07EE905A0023C4F279
:1041B000C623F8EE676A07EE103A86EE870A0023F8
:1041C00007EE903A4BF20063C2F2000330EE270A8A
:1041D000186808F005FA49F2FC23C1F6FF731D7355
:1041E00038BD00BF38B5054649F2E86440F6A47012
:1041F0001621C1F6FF74C0F2020015F0BDF8294681
:1042000000230A22204611F015FD204611F000FD82
:1042100007EE905A0023C4F2C623F8EE676A07EE51
:10422000103A86EE870A002307EE903A4BF20063BD
:10423000C2F2000330EE270A186808F0E5F849F2E8
:10424000FC23C1F6FF735D7338BD00BF38B505466A
:1042500049F2E86440F6BC701321C1F6FF74C0F265
:10426000020015F089F8294600230A22204611F0A1
:10427000E1FC204611F0CCFC07EE905A0023C4F27A
:10428000C623F8EE676A07EE103A86EE870A002327
:1042900007EE903A4BF20063C2F2000330EE270AB9
:1042A000186807F0C5FF49F2FC23C1F6FF739D7340
:1042B00038BD00BF38B5054649F2E86440F6D07015
:1042C0000E21C1F6FF74C0F2020015F055F8294620
:1042D00000230A22204611F0ADFC204611F098FC84
:1042E00007EE905A0023C4F2C623F8EE676A07EE81
:1042F000103A86EE870A002307EE903A4BF20063ED
:10430000C2F2000330EE270A186808F01BFD49F2DC
:10431000FC23C1F6FF73DD7338BD00BF30B5054621
:1043200049F2E86440F6E07083B0C1F6FF740E21F4
:10433000C0F2020015F020F8294600230A22204688
:1043400011F078FC204611F063FC49F2FC2407EEE2
:10435000905AC1F6FF740023F8EE676A07EE903AB0
:10436000B6EE007A637D627CE6EE877A44F2D04056
:10437000C2F2000001EE103A237D00EE903AFCEE0E
:10438000E77AB8EE411AF8EE600ACDED017AF2EE66
:10439000047A81EE271AE37C9DF80410C0EEA70A88
:1043A00000EE103AA37CB8EE400A0AF02DF825740E
:1043B00003B030BD30B5054649F2E86440F6F07010
:1043C00083B0C1F6FF741221C0F2020014F0D4FFD2
:1043D000294600230A22204611F02CFC204611F029
:1043E00017FC07EE905AF8EE676AB0EE087AC6EE50
:1043F000877A49F2FC24C1F6FF740022637D217C98
:1044000044F2D040C2F2000007EE102A01EE103A4A
:10441000237D77EE877A00EE903AFCEEE77AB8EEED
:10442000411AF8EE600ACDED017AF2EE047A81EEDF
:10443000271AE37C9DF80420C0EEA70A00EE103A8C
:10444000A37CB8EE400A09F0DFFF657403B030BD0D
:1044500030B5054649F2E86441F2040083B0C1F684
:10446000FF740F21C0F2020014F086FF29460023DA
:104470000A22204611F0DEFB204649F2FC24C1F658
:10448000FF7411F0C5FB07EE905A002307EE103AB7
:10449000637D627C217CF8EE677A01EE103A237D21
:1044A00077EE877A00EE903AFCEEE77AB8EE411AA2
:1044B000F8EE600ACDED017AF2EE047A81EE271A69
:1044C000E37C44F2D040C2F20000C0EEA70A00EE46
:1044D000103A9DF80430B8EE400A09F095FF003517
:1044E00018BF0125A57403B030BD00BF70B50646E6
:1044F00049F2E86541F214001321C1F6FF75C0F2DC
:10450000020049F2FC2414F037FFC1F6FF74314673
:1045100000230A22284611F08DFB284611F078FB73
:10452000637D627C217C01EE103A237D00EE903A9F
:10453000B8EE411AF8EE600AF2EE047A81EE271A1C
:1045400044F2D040A37CC2F20000C0EEA70A07EEFE
:10455000906AB8EE670A09F057FFE67470BD00BFB5
:1045600070B5064649F2E86541F228001021C1F60F
:10457000FF75C0F2020049F2FC2414F0FDFEC1F602
:10458000FF74314600230A22284611F053FB2846C7
:1045900011F03EFB637D627C217C01EE103A07EE58
:1045A000906AE37CF8EE670A00EE103AB8EE411A22
:1045B000F2EE047A44F2D040A37C81EE271AC2F2D4
:1045C0000000C0EEA70AB8EE400A09F01DFF2675EC
:1045D00070BD00BF70B5064649F2E86541F23C0087
:1045E0000F21C1F6FF75C0F2020049F2FC2414F05D
:1045F000C3FEC1F6FF74314600230A22284611F09B
:1046000019FB284611F004FB237D627C217C00EE1F
:10461000903A07EE906AE37CB8EE671A00EE103A23
:10462000F8EE600AF2EE047A44F2D040A37CC0EEC9
:10463000A70AC2F2000081EE271AB8EE400A09F07C
:10464000E3FE667570BD00BF10B5044641F24C0034
:104650001421C0F2020014F08FFE49F2E86000233A
:1046600021460A22C1F6FF7011F0E4FA49F2E8602F
:10467000C1F6FF7011F0CCFA07EE904A0023C4F2A5
:10468000C62307EE103AB8EE676A0023C6EE077A33
:1046900006EE903A77EEA67AB7EE007AF4EEC77A95
:1046A000F1EE10FA15DD44F2DC42C2F2000245F2EE
:1046B000606147F67053535249F2FC224BF65C712D
:1046C000C1F6FF72C1F6FF7145F2606094750B523E
:1046D00010BDF4EEE67AF1EE10FA33D445F6294334
:1046E000C4F20F6307EE103A27EE877ABDEEC77A61
:1046F00017EE103A03F5B34319331BB244F2DC4210
:10470000B7EE007AC2F2000245F26061F4EEC77AB9
:10471000F1EE10FA53521BDCF5EEC07AF1EE10FA0E
:1047200013D445F62943C4F20F6307EE103A67EE3F
:10473000877AFDEEE77A17EE903A03F5B343193323
:104740001BB2B9E745F69913D8E745F69913B3E7D5
:1047500047F67053B0E700BF38B5044641F2640035
:104760001321C0F2020014F007FE49F2E8600023B2
:1047700021460A22C1F6FF7011F05CFA49F2E860A6
:10478000C1F6FF7011F044FA07EE904A0023C4F21C
:10479000C62307EE103AB8EE676A0023C6EE077A22
:1047A00006EE903A77EEA67AB7EE007AF4EEC77A84
:1047B000F1EE10FA42DD44F6CD4143F2333272B6E7
:1047C00044F2DC43C2F2000345F25C6545F25E60F0
:1047D0005A53195262B6B7EE007AF4EEC77AF1EE88
:1047E00010FA15DD44F6CD4143F2333372B64BF681
:1047F0005C72C1F6FF7245F25C6545F25E60535330
:10480000115262B649F2FC23C1F6FF73DC7538BD64
:10481000F5EEC07AF1EE10FA2CD44CF6CD43C4F28A
:104820004C6307EE103A67EE877AFDEEE77A17EEF3
:10483000903AC3F5004109B21BB2D7E7F4EEE67A2D
:10484000F1EE10FA10D44CF6CD43C4F24C6307EEEF
:10485000103A27EE877ABDEEC77A17EE102AC2F516
:10486000004109B212B2AAE74FF40041CFF6FF713E
:104870000022A4E74FF40041CFF6FF710023B5E713
:1048800010B5044641F278001121C0F2020014F084
:1048900073FD49F2E860214600230A22C1F6FF7049
:1048A00011F0C8F949F2E860C1F6FF7011F0B0F9F3
:1048B00007EE904A0023C4F2C62306EE103AF8EE43
:1048C000675A0023C5EE867A4EF2F8124EF2B00116
:1048D000C2F20002C2F2000106EE903A4FF47E43AB
:1048E000C4F2FF6307EE103A77EEA67A4FF48033F6
:1048F000F4EEC77AF1EE10FA93618B612BDC4FF482
:104900007E43CCF2FF6307EE103AF4EEC77AF1EE85
:1049100010FA2BD4B0EE677ABEEEC87A17EE103AD2
:104920004FF47E40C4F2FF6007EE100AF4EEC77A3F
:10493000F1EE10FAD36124DC4FF47E43CCF2FF6336
:1049400007EE103AF4EEC77AF1EE10FA12D5002312
:10495000C8F2010303E00023C7F6FF73D36149F2F5
:10496000FC22C1F6FF72CB61147610BD0023C8F2A1
:104970000103D5E7B0EE677ABEEEC87A17EE103ABB
:10498000EDE70023C7F6FF73E9E700BF38B505463A
:1049900049F2E86441F28C001521C1F6FF74C0F2BF
:1049A000020014F0E9FC002329460A22204611F0F7
:1049B00041F9204611F02CF949F2FC23C1F6FF73AE
:1049C0005D7638BD38B5054649F2E86441F2A40089
:1049D0001121C1F6FF74C0F2020014F0CDFC0023D7
:1049E00029460A22204611F025F9204611F010F937
:1049F00049F2FC23C1F6FF739D7638BD38B50546F4
:104A000049F2E86441F2B8001121C1F6FF74C0F226
:104A1000020014F0B1FC002329460A22204611F0BE
:104A200009F9204611F0F4F849F2FC23C1F6FF73AE
:104A3000DD7638BD70B5064649F2E86541F2CC0036
:104A40001221C1F6FF75C0F2020049F2FC2414F0F5
:104A500093FCC1F6FF74314600230A22284611F068
:104A6000E9F8284611F0D4F8637F06EE106A07EEE5
:104A7000903A0023C4F2C62306EE903AF8EE677A25
:104A8000B8EE466AC7EEA60A002344F2D040C2F24E
:104A9000000086EE260A07EE103A70EE870A30EE26
:104AA000070A09F025F8267770BD00BF70B50646E5
:104AB00049F2E86541F2E0001421C1F6FF75C0F249
:104AC000020049F2FC2414F057FCC1F6FF74314691
:104AD00000230A22284611F0ADF8284611F098F874
:104AE000237F06EE106A07EE903A0023C4F2C62335
:104AF00006EE903AF8EE677AB8EE466A87EEA60AB6
:104B0000002344F2D040C2F20000C6EE260A07EEAF
:104B1000103A30EE070A70EE870A08F0E9FF667770
:104B200070BD00BF70B5064649F2E86541F2F80075
:104B30000C21C1F6FF75C0F2020049F2FC2414F00A
:104B40001BFCC1F6FF74314600230A22284611F0EF
:104B500071F8284611F05CF894F91F3007EE106ADE
:104B600007EE903A0023C4F2482306EE103AF8EE1E
:104B7000E77AB8EE477A77EE867A37EE067A002340
:104B8000C4F2C82306EE903A77EEA77A37EE077A9A
:104B9000C7EEA60A44F2D040C2F2000087EE260A11
:104BA000F7EE007A70EEE70A30EE670A09F0D4F803
:104BB000A67770BD70B5064649F2E86541F2081067
:104BC0000E21C1F6FF75C0F2020049F2FC2414F078
:104BD000D3FBC1F6FF74314600230A22284611F0A8
:104BE00029F8284611F014F894F91E3007EE106ADF
:104BF00007EE903A0023C4F2482306EE103AF8EE8E
:104C0000E77AB8EE477A77EE867A37EE067A0023AF
:104C1000C4F2C82306EE903A77EEA77A37EE077A09
:104C200087EEA60A44F2D040C2F20000C7EE260A80
:104C3000F7EE007A30EE670A70EEE70A09F08CF8BA
:104C4000E67770BD38B5054649F2E86441F21810C0
:104C50000D21C1F6FF74C0F2020014F08DFB002399
:104C60000A222946204610F0E5FF204610F0D0FF2A
:104C700007EE905A0023C4F2C62306EE903AB8EE2F
:104C8000676A0023C6EE267A49F2FC22C1F6FF725B
:104C900082F8205007EE103A4BF2881377EE877AAD
:104CA000C1F6FF73C3ED007A38BD00BF38B50546C5
:104CB00049F2E86441F228101121C1F6FF74C0F2F4
:104CC000020014F059FB002329460A22204610F066
:104CD000B1FF204610F09CFF49F2FC23C1F6FF73A0
:104CE00083F8215038BD00BF38B5044649F2E86565
:104CF00041F23C101321C1F6FF75C0F2020014F01E
:104D00003BFB214600230A22284610F093FF284649
:104D100010F07EFF49F2FC230034C1F6FF7318BF88
:104D2000012483F8224038BD70B5064649F2E86593
:104D300041F25010C1F6FF750D21C0F202004BF296
:104D4000006414F019FBC2F20004314600230A2269
:104D5000284610F06FFF284610F05AFF20683146B1
:104D600007F016FE49F2FC23C1F6FF73206883F8B2
:104D70002360BDE8704006F0BDBB00BF2DE9F041E7
:104D800049F2FC24C1F6FF74002394F80480C4F2B5
:104D9000C62340F624702DED028BC0F2020008EE0F
:104DA000903A002308EE103AFBF7BEFC4046FBF7B2
:104DB000A9FC07EE908AF8EE677A4BF2006587EE61
:104DC000A80AC2F2000549F2E8662868C1F6FF7633
:104DD00030EE080A06F080FE677984F8048040F619
:104DE0003070C0F20200FBF79FFC3846FBF78AFCEC
:104DF00007EE907AF8EE677A286887EEA80A30EE18
:104E0000080A06F055FF94F80680677140F6407076
:104E1000C0F20200FBF788FC4046FBF773FC07EE8C
:104E2000908AF8EE677A286887EEA80A30EE080ABA
:104E300007F02AF8E77984F8068040F65070C0F24F
:104E40000200FBF771FC3846FBF75CFC07EE907A3A
:104E5000F8EE677A286887EEA80A30EE080A07F0AD
:104E6000FDF894F90880E77140F65C700B21C0F200
:104E7000020014F081FA4146304610F06BFE3046D5
:104E800010F0C6FE07EE908AF8EEE77A286887EE03
:104E9000A80A30EE080A07F08FFC94F90A7084F82B
:104EA000088040F678700921C0F2020014F064FA1C
:104EB0003946304610F04EFE304610F0A9FE07EE9F
:104EC000907A0023C4F2482306EE903AF8EEE77A8F
:104ED0000023C4F2C82377EEA67A07EE103A87EED5
:104EE000870A286830EE080A07F054FDE67AA772B0
:104EF00040F68470C0F20200FBF716FC3046FBF768
:104F000001FC07EE906AF8EE677A286887EEA80A37
:104F100030EE080A07F02AFE277BE67240F6907012
:104F2000C0F20200FBF700FC3846FBF7EBFB07EE94
:104F3000907AF8EE677A286887EEA80A30EE080AB9
:104F400007F04EFB667B277340F6A470C0F20200A8
:104F5000FBF7EAFB3046FBF7D5FB07EE906AF8EE6D
:104F6000677A286887EEA80A30EE080A07F04CFA3C
:104F7000A77B667340F6BC70C0F20200FBF7D4FB5F
:104F80003846FBF7BFFB07EE907AF8EE677A2868A1
:104F900087EEA80A30EE080A07F04AF9E67BA77305
:104FA00040F6D070C0F20200FBF7BEFB3046FBF7C4
:104FB000A9FB07EE906AF8EE677A286887EEA80AE0
:104FC00030EE080A07F0BEFE207CE673FFF7A6F974
:104FD000607CFFF7EFF9A07CFFF73AFAE07CFFF77F
:104FE00085FA207DFFF7BCFA607DFFF7F3FAA07D1C
:104FF000FFF72AFBE07DFFF7AFFB207EFFF740FCC9
:10500000667E41F28C00C0F20200FBF78DFB304659
:10501000FBF778FBA77E667641F2A400C0F202009F
:10502000FBF782FB3846FBF76DFBE67EA77641F285
:10503000B800C0F20200FBF777FB3046FBF762FBDB
:10504000207FE676FFF7F6FC607FFFF72FFDA07F5D
:10505000FFF768FDE07FFFF7ADFD94F8206041F2B7
:105060001810C0F20200FBF75FFB3046FBF74AFB6B
:1050700007EE906AB8EE677A94F8218084F8206091
:10508000C7EE287A4BF2881341F22810C1F6FF735D
:10509000C0F2020037EE888A83ED008AFBF744FBFA
:1050A0004046FBF72FFB94F8227084F8218041F2F0
:1050B0003C10C0F20200FBF737FB3846FBF722FB3F
:1050C00094F8236084F8227041F25010C0F202007C
:1050D000FBF72AFB3046FBF715FB2868314607F043
:1050E00057FCBDEC028B286884F82360BDE8F041D2
:1050F00006F000BAF8B544F2F414C2F2000447F620
:105100001221A06C0368DB69984741F2C13541F276
:10511000193141F269420326C0F20005C0F20001D4
:10512000C0F2000240F6E54084F8646065602160EA
:10513000E260C0F2000040F6617340F66D4742F64F
:10514000114640F6E12540F65D5142F60D126061D0
:10515000C0F20003C0F20007C0F20006C0F2000572
:10516000C0F20001C0F2000242F6A900A36127616B
:10517000E6612562A160A262C0F2000042F64933F6
:1051800042F61D2742F67D4642F6E52542F6AD3150
:1051900042F68122C0F20001C0F20002E062C0F2D9
:1051A0000003C0F20007C0F20006C0F2000541F2A1
:1051B0006010216462642363676300234FF6FF7706
:1051C000A663E563C0F2020084F84C3084F84E30E8
:1051D00084F84D30A365636584F8E93084F866305F
:1051E00084F8653084F8673084F86830E7652766AE
:1051F000FBF7A4FA0DF07AFD4EF28073C2F20003C1
:1052000047F2595447F2C16147F62902C0F200043F
:10521000C0F20001C0F2000247F68910C3F86841ED
:10522000C3F86411C3F87021C0F2000047F691275B
:1052300047F6C93642F67D1540F6696447F6D14116
:1052400040F6F152C3F87801C0F20007C0F2000640
:10525000C0F20005C0F20004C0F20001C0F200027A
:1052600040F67510C3F87C71C3F87461C3F88451BB
:10527000C3F88841C3F86C11C3F89021C0F2000054
:1052800042F27D7742F6450642F2E17542F2197428
:1052900042F2516142F2B562C0F20001C0F2000276
:1052A000C3F89401C0F20007C0F20006C0F2000586
:1052B000C0F2000441F27810C3F89871C3F89C6101
:1052C000C3F8A051C3F8A441C3F8A811C3F8AC2196
:1052D000C0F20200FBF732FA40F65803C2F20103B3
:1052E00047F2096EC0F2000E40F65007C3F800E026
:1052F000C2F2010747F2717EC0F2000E40F654047C
:10530000C7F800E0C2F2010447F6D50EC0F2000E65
:1053100040F62806C4F800E0C2F2010647F6092E5E
:10532000C0F2000E40F61802C6F800E0C2F2010218
:1053300047F6293EC0F2000E40F61400C2F800E025
:10534000C2F2010047F6494EC0F2000E40F63805A1
:10535000C0F800E0C2F2010540F63D2EC0F2000E9A
:1053600040F63001C5F800E0C2F2010140F6E97EE6
:10537000C0F2000E40F62403C1F800E0C2F20103BF
:1053800047F6595EC0F2000E40F64C07C3F800E045
:10539000C2F2010740F6E16EC0F2000E40F634049E
:1053A000C2F20104C7F800E040F6B537C0F20007CA
:1053B00040F2FC76C2F20106276040F62C0240F271
:1053C000D577C2F20102C0F2000740F60C0040F6A9
:1053D000A504C2F20100C0F20004376040F64405A3
:1053E00040F6040140F6000340F63D07C2F2010515
:1053F000C2F20103C0F200071460C2F2010140F6DC
:105400000D1640F64D3440F6D512C0F20006C0F23B
:1054100000040760C0F2000241F298102E600C6098
:105420001A60C0F20200BDE8F840FBF787B900BF80
:1054300070B54BF20352C0EB8023CAF27E5282FB5E
:1054400003122DED048B1A44DB17C3EBA21349F2B0
:10545000FC249A1C0546C1F6FF7441F2B41082B0D8
:1054600003FB02F30026C0F2020008EE103A84F8B3
:105470002460FBF759F949F2E8600A2233462946CD
:10548000C1F6FF7010F0D6FBBAEEC68A41F2CC101E
:10549000C0F20200FBF748F918EE100A16F0B0FB54
:1054A00041EC100B49F2E8600321C1F6FF7010F0E7
:1054B00001FC41F2D010C0F20200FBF735F949F2CD
:1054C000E86094F92410C1F6FF7010F043FB41F23C
:1054D000CC100121C0F2020013F04EFF49F2E86047
:1054E0009FED550B0321C1F6FF7010F0E3FB41F275
:1054F000D8100221C0F2020013F03EFF40F2F34345
:10550000C3F6357307EE903A28EE278A18EE100A94
:1055100016F076FB41EC190B49F2E860B0EE490A4F
:10552000F0EE690A0321C1F6FF7010F0C3FB41F2EF
:10553000DC10C0F20200FBF7F7F8B0EE490AF0EE1B
:10554000690A49F2E8600321C1F6FF7010F0B2FB6E
:1055500049F2E860C1F6FF7010F05AFB4FF47E4349
:10556000C4F2FF6307EE903AB4EEE78AF1EE10FA68
:105570002FDC4FF47E43CCF2FF6307EE903AB4EE9B
:10558000E78AF1EE10FA47D4F0EE487AFEEEC87AD8
:1055900017EE902A4FF47E41C4F2FF6107EE901A95
:1055A0004EF2F813C2F20003B4EEE78AF1EE10FAFD
:1055B0009A613CDC4FF47E43CCF2FF6307EE903AF5
:1055C000B4EEE78AF1EE10FA2AD50023C8F20103FF
:1055D00007E04EF2F812C2F200020023C7F6FF7392
:1055E000936140F23462C2F201024FF20420126869
:1055F0000192C2F200004EF2B0014DF69C72C2F26E
:105600000001C2F20002019C046001208B61107055
:1056100002B0BDEC048B70BD0022C8F20102B9E7F4
:10562000F0EE487AFEEEC87A17EE903AD9E70023FA
:10563000C7F6FF73D5E700BF000000000000E03FA1
:105640002DE9F04340F23C54C0F202040FCC91B07B
:105650006D460FC50FCC0FC50FCC0FC594E80F00DA
:1056600085E80F0049F20031C1F6FF710D1F05F109
:1056700028074FF0FF3411F8013B83EA040210A819
:1056800002F00F0200EB820249F2FC2652F8402C95
:1056900082EA141484EA131303F00F0300EB83036C
:1056A000B94253F8403C83EA1414C1F6FF766FEA1E
:1056B0000404E0D140F23C5CC0F2020CBCE80F00F4
:1056C000EE46AEE80F00BCE80F00AEE80F00BCE805
:1056D0000F004BF63418AEE80F009CE80F00C1F63F
:1056E000FF7846F8044B98F800408EE80F00601EE3
:1056F00000EB8000C0004FF0FF3216F8013B83EA58
:10570000020110AC01F00F0104EB8101BE4251F81F
:10571000401C81EA121282EA131303F00F0310A94E
:1057200001EB830349F2FC2453F8403C83EA121254
:10573000C1F6FF746FEA0202DFD1C5F1010505EB86
:105740000009227014F8016B04EB0905284610F0DB
:10575000B3FC86423146284601D010F0C7FCBC425B
:10576000F0D141F2E0102821C0F2020013F004FE53
:1057700049F2E86000230A2298F80010C1F6FF7091
:1057800010F058FA41F20C200621C0F2020013F08A
:10579000F3FD98F80030013B03EB8303D90049F295
:1057A000E860023100231022C1F6FF7010F042FAC7
:1057B00049F2E860C1F6FF7010F02AFA002388F879
:1057C000003011B0BDE8F0832DE9F84340F20E69D6
:1057D000C2F2010941F238202DED028BC0F2020025
:1057E000FAF7A2FFB9F8003007EE103A43F233336C
:1057F000C4F2233308EE903AB8EEC77A43F233335B
:10580000C4F2A33308EE103A37EE287A49F2E8647E
:10581000C7EE087AC1F6FF7440F20867C2F20107CA
:1058200040F20C68C2F2010840F28C56C2F2010646
:105830004CF68465C2F2000517EE900A16F0E0F906
:1058400041EC100B0A21204610F034FA41F24020BE
:10585000C0F20200FAF768FF3B8807EE903AF8EED4
:10586000E77A77EEA87A87EE887A17EE100A16F0B4
:10587000C7F941EC100B0A21204610F01BFA41F247
:105880005020C0F20200FAF74FFFB8F8001020468F
:1058900010F060F941F25820C0F20200FAF744FF1C
:1058A0003188204610F056F941F26820C0F202001B
:1058B000FAF73AFF2988204610F04CF941F280208F
:1058C000C0F20200FAF730FF4DF22433C2F20003B7
:1058D0000A2219682046002310F0ACF941F28C200E
:1058E000C0F20200FAF720FF42F64C13C2F20003A6
:1058F0000A2219682046002310F09CF941F29C20EE
:10590000C0F20200FAF710FF42F68C33C2F2000335
:105910000A2219682046002310F08CF941F2A820D1
:10592000C0F20200FAF700FF4BF20063C2F200037C
:10593000186807F0F3FA0146204610F00BF92046EC
:1059400010F066F9BDEC028BB9F80030B8F8002011
:105950003B80002332802B80BDE8F88341F2BC20DD
:1059600038B5C0F20200FAF7DFFE49F2F323C1F6C0
:10597000FF7349F2FC241878FAF7B2FE41F2CC200A
:10598000C0F20200FAF7D0FE49F24433C1F6FF73C9
:10599000C1F6FF741878FAF7A3FE49F2E86541F200
:1059A000D420C1F6FF75C0F20200FAF7BDFE002355
:1059B00010222168284610F03DF9284610F028F9F9
:1059C00041F2E420C0F20200FAF7AEFE2079FAF7C5
:1059D00087FE41F2EC20C0F20200FAF7A5FE6079E2
:1059E000FAF77EFE41F2F820C0F20200FAF79CFEC0
:1059F000A079FAF775FE41F20430C0F20200FAF71E
:105A000093FEE079FAF76CFE41F21030C0F202002A
:105A1000FAF78AFE94F90810284610F09BF82846F9
:105A200010F0F6F841F21C30C0F20200FAF77CFEEA
:105A300094F90910284610F08DF8284610F0E8F87F
:105A400041F22830C0F20200FAF76EFE94F90A1013
:105A5000284610F07FF8284610F0DAF841F230308E
:105A6000C0F20200FAF760FEE07AFAF739FE41F27E
:105A70003C30C0F20200FAF757FE207BFAF730FE06
:105A800041F25030C0F20200FAF74EFE607BFAF7A6
:105A900027FE41F26830C0F20200FAF745FEA07B13
:105AA000FAF71EFE41F27C30C0F20200FAF73CFE2B
:105AB000E07BFAF715FE41F28830C0F20200FAF7F7
:105AC00033FE207CFAF70CFE41F29C30C0F202005B
:105AD000FAF72AFE607CFAF703FE41F2B430C0F216
:105AE0000200FAF721FEA17C284610F033F8284680
:105AF00010F08EF841F2C830C0F20200FAF714FE3E
:105B0000E07CFAF7EDFD41F2E030C0F20200FAF776
:105B10000BFE207DFAF7E4FD41F2F430C0F2020002
:105B2000FAF702FE607DFAF7DBFD41F20840C0F2B1
:105B30000200FAF7F9FDA07DFAF7D2FD41F21C4010
:105B4000C0F20200FAF7F0FDE07DFAF7C9FD41F27C
:105B50003040C0F20200FAF7E7FD207EFAF7C0FD00
:105B600041F24040C0F20200FAF7DEFD607EFAF733
:105B7000B7FD41F25440C0F20200FAF7D5FDA07E15
:105B8000FAF7AEFD41F26440C0F20200FAF7CCFD34
:105B9000E07EFAF7A5FD41F27440C0F20200FAF788
:105BA000C3FD207FFAF79CFD41F28840C0F202005D
:105BB000FAF7BAFD607FFAF793FD41F29C40C0F21C
:105BC0000200FAF7B1FD94F91E1028460FF0C2FF4B
:105BD000284610F01DF841F2A840C0F20200FAF782
:105BE000A3FD94F91F1028460FF0B4FF284610F0CB
:105BF0000FF841F2B440C0F20200FAF795FD94F8B4
:105C00002000FAF76DFD41F2C040C0F20200FAF741
:105C10008BFD94F82100FAF763FD41F2D040C0F209
:105C20000200FAF781FD94F8221028460FF092FF47
:105C300028460FF0EDFF41F2E440C0F20200FAF70F
:105C400073FD94F82300FAF74BFD41F2F840C0F2DF
:105C50000200FAF769FD94F9241028460FF07AFF44
:105C60002846BDE838400FF0D3BF00BFF0B549F279
:105C70004435C1F6FF759BB02E781AAB013E06EB9A
:105C80008606C3F16B0303EBC6060DF1FF340DF17D
:105C90002707301910F010FA04F8010FA742F8D1C5
:105CA00040F23C54C0F202040FCC0AAE37460FC794
:105CB0000FCC0FC70FCC0FC794E80F004FF0FF3485
:105CC00087E80F0001A911F8013B83EA04021AA832
:105CD00002F00F0200EB8202B14252F8402C82EA3D
:105CE000141484EA131303F00F0300EB830353F837
:105CF000403C83EA14146FEA0404E4D141F20450F6
:105D00001321C0F2020013F037FB009E49F2E86055
:105D1000002310223146C1F6FF700FF08BFF41F2D5
:105D200018500521C0F2020013F026FB49F2E8608A
:105D3000C1F6FF700023102221460FF07BFFA64220
:105D40000AD041F23850C0F20200FAF7F7FC1BB05B
:105D5000BDE8F040FFF702BE2E7849F2FB24C1F601
:105D6000FF74013E06EB8606C4F1020303EBC60690
:105D700004F12807301910F09FF904F8010FBC4214
:105D8000F8D141F22050C0F20200FAF7CDFC49F2FE
:105D9000E860297800230A22C1F6FF700FF04AFF5D
:105DA0001BB0BDE8F040FFF7D9BD00BF38B549F2E0
:105DB0004434C1F6FF7441F2605049F2E865C1F61F
:105DC000FF750B21C0F2020013F0D6FA21780023F0
:105DD0000A2228460FF02EFF28460FF019FF2178DF
:105DE000012010F083F9BDE83840FFF73FBF00BF46
:105DF0002DE9F04140F23465C2F2010582B044F26F
:105E000018062B680093C2F20006009B32689B1AAA
:105E1000B3F5487F00F2508243F2B444C2F200046A
:105E20004EF66060C2F200000CF018FF44F29040A1
:105E3000C2F20000FDF78CFE236843F2B44898429A
:105E40000746C2F2000800F3C384C0F299849F425F
:105E500027D049F2F328FBB2C1F6FF78184688F83C
:105E60000030FFF7E5FA41F23C60C0F20200FAF7B9
:105E70005BFC98F80000FAF745FC4CF240014DF647
:105E8000FC30C2F20001C2F200000CF06FFE4DF6D1
:105E9000FC30C2F200000CF0B5FE2B680193019BB0
:105EA00033604EF66060C2F2000027600CF014FF11
:105EB000002840F059824EF26815C2F200054EF6F5
:105EC0007060C2F200000CF0C9FE44F2B040C2F2B1
:105ED0000000FDF73DFE06464DF6FC30C2F2000024
:105EE0000CF060FE854200F030824DF6FC30C2F2CC
:105EF00000000CF057FE4BF6D023C1F6FF7383422F
:105F000000F001854DF6FC30C2F200000CF04AFEB4
:105F100042F2F853C2F20003834200F002854DF6CC
:105F2000FC30C2F200000CF03DFE4BF2B053C2F266
:105F30000003834200F03E844DF6FC30C2F20000C4
:105F40000CF030FE4CF68863C2F20003834200F08E
:105F500028854DF6FC30C2F200000CF023FE4EF214
:105F60005C33C2F20003834200F036854DF6FC300C
:105F7000C2F200000CF016FE42F65013C2F200030B
:105F8000834200F072854DF6FC30C2F200000CF046
:105F900009FE43F21803C2F20003834200F0D284E8
:105FA0004DF6FC30C2F200000CF0FCFD4BF618037D
:105FB000C1F6FF73834200F0A2854DF6FC30C2F2B9
:105FC00000000CF0EFFD4CF26863C2F20003834264
:105FD00000F0BA854DF6FC30C2F200000CF0E2FD94
:105FE0004EF68063C2F20003834200F0D5854DF681
:105FF000FC30C2F200000CF0D5FD4BF27073C2F21F
:106000000003834200F0ED854DF6FC30C2F2000043
:106010000CF0C8FD42F64863C2F20003834200F070
:1060200005864DF6FC30C2F200000CF0BBFD4CF2D0
:106030008C13C2F20003834200F01D864DF6FC3043
:10604000C2F200000CF0AEFD4DF20823C2F20003D4
:10605000834200F035864DF6FC30C2F200000CF0B1
:10606000A1FD4BF26053C2F20003834200F04D8663
:106070004DF6FC30C2F200000CF094FD4DF60C73AE
:10608000C2F20003834200F086864DF6FC30C2F275
:1060900000000CF087FD4DF67403C2F2000383424A
:1060A00000F0D5864DF6FC30C2F200000CF07AFD0F
:1060B0004FF20823C2F20003834200F0E6864DF659
:1060C000FC30C2F200000CF06DFD4CF66853C2F2D9
:1060D0000003834200F0CA864DF6FC30C2F2000095
:1060E0000CF060FD42F26473C2F20003834200F0E0
:1060F000DB864DF6FC30C2F200000CF053FD4CF292
:10610000A823C2F20003834200F0DD864DF6FC3086
:10611000C2F200000CF046FD4DF62833C2F2000337
:10612000834200F0EE864DF6FC30C2F200000CF027
:1061300039FD4BF2E803C1F6FF73834200F0D286CB
:106140004DF6FC30C2F200000CF02CFD43F2CC23E3
:10615000C2F20003834200F0AB874DF6FC30C2F27E
:1061600000000CF01FFD4BF2FC63C1F6FF7383428D
:1061700000F08F874DF6FC30C2F200000CF012FDEB
:106180004EF2AC33C2F20003834200F073874DF647
:10619000FC30C2F200000CF005FD4CF6D803C2F250
:1061A0000003834200F057874DF6FC30C2F2000036
:1061B0000CF0F8FC4EF26063C2F20003834200F080
:1061C0003B874DF6FC30C2F200000CF0EBFC4CF2C9
:1061D000B863C2F20003834200F0B7804DF6FC3092
:1061E000C2F200000CF0DEFC44F2E023C2F2000335
:1061F000834200F00D874DF6FC30C2F200000CF037
:10620000D1FC43F2F073C2F20003834200F0F18646
:106210004DF6FC30C2F200000CF0C4FC4CF61C033E
:10622000C2F20003834200F0D5864DF6FC30C2F284
:1062300000000CF0B7FC4BF23813C1F6FF73834239
:1062400000F0B9864DF6FC30C2F200000CF0AAFC5A
:106250004AF62813C2F200038342636800F09D8669
:1062600043F2B4479E42C2F2000700F3908616DA6A
:1062700041F27C50C0F20200FAF756FA49F2E860A7
:106280003146C1F6FF70FCF72BFDF0B23979FDF70E
:106290009BFC4DF6FC30C2F200000CF0B9FC4EF64F
:1062A0007060C2F2000066600CF016FD002840F03D
:1062B000948202B0BDE8F0814DF6FC30C2F20000DD
:1062C0000CF070FC42F21473C2F2000383427FF4BC
:1062D000A3AD41F6B82044F29047C2F20007C0F2E5
:1062E0000200FAF72BFA07F12000FDF731FC4CF61B
:1062F0006C08C2F200084BF6F46188F828004DF6ED
:10630000FC30C2F20001C2F200000CF02FFC4DF68E
:10631000FC300221C2F2000043F2B4440CF04EFC07
:10632000C2F2000498F90030636000220521B963CD
:1063300023EAE37387F83C207A6372B68B42A8BFE6
:106340000B469B00FB6262B66AE563689E42A6D07C
:1063500049F24433C1F6FF734DF6FC30C2F200003F
:106360001E700CF04FFC9AE741F24C60C0F2020044
:10637000FAF7DAF94DF6FC30C2F200000CF012FC2C
:106380004EF26815C2F20005854200F048834DF6D2
:10639000FC30C2F200000CF005FC4BF22073C2F29C
:1063A0000003834200F046834DF6FC30C2F2000049
:1063B0000CF0F8FB4BF6D023C1F6FF73834200F0DC
:1063C00062834DF6FC30C2F200000CF0EBFB42F2AF
:1063D000F853C2F20003834200F060834DF6FC30B4
:1063E000C2F200000CF0DEFB4BF2B053C2F200032D
:1063F000834200F05E834DF6FC30C2F200000CF0E8
:10640000D1FB4CF68863C2F20003834200F05C8348
:106410004DF6FC30C2F200000CF0C4FB4EF25C33CF
:10642000C2F20003834200F079834DF6FC30C2F2E1
:1064300000000CF0B7FB42F65013C2F20003834297
:1064400000F077834DF6FC30C2F200000CF0AAFB9E
:1064500043F21803C2F20003834200F081824DF63A
:10646000FC30C2F200000CF09DFB4BF61803C1F6A5
:10647000FF73834200F07A834DF6FC30C2F20000D5
:106480000CF090FB4CF26863C2F20003834200F010
:1064900078834DF6FC30C2F200000CF083FB4BF227
:1064A0000C23C1F6FF73834200F085834DF6FC3068
:1064B000C2F200000CF076FB4EF68063C2F20003DD
:1064C000834200F083834DF6FC30C2F200000CF0F2
:1064D00069FB4BF27073C2F20003834200F09083B9
:1064E0004DF6FC30C2F200000CF05CFB42F6486353
:1064F000C2F20003834200F08E834DF6FC30C2F2FC
:1065000000000CF04FFB4CF28C13C2F200038342EC
:1065100000F09B834DF6FC30C2F200000CF042FB11
:106520004DF20823C2F20003834200F099834DF636
:10653000FC30C2F200000CF035FB4BF26053C2F2AB
:106540000003834200F0A6834DF6FC30C2F2000047
:106550000CF028FB4DF60C73C2F20003834200F0EE
:10656000A4834DF6FC30C2F200000CF01BFB4DF68C
:106570007403C2F20003834200F0BC834DF6FC308A
:10658000C2F200000CF00EFB4FF20823C2F200032F
:10659000834200F0A4834DF6FC30C2F200000CF000
:1065A00001FB4CF66853C2F20003834200F0C7833C
:1065B0004DF6FC30C2F200000CF0F4FA42F26473C3
:1065C000C2F20003834200F0AF834DF6FC30C2F20A
:1065D00000000CF0E7FA4CF2A823C2F20003834259
:1065E00000F0C3834DF6FC30C2F200000CF0DAFA82
:1065F0004DF62833C2F20003834200F0AB834DF620
:10660000FC30C2F200000CF0CDFA4BF2E803C1F608
:10661000FF73834200F0B4834DF6FC30C2F20000F9
:106620000CF0C0FA43F2CC23C2F20003834200F024
:1066300003844DF6FC30C2F200000CF0B3FA4BF2CA
:10664000FC63C1F6FF73834200F0BF834DF6FC305C
:10665000C2F200000CF0A6FA4EF2AC33C2F2000314
:10666000834200F0A7834DF6FC30C2F200000CF02C
:1066700099FA4CF6D803C2F20003834200F0D183AA
:106680004DF6FC30C2F200000CF08CFA4EF2606362
:10669000C2F20003834200F0B9834DF6FC30C2F22F
:1066A00000000CF07FFA4CF2B863C2F200038342A0
:1066B00000F0A1834DF6FC30C2F200000CF072FA3B
:1066C00044F2E023C2F20003834200F089834DF6D6
:1066D000FC30C2F200000CF065FA4BF2D063C2F25B
:1066E0000003834200F03D844DF6FC30C2F200000E
:1066F0000CF058FA43F2F073C2F20003834200F048
:1067000025844DF6FC30C2F200000CF04BFA4CF63A
:106710001C03C2F20003834200F00D844DF6FC30EE
:10672000C2F200000CF03EFA4BF23813C1F6FF73D0
:10673000834200F0F5834DF6FC30C2F200000CF00D
:1067400031FA4AF62813C2F20003834200F014849F
:106750004DF6FC30C2F200000CF024FA4DF2CC539E
:10676000C2F2000383427FF4AAAB41F6A420C0F238
:106770000200F9F7E3FF0620FDF74AFAFFF79FBB97
:1067800041F23060C0F20200F9F7CEFF49F2E86052
:106790003946C1F6FF700FF0DDF949F2E860C1F645
:1067A000FF700FF035FAD8F800309F427FF451ABFC
:1067B000FFF777BB63689E423FF471ADF0B2FDF71F
:1067C000BDFB4DF6FC30C2F200000CF01BFA66E592
:1067D00041F22060C0F20200D6E741F28850C0F2D8
:1067E0000200F9F7ABFF4DF6FC30C2F200000CF0EE
:1067F000D9F9854200F001814DF6FC30C2F200006B
:106800000CF0D0F94CF2B863C2F20003834200F0FE
:106810001C814DF6FC30C2F200000CF0C3F944F2CA
:10682000E023C2F20003834200F0C9804DF6FC3041
:10683000C2F200000CF0B6F94BF22073C2F2000372
:10684000834200F0D7804DF6FC30C2F200000CF01D
:10685000A9F94BF20C23C1F6FF7383426FD04DF6BA
:10686000FC30C2F200000CF09DF94BF2D063C2F292
:106870000003834200F077810026354641F2B8508C
:10688000C0F20200F9F750FF616849F2E860314454
:10689000C1F6FF700FF05EF949F2E860C1F6FF70D3
:1068A0000FF0B6F941F2D450C0F20200F9F73CFF04
:1068B00049F2E8606168C1F6FF700FF04BF941F2F0
:1068C000F450C0F20200F9F72FFF2846F9F708FF4D
:1068D0006168013129444DF6FC3043F2B444C9B239
:1068E000C2F20000C2F200040CF06EF9002842D09F
:1068F0006168013129444DF6FC30C9B2C2F2000092
:106900000CF068F9D5E463689E423FF4C8ACF0B27D
:10691000FDF7ACFA4DF6FC30C2F200000CF072F953
:10692000BDE463689E423FF4BAACF0B2FDF7D2FA20
:106930004DF6FC30C2F200000CF064F9AFE40F2613
:1069400035469BE763689E423FF4A9AC70B2FDF701
:10695000A9FB4DF6FC30C2F200000CF053F99EE4A6
:1069600041F24070C0F20200F9F7E8FE0D20FDF799
:1069700085F9FFF7A4BA41F20C60C0F20200F9F702
:10698000D3FE616849F2E86001313144C1F6FF701D
:106990000FF0E0F849F2E860C1F6FF700FF038F947
:1069A00087E463689E423FF47AACF0B2FDF7FAFAEE
:1069B0004DF6FC30C2F200000CF024F96FE4012E19
:1069C00000F08D8041F2A450C0F20200F9F7B6FE4B
:1069D0000420FDF71DF96CE463689E423FF45FAC50
:1069E00070B2FDF713FB4DF6FC30C2F200000CF064
:1069F00009F954E40626354640E741F26050C0F2FA
:106A00000200F9F791FE49F2E860C1F6FF700FF05D
:106A1000FFF8FFF7CBF90120FDF7FAF849E441F25E
:106A20006460C0F20200F9F789FE0120FDF7F0F87A
:106A3000FFF745BA41F27C60C0F20200F9F77EFE32
:106A40000220FDF7E5F8FFF73ABA41F29450C0F2A0
:106A50000200F9F769FE49F2E860C1F6FF700FF035
:106A6000D7F80420FDF7ACF923E463689E423FF4B5
:106A700016AC70B2FDF7FCFA4DF6FC30C2F2000025
:106A80000CF0C0F80BE441F29460C0F20200F9F798
:106A900055FE0720FDF7F2F8FFF711BA41F2B0609A
:106AA000C0F20200F9F74AFE0820FDF7E7F8FFF709
:106AB00006BA41F2CC60C0F20200F9F73FFE0920AD
:106AC000FDF7DCF8FFF7FBB941F2E860C0F2020025
:106AD000F9F734FE0A20FDF7D1F8FFF7F0B940F6D8
:106AE0001870C0F20200F9F71FFE49F24433C1F6F4
:106AF000FF731878F9F7F4FDFDF792F968E763681A
:106B00009E423FF4CCABF0B2FDF704FB4DF6FC30F7
:106B1000C2F200000CF076F8FFF7C1BB41F204703E
:106B2000C0F20200F9F70AFE0B20FDF7A7F8FFF705
:106B3000C6B941F22070C0F20200F9F7FFFD0C2047
:106B4000FDF79CF8FFF7BBB963689E423FF4A7AB23
:106B5000F0B2FDF713FB4DF6FC30C2F200000CF072
:106B600051F8FFF79CBB2226354687E641F2587064
:106B7000C0F20200F9F7E2FD0E20FDF77FF8FFF703
:106B80009EB941F27470C0F20200F9F7D7FD0F20F0
:106B9000FDF774F8FFF793B963689E423FF47FAB4B
:106BA000F0B2FDF71FFB4DF6FC30C2F200000CF016
:106BB00029F8FFF774BB41F29870C0F20200F9F7B0
:106BC000BDFD0320FDF724F8FFF779B941F2AC7061
:106BD000C0F20200F9F7B2FD1020FDF785F8FFF7CB
:106BE0006EB963689E423FF45AABF0B2FDF72EFBDC
:106BF0004DF6FC30C2F200000CF004F8FFF74FBB7A
:106C000041F2D070C0F20200F9F798FD1120FDF7B3
:106C10006BF8FFF754B941F2F070C0F20200F9F7D7
:106C20008DFD1220FDF760F8FFF749B963689E42B9
:106C30003FF435ABF0B2FDF73DFB4DF6FC30C2F250
:106C400000000BF0DFFFFFF72ABB41F60C00C0F29B
:106C50000200F9F773FD1320FDF746F8FFF72FB98F
:106C600041F62800C0F20200F9F768FD1420FDF794
:106C70003BF8FFF724B963689E423FF410ABF0B2D3
:106C8000FDF74CFB4DF6FC30C2F200000BF0BAFFF2
:106C9000FFF705BB41F64800C0F20200F9F74EFDD0
:106CA0001520FDF721F8FFF70AB941F66400C0F29C
:106CB0000200F9F743FD1620FDF716F8FFF7FFB8BD
:106CC00063689E423FF4EBAAF0B2FDF773FB4DF60A
:106CD000FC30C2F200000BF095FFFFF7E0BA41F67E
:106CE000A000C0F20200F9F729FD1820FCF7FCFF14
:106CF000FFF7E5B841F68400C0F20200F9F71EFD87
:106D00001720FCF7F1FFFFF7DAB863689E423FF403
:106D1000C6AAF0B2FDF79CFB4DF6FC30C2F20000B3
:106D20000BF070FFFFF7BBBA41F6DC00C0F20200C7
:106D3000F9F704FD1A20FCF7D7FFFFF7C0B841F6BA
:106D4000BC00C0F20200F9F7F9FC1920FCF7CCFFF7
:106D5000FFF7B5B841F61C10C0F20200F9F7EEFCDF
:106D60001C20FCF7C1FFFFF7AAB841F6FC00C0F2F7
:106D70000200F9F7E3FC1B20FCF7B6FFFFF79FB812
:106D800041F64010C0F20200F9F7D8FC1D20FCF7D4
:106D9000ABFFFFF794B863689E423FF480AAF0B25D
:106DA000FDF7A4FB4DF6FC30C2F200000BF02AFF09
:106DB000FFF775BA41F6A010C0F20200F9F7BEFC69
:106DC0002020FCF791FFFFF77AB841F68010C0F25F
:106DD0000200F9F7B3FC1F20FCF786FFFFF76FB83E
:106DE00041F60820C0F20200F9F7A8FC0420FCF7E5
:106DF0000FFFFFF764B841F6F010C0F20200F9F798
:106E00009DFC0420FCF704FFFFF759B841F6D810A9
:106E1000C0F20200F9F792FC2220FCF765FFFFF7B1
:106E20004EB841F6C010C0F20200F9F787FC2120ED
:106E3000FCF75AFFFFF743B841F66010C0F20200BA
:106E4000F9F77CFC1E20FCF74FFFFFF738B86368AA
:106E50009E423FF424AAF0B2FDF782FB4DF6FC30CF
:106E6000C2F200000BF0CEFEFFF719BA63689E4233
:106E70003FF415AAF0B2FDF7E7FB4DF6FC30C2F285
:106E800000000BF0BFFEFFF70ABA63689E423FF4B2
:106E900006AAF0B2FDF79EFB4DF6FC30C2F20000F0
:106EA0000BF0B0FEFFF7FBB963689E423FF4F7A911
:106EB000F0B2FDF751FC4DF6FC30C2F200000BF0D1
:106EC000A1FEFFF7ECB963689E423FF4E8A9F0B277
:106ED000FDF7D6FC4DF6FC30C2F200000BF092FE3E
:106EE000FFF7DDB963689E423FF4D9A9F0B2FDF720
:106EF00069FD4DF6FC30C2F200000BF083FEFFF797
:106F0000CEB963689E423FF4CAA9F0B2FDF73EFDD8
:106F10004DF6FC30C2F200000BF074FEFFF7BFB973
:106F200041F66C20C0F20200F9F708FC2520FCF7BE
:106F300011FFFEF7C4BF41F65020C0F20200F9F77E
:106F4000FDFB2420FCF706FFFEF7B9BF41F6382011
:106F5000C0F20200F9F7F2FB2320FCF7FBFEFEF77C
:106F6000AEBF41F62420C0F20200F9F7E7FB05208E
:106F7000FCF74EFEFEF7A3BF41F68C20C0F20200E4
:106F8000F9F7DCFB2620FCF7E5FEFEF798BF41F29F
:106F90006C50C0F20200FFF76FB99E423FF47FA928
:106FA000F0B2FDF7C1FE4DF6FC30C2F200000BF06E
:106FB00029FEFFF774B963689E423FF470A9F0B2EE
:106FC000FDF792FE4DF6FC30C2F200000BF01AFE07
:106FD000FFF765B963689E423FF461A9F0B2FDF71F
:106FE00065FE4DF6FC30C2F200000BF00BFEFFF721
:106FF00056B963689E423FF452A9F0B2FDF722FEF3
:107000004DF6FC30C2F200000BF0FCFDFFF747B973
:1070100063689E423FF443A94DF67833321CC2F2B6
:1070200000034DF6FC3018BF0122C2F200001A70B6
:107030000BF0E8FDFFF733B963689E423FF42FA9D8
:10704000F0B2FDF7B7FD4DF6FC30C2F200000BF0D8
:10705000D9FDFFF724B963689E423FF420A9F0B23E
:10706000FDF760FD4DF6FC30C2F200000BF0CAFDEA
:10707000FFF715B963689E423FF411A9F0B2FDF71E
:1070800015FD4DF6FC30C2F200000BF0BBFDFFF722
:1070900006B963689E423FF402A9F0B2FDF7CAFC4C
:1070A0004DF6FC30C2F200000BF0ACFDFFF7F7B874
:1070B00063689E423FF4F3A8F0B2FDF79FFC4DF6E3
:1070C000FC30C2F200000BF09DFDFFF7E8B800BFF6
:1070D0002DE9F04149F24435C1F6FF759AB02E789A
:1070E0001AAB013E06EB8606C3F16B0303EBC60643
:1070F0000DF1FF340DF1270730190EF0DDFF04F814
:10710000010FA742F8D140F23C54C0F202040FCC68
:107110000AAE37460FC70FCC0FC70FCC0FC794E886
:107120000F004FF0FF3487E80F0001A911F8013B71
:1071300083EA04021AA802F00F0200EB8202B142B5
:1071400052F8402C82EA141484EA131303F00F035C
:1071500000EB830353F8403C83EA14146FEA040401
:10716000E4D141F20450C0F20200F9F7DDFA009ECA
:1071700049F2E860314600231022C1F6FF700EF09C
:1071800059FD41F21850C0F20200F9F7CDFA49F268
:10719000E860C1F6FF700023102221460EF04AFD80
:1071A000A6424ED041F61C30C0F20200F9F7C6FAF2
:1071B0004BF63413C1F6FF732A781A70FEF740FAC3
:1071C00049F2F328C1F6FF7841F6E420C0F202004C
:1071D000F9F7AAFA49F2E86098F8001000230A22A9
:1071E000C1F6FF700EF026FD41F6F820C0F2020055
:1071F000F9F79AFA49F2E86000230A222978C1F6E1
:10720000FF700EF017FD49F2E860C1F6FF700EF056
:10721000FFFC41F60430C0F20200F9F785FA49F2AA
:10722000E8606321C1F6FF700EF094FC49F2E8605B
:10723000C1F6FF700EF0ECFC1AB0BDE8F041FEF7AD
:107240008DBB4EF66060C2F200000BF043FD40B310
:1072500001200EF031FF064600202E7049F2FB247B
:107260000EF02AFF49F2F328C1F6FF74013EC1F681
:10727000FF7806EB8606C4F1020303EBC60688F826
:10728000000004F1280730190EF016FF04F8010F72
:10729000BC42F8D141F6D420C0F20200F9F744FA1A
:1072A00092E74EF67060C2F200000BF013FD00286A
:1072B0003FF478AFCCE700BFF8B50446551E4F1E2B
:1072C0002270A57001220025617022712946A571E6
:1072D00084F8C950C4F8B050C4F8B450C4F8B850D9
:1072E000C4F8BC50C4F8C050C4F8C450A82284F8F4
:1072F000C850E77004F108001E4615F005FD022293
:10730000627120460BF0B6F8A579042D0CD805F172
:107310002C03254444F8236030780BF083FC85F877
:10732000C400A3790133A3712046F8BDF8B5044623
:10733000551E4F1E2270A57001220025617022711A
:107340002946A57184F8C950C4F8B050C4F8B450A7
:10735000C4F8B850C4F8BC50C4F8C050C4F8C45005
:10736000A82284F8C850E77004F108001E4615F002
:10737000CBFC0222627120460BF07CF8A579042D2B
:107380000DD805F12C03254444F8236096F900003C
:107390000BF046FC85F8C400A3790133A3712046A5
:1073A000F8BD00BFF8B50446551E4F1E2270A570EB
:1073B00001220025617022712946A57184F8C95007
:1073C000C4F8B050C4F8B450C4F8B850C4F8BC50B5
:1073D000C4F8C050C4F8C450A82284F8C850E7705C
:1073E00004F108001E4615F08FFC0222627120464F
:1073F0000BF040F8A579042D0CD805F12C0330468C
:1074000044F823600BF010FC254485F8C400A379F0
:107410000133A3712046F8BDF8B50446551E4F1E32
:107420002270A57001220025617022712946A57184
:1074300084F8C950C4F8B050C4F8B450C4F8B85077
:10744000C4F8BC50C4F8C050C4F8C450A82284F892
:10745000C850E77004F108001E4615F055FC0222E2
:10746000627120460BF006F8A579042D0CD805F1C1
:107470002C03304644F823600BF0D0FB254485F8FC
:10748000C400A3790133A3712046F8BD2DE9F04172
:1074900093F0010807460E46154610D169B1013D2B
:1074A0000024B86C15F8011F036801341B68984765
:1074B000A642F6D8B8F1000F08D1BDE8F081806C83
:1074C0000368F021DB6C9847002EE8D1B86C0368A4
:1074D000F721DB6CBDE8F041184700BF2DE9F0470C
:1074E0009DF82040013CE4B20F2C03D84EB2002E90
:1074F0000D4601DBBDE8F087E0290FD9F729F9D95E
:107500000835EDB2012303FA05F515F0DD0FF1D0D2
:10751000806C0368BDE8F0471B6818478146806CA3
:107520001F46036846EA0401C9B21B6890469847A3
:10753000D9F84800036808F07F011B6805F0EF05E3
:107540009847C02DD6D0D9F84800036807F07F01CE
:107550001B68BDE8F0471847F0B549F2FC24C1F6B6
:10756000FF7483B094F821300E461546074623B1C8
:10757000984202D0F9F79EFE50B14BF20063C2F27E
:10758000000394F90910186831442A4605F0CAFC32
:1075900041F64C30C0F20200162111F0EDFE94F8D5
:1075A00022303BB344F2F4102B4632469021C2F213
:1075B00000000097FFF792FF2D0640F29C60C0F29A
:1075C000020005F0FE45F9F7AFF845F41045360422
:1075D000781E45F0090506F4FE060002354300F466
:1075E0007060284311F03EF840F21870C0F20200BB
:1075F000F9F79AF849F2E860C1F6FF7003B0BDE808
:10760000F0400EF005BB00BFF0B549F2FC24C1F616
:10761000FF7483B094F821300E461546074623B117
:10762000984202D0F9F746FE50B14BF20063C2F225
:10763000000394F90910186831442A4605F072FCD9
:1076400041F66430C0F20200112111F095FE94F869
:1076500022305BB344F2F4102B4632469021C2F242
:1076600000000097FFF73AFF2D0640F29C60C0F241
:10767000020005F0FE45F9F757F845F410453604C9
:10768000791E45F0090506F4FE060902354301F4AA
:1076900070614EF28070C2F2000029430DF056F97D
:1076A00040F2AC60C0F20200F9F73EF849F2E8603F
:1076B000C1F6FF7003B0BDE8F0400EF0A9BA00BFFC
:1076C000F0B549F2FC24C1F6FF7483B094F8213080
:1076D0000E461546074623B1984202D0F9F7EAFD57
:1076E00050B14BF20063C2F2000394F9091018681C
:1076F0003144002205F016FC41F67830C0F2020059
:10770000172111F039FE94F822303BB344F2F41003
:107710002B4632468021C2F200000097FFF7DEFEC2
:107720002D0640F29C60C0F2020005F0FE45F8F71D
:10773000FBFF45F400453604781E45F0080506F4C5
:10774000FE060002354300F47060284310F08AFF03
:1077500040F21870C0F20200F8F7E6FF49F2E86064
:10776000C1F6FF7003B0BDE8F0400EF051BA00BFA3
:10777000F0B549F2FC24C1F6FF7483B094F82130CF
:107780000E461546074623B1984202D0F9F792FDFE
:1077900050B14BF20063C2F2000394F9091018686B
:1077A0003144002205F0BEFB41F69030C0F20200E9
:1077B000122111F0E1FD94F822305BB344F2F41091
:1077C0002B4632468021C2F200000097FFF786FE6A
:1077D0002D0640F29C60C0F2020005F0FE45F8F76D
:1077E000A3FF45F400453604791E45F0080506F46C
:1077F000FE060902354301F470614EF28070C2F258
:10780000000029430DF0A2F840F2AC60C0F2020083
:10781000F8F78AFF49F2E860C1F6FF7003B0BDE8EF
:10782000F0400EF0F5B900BFF0B549F2FC25C1F605
:10783000FF7583B095F821300E461446074623B1F4
:10784000984202D0F9F736FD48B14BF20063C2F21C
:10785000000322461868036831465B68984741F682
:10786000A430C0F20200122111F086FD95F82230FA
:107870003BB344F2F41023463246B021C2F200007A
:107880000097FFF72BFE240640F29C60C0F2020036
:1078900004F0FE44F8F748FF44F430443604781E00
:1078A00044F00B0406F4FE060002344300F470605A
:1078B000204310F0D7FE40F21870C0F20200F8F733
:1078C00033FF49F2E860C1F6FF7003B0BDE8F04055
:1078D0000EF09EB9F0B549F2FC25C1F6FF7583B0F4
:1078E00095F821300E461446074623B1984202D03F
:1078F000F9F7E0FC48B14BF20063C2F20003224604
:107900001868036831465B68984741F6B830C0F2A2
:1079100002000D2111F030FD95F822305BB344F2E6
:10792000F41023463246B021C2F200000097FFF760
:10793000D5FD240640F29C60C0F2020004F0FE4433
:10794000F8F7F2FE44F430443604791E44F00B0498
:1079500006F4FE060902344301F470614EF28070B1
:10796000C2F2000021430CF0F1FF40F2AC60C0F223
:107970000200F8F7D9FE49F2E860C1F6FF7003B0E3
:10798000BDE8F0400EF044B930B5054641F6C830C8
:1079900083B00C46C0F20200122111F0EDFC49F256
:1079A000FC23C1F6FF7393F822301BB344F2F410AA
:1079B00022460023D021C2F200000095FFF78EFD81
:1079C00040F29C60C0F202002404F8F7ADFE04F41B
:1079D000FE04681E44F45044000244F00D0400F418
:1079E0007060204310F03EFE40F21870C0F20200BA
:1079F000F8F79AFE49F2E860C1F6FF7003B0BDE8FF
:107A000030400EF005B900BF30B5054641F6DC3018
:107A100083B00C46C0F202000D2111F0ADFC49F21A
:107A2000FC23C1F6FF7393F822303BB344F2F41009
:107A300022460023D021C2F200000095FFF74EFD40
:107A400040F29C60C0F202002404F8F76DFE04F4DA
:107A5000FE04691E44F45044090244F00D0401F48C
:107A600070614EF28070C2F2000021430CF06EFF94
:107A700040F2AC60C0F20200F8F756FE49F2E8604E
:107A8000C1F6FF7003B0BDE830400EF0C1B800BFD2
:107A900030B5054641F6EC3083B00C46C0F202002A
:107AA000122111F069FC49F2FC23C1F6FF7393F82F
:107AB00022307BB304F5005244F2F410C2F3C61333
:107AC000E02102F07F020095C2F20000FFF706FD00
:107AD00004F30D0440F29C6004F50054C0F202006F
:107AE000013DF8F721FE2D02200400F4FE0005F40C
:107AF0007065054345F46040640440F00E0004F0F6
:107B0000FE44204310F0AEFD40F21870C0F20200B7
:107B1000F8F70AFE49F2E860C1F6FF7003B0BDE86D
:107B200030400EF075B800BF30B5054641F6004054
:107B300083B00C46C0F202000D2111F01DFC49F289
:107B4000FC23C1F6FF7393F822309BB304F5005277
:107B500044F2F410C2F3C613E02102F07F02009554
:107B6000C2F20000FFF7BAFC04F30D0440F29C607F
:107B700004F50054C0F20200013DF8F7D5FD2D02D6
:107B8000210401F4FE0105F470650D4345F46041E4
:107B9000640441F00E0104F0FE444EF28070C2F223
:107BA000000021430CF0D2FE40F2AC60C0F20200B3
:107BB000F8F7BAFD49F2E860C1F6FF7003B0BDE81E
:107BC00030400EF025B800BF30B5054641F61040F4
:107BD00083B00C46C0F20200122111F0CDFB49F235
:107BE000FC23C1F6FF7393F822301BB344F2F41068
:107BF00022460023C021C2F200000095FFF76EFC70
:107C000040F29C60C0F202002404F8F78DFD04F4F9
:107C1000FE04681E44F44044000244F00C0400F4E6
:107C20007060204310F01EFD40F21870C0F2020098
:107C3000F8F77AFD49F2E860C1F6FF7003B0BDE8DD
:107C400030400DF0E5BF00BF30B5054641F6244099
:107C500083B00C46C0F202000D2111F08DFB49F2F9
:107C6000FC23C1F6FF7393F822303BB344F2F410C7
:107C700022460023C021C2F200000095FFF72EFC2F
:107C800040F29C60C0F202002404F8F74DFD04F4B9
:107C9000FE04691E44F44044090244F00C0401F45B
:107CA00070614EF28070C2F2000021430CF04EFE73
:107CB00040F2AC60C0F20200F8F736FD49F2E8602D
:107CC000C1F6FF7003B0BDE830400DF0A1BF00BFAA
:107CD00070B5064641F6344082B00C46C0F2020050
:107CE0001721154611F048FB49F2FC23C1F6FF733A
:107CF00093F8223043B949F2E860C1F6FF7002B050
:107D0000BDE870400DF084BF44F2F410C2F20000F0
:107D100000962B462246A021FFF7E0FB41F64C409F
:107D2000C0F20200F8F700FD36B140F21870C0F260
:107D30000200F8F7F9FCDEE7681E0002240404F4F0
:107D4000FE0400F47060204340F4504040F00D0009
:107D500010F088FCE9E700BF70B5064641F65840D0
:107D600082B00C46C0F202001221154611F004FB4D
:107D700049F2FC23C1F6FF7393F8223053B344F267
:107D8000F41022462B46A021C2F200000096FFF715
:107D9000A5FB41F64C40C0F20200F8F7C5FC691E95
:107DA0000902240401F4706104F4FE040C4344F459
:107DB0005044310144F00D04C9B24EF28070C2F259
:107DC000000021430CF0C2FD40F2AC60C0F20200A2
:107DD000F8F7AAFC49F2E860C1F6FF7002B0BDE80E
:107DE00070400DF015BF00BFF8B50446806C036805
:107DF0001B69984708B90020F8BDA06C03685B694F
:107E00009847C3B203F0FB01F929F4D0A26D7AB907
:107E100094F84D2084F84F30150666D440B20028FF
:107E2000C0F24781002084F84D00A0656065F8BD70
:107E3000010633D494F84F10F02904EB020124D04A
:107E400081F84F30616D4B1E9A4224D394F84F2035
:107E5000F02AE7D0130600F1C280002094F85030D9
:107E600084F86600032984F8650084F8673000F020
:107E7000CD80012384F86800A065606584F8E9304E
:107E8000002384F84D300120F8BD81F86930636D1E
:107E9000013B9A42C6D20132A265ACE7A3F1F701D9
:107EA0000829C7D8012505FA01F010F4DD7F40F05C
:107EB000CD800029BED194F86930F02BB2D1561C88
:107EC0002244F720370A82F8690084F8676084F852
:107ED000687084F8651084F84D10284684F8663080
:107EE00084F8E950A1656165F8BD02F10C05EEB2B8
:107EF000012E93D902F0FB0EBEF1F90F8ED0EF2ABE
:107F000036D802F0F007802F33D140B2002886DB4C
:107F1000012184F84F2084F85030A165EDB2012D85
:107F200080D9BEF1F90F3FF47DAFEF2A00F29B80BC
:107F300002F0F003F12B4ED000F29780B02B43D02B
:107F40003BD9D02B47D043D9E02B3DD0F02B7FF449
:107F500069AF0021802084F84D1084F86930606595
:107F60007F21A36D8B4211D20133A3650020F8BDA0
:107F7000174607F0DF06902EC7D007F0BF06A02EE9
:107F8000C3D007F0EF07C02FBFD047E71046F8F780
:107F900099FB02F00F020023013294F8501084F88C
:107FA000660084F86520012084F8671084F8683042
:107FB000A365636584F8E900F8BD902B04D0A02B7D
:107FC00002D0802B7FF42EAF032363650221C8E724
:107FD000C02B7FF427AF022363650121C1E7F42A98
:107FE0003FF43BAF1046F8F76DFB802884F866003D
:107FF00064D102F00F03013394F8505084F86750B5
:10800000032984F8653018BF002501D194F8515038
:1080100084F8685000230121B028A365636584F8C3
:10802000E91007D00AD8902804D0A02802D08028D0
:108030007FF426AF84F84D200120F8BDD028F9D078
:10804000E028F7D0C0287FF41BAFF3E7002284F8C4
:10805000672084F8682084F8652084F8663084F806
:10806000E9502846F8BD134664E7F82B06D018D827
:10807000F32BB0D0A8D3F62B7FF4D4AE1046F8F78C
:1080800021FB0022012384F8652084F8672084F80E
:10809000682084F86600A265626584F8E9301846B5
:1080A000F8BDFA2BFFF4BEAEFC2BE7D9FE2BE5D2D0
:1080B000B8E61A468E4603F10C052FE7902898D0B3
:1080C000B02896D0A02894D0D02892D0E02890D084
:1080D000C0288ED000238FE790F86630F12B7CD03B
:1080E0000ED9FA2B2BD01FD8F32B38D0C0F08180BB
:1080F000F62B7AD0F82B40F08B80036BF3B1184746
:10810000B02B6ED031D9D02B21D03ED9E02B42D02C
:10811000F02B7ED1C3698BB1B0F86710802900F1D4
:10812000690028BF80211847FC2B0CD051D3FE2BAF
:108130004BD0FF2B6BD1436C002BE0D17047436BCE
:10814000002BDCD1FAE7C36B002BD8D1F6E74369EB
:10815000002BF3D090F8671090F865001847836AF9
:10816000002BEBD090F867001847902B29D0A02B5C
:1081700023D0802BE2D10368002BDFD090F8682059
:1081800090F8671090F865001847C02B42D103693A
:10819000002BDFD1D2E78269002ACFD090F8681097
:1081A00090F8673090F86500C90101F47E5103F042
:1081B0007F031943A1F5005110478368002BDDD1DF
:1081C000BCE74368002BD9D1B8E7036C002B96D1EC
:1081D000B4E7836B002B92D1B0E7036A002BC1D1C7
:1081E000ACE7C368002BC9D1A8E7C36A002B86D1CE
:1081F000A4E7426A002AA1D090F8683090F867009E
:10820000DB0103F47E5300F07F00184310477047F2
:1082100070477047704700BF90F86430DA0725D583
:1082200013F0FE0F22D070B590F8665085F08002F2
:10823000602A82B004461AD9F62D66D05FD8F12D97
:1082400076D04FD9F22D2DD0F32D1AD1806C94F821
:108250006760036829461B689847A06C0368DB6C5D
:1082600006F07F0102B0BDE870401847704790F8F3
:1082700065608E4207D031B15B08012B08D0032B1B
:1082800027D002B070BD5B08012B01D0022BF8D1C2
:1082900094F8683094F86720009629462046FFF746
:1082A0001DF9EEE7806C94F86730026894F8686016
:1082B0001268294643EAC6159047A06C036805F08A
:1082C0007F019B6C9847A06C0368C5F3C6119B6C3B
:1082D000C8E794F8683094F8672000962946FFF7BD
:1082E000FDF8CEE7F02DCCD1B0F86710802900F171
:1082F000690228BF80210123FFF7C8F8C1E7FC2DE0
:1083000026D8FA2D01D2F82DBBD105F10803DBB236
:10831000072BB6D8012202FA03F313F0DD0FB0D019
:10832000A06C03681B68294602B0BDE8704018477E
:10833000806C94F8672094F868300668120129462A
:1083400003F00F0302F0700532681D439047E7E722
:10835000FE2D96D3D9E700BFF0B542F6787087B00E
:10836000C2F2000007F09EFC00287FD140F2346486
:10837000C2F2010444F2F415C2F2000595F84C6013
:10838000102E1CD9002010F00FFC0BF0E5FC4EF273
:1083900080700021C2F200000CF0D0FB43F2BC431D
:1083A00022680392C2F20003039A1868121A40F27C
:1083B0003461642AC2F201011ED807B0F0BD28461C
:1083C000FFF712FD0028DDD095F86630902B00F005
:1083D000358183F08003602B40F2338144F2F41046
:1083E000C2F20000FFF778FE44F2F4103146C2F208
:1083F0000000FFF711FFC5E70A680492049A1A60AB
:10840000FDF7F6FC4BF63413C1F6FF731B78002B17
:1084100040F024814DF69C73C2F200031A78002AC2
:10842000CBD04FF2042122680592C2F20001059AD6
:10843000086841F28831121A8A42BED949F2F32201
:10844000C1F6FF720024204615781C700DF034FE32
:10845000854203D0294620460DF048FE41F2142003
:10846000C0F20200F8F76AF907B0F0BD42F6A85072
:10847000C2F2000007F016FC00283FF477AF43F685
:10848000F466C2F200060EF0DFFB3368C01A40F259
:108490003464B0F5356FC2F201047FF66BAF4DF670
:1084A000A0750EF0D1FBC2F20005236801932A6883
:1084B000019B30609B1A41F28832934200F2DB80CC
:1084C00042F67870C2F2000007F0FCFB0646002876
:1084D00000F0D88042F6A850C2F2000007F0F2FB8C
:1084E0000746002800F0D5800EF0AEFB4BF200638B
:1084F000C2F200030546186803683A461B68314615
:1085000098470EF0A1FB40F65A33401B984206D91B
:108510004DF22433C2F200031A6801321A604CF69D
:108520008463C2F200031A88824238BF188072B690
:108530004CF2F873C2F200031A7F02F0FF010AB195
:1085400000221A7762B679B372B647F6FF754FF418
:108550000040B3F91E10B3F92020DD83188462B601
:10856000002982EAE273A3EBE273B8BF49428B426F
:10857000B8BF0B4607EE903A4FF47E43C4F2FF6358
:10858000F8EEE77A06EE903A87EEA67AF7EE007AF2
:10859000B4EEE77AF1EE10FA06DD42F68C33C2F261
:1085A00000031A6801321A6072B64CF20873C2F204
:1085B00000031A7F02F0FF010AB100221A7762B6A7
:1085C00079B372B647F6FF754FF40040B3F91E1049
:1085D000B3F92020DD83188462B6002982EAE273B1
:1085E000A3EBE273B8BF49428B42B8BF0B4607EE1C
:1085F000903A4FF47E43C4F2FF63F8EEE77A06EE5A
:10860000903A87EEA67AF7EE007AB4EEE77AF1EECA
:1086100010FA06DD42F68C33C2F200031A6801320A
:108620001A6042F67870C2F2000007F05DFB42F675
:10863000A850C2F2000007F057FB9BE695F868309F
:1086400043B195F865309E423FF4C8AE002E3FF42A
:10865000C5AEC9E6802385F86630F2E74BF20063C9
:10866000C2F20003186804F059FC00287FF4D2AE6F
:10867000FCF7E6FFCEE6FDF7A7F823680293029B1E
:108680002B601DE741F66C40C0F20200F8F756F887
:1086900020E741F69440C0F20200F8F74FF823E7D4
:1086A0002DE9F04F4CF628148FB0C2F2000444F2CA
:1086B0009046C2F200060DF0ADFC022320461022C7
:1086C0002721002509F0FAFA4FF060496FF0604861
:1086D0003046022203214EF66067FBF7F9F9C2F239
:1086E0000007C6F81490C6F81880357706F1200008
:1086F0001D221C21FBF7ECF9C6F83490C6F838802F
:1087000086F83C503846142204210AF08FFA07F10B
:10871000100014221E210AF089FA40F23463C2F2DA
:10872000010344F218021B680A93C2F200020A997C
:10873000116040F2E85343F640002A46C0F20203BB
:108740000121C2F20000FEF767FE012240F2F4535D
:1087500043F60C101146C0F20203C2F20000FEF70D
:108760005BFE012241F61C6343F6D8101146C0F2AD
:108770000203C2F20000FEF74FFE012240F2006346
:1087800043F6A4201146C0F20203C2F20000FEF735
:1087900043FE012240F20C6343F670301146C0F2F2
:1087A0000203C2F20000FEF737FE012240F214631A
:1087B00043F63C40C0F202031146C2F20000FEF74D
:1087C0002BFE4FF26800C2F200000AF0E7F84BF609
:1087D000F46021460122C2F2000009F0CDFF41F60B
:1087E000BC734BF65C502A46C0F202030121C2F270
:1087F000000049F24437FEF70FFEC1F6FF77012271
:108800004CF678103B461146C2F20000FEF754FDCC
:108810004EF26810C2F200000AF0C0F84AF640605A
:1088200021460122C2F2000009F0A6FF41F61463BE
:108830004AF290702A46C0F202030121C2F20000FF
:10884000FEF7EAFD012242F224034AF65C001146DB
:10885000C0F20203C2F20000FEF7DEFD012242F286
:108860002C034BF294401146C0F20203C2F2000006
:10887000FEF7D2FD012241F66C734AF678101146DC
:10888000C0F20203C2F20000FEF7C6FD012242F26E
:1088900038034AF644201146C0F20203C2F2000037
:1088A000FEF7BAFD012242F248034AF610301146A3
:1088B000C0F20203C2F20000FEF7AEFD012242F256
:1088C00054034AF6DC301146C0F20203C2F2000043
:1088D000FEF7A2FD012242F25C034AF6A8401146CF
:1088E000C0F20203C2F20000FEF796FD012242F23E
:1088F00064034AF67450C0F202031146C2F200004B
:10890000FEF78AFD4BF22070C2F200000AF046F832
:1089100042F6A01021460122C2F2000009F02CFF0D
:1089200041F6B4734BF25C202A46C0F202030121E7
:10893000C1F6FF7049F2FC26C1F6FF76FEF76CFD2A
:1089400001224BF22830331D1146C1F6FF70FEF7AD
:10895000B3FC4BF6D020C1F6FF700AF01FF84CF2C2
:108960004C1021460122C2F2000009F005FF40F23E
:108970001C634BF654002A46C0F202030121C2F2E6
:108980000000FEF749FD01224BF62010731D114631
:10899000C2F20000FEF790FC42F2F850C2F2000072
:1089A00009F0FCFF42F6485021460122C2F20000C5
:1089B00009F0E2FE41F6C8734BF6C4502A46C0F2F5
:1089C00002030121C1F6FF70FEF726FD01224BF6DE
:1089D0009060B31D1146C1F6FF70FEF76DFC4BF2BF
:1089E000B050C2F2000009F0D9FF44F284302146B1
:1089F0000122C2F2000009F0BFFE41F6506343F6C7
:108A000048502A46C0F202030121C2F20000FEF7DC
:108A100003FD012243F61460F31D1146C2F200006B
:108A2000FEF74AFC4CF68860C2F2000009F0B6FF7F
:108A30004BF2C07021460122C2F2000009F09CFEF8
:108A400042F21C034DF6C4002A46C0F20203012183
:108A5000C2F20000FEF7E0FC01224DF6901006F194
:108A600008031146C2F20000FEF760FC4EF25C30D3
:108A7000C2F2000009F092FF4CF698002146012254
:108A8000C2F2000009F078FE41F608634BF21C00C8
:108A90002A46C0F202030121C1F6FF70FEF7BCFCBA
:108AA00001224BF6603006F109031146C1F6FF7052
:108AB000FEF73CFC42F65010C2F2000009F06EFFD7
:108AC0004EF2700021460122C2F2000009F054FE6D
:108AD00042F2040342F2B4702A46C0F202030121BA
:108AE000C2F20000FEF798FC012240F2416342F618
:108AF0008000C0F200031146C2F20000FEF752FCF3
:108B000043F21800C2F2000009F048FF4BF258404F
:108B100021460122C1F6FF7009F02EFE41F668637E
:108B20004CF2D0402A46C0F202030121C2F20000FA
:108B3000FEF772FC01224CF29C5006F10B03114629
:108B4000C2F20000FEF7B8FB4BF61800C1F6FF704A
:108B500009F024FF43F6085021460122C2F200002A
:108B600009F00AFE41F6AC634DF6A8402A46C0F271
:108B700002030121C2F20000FEF74EFC01224EF278
:108B8000B06006F10C031146C2F20000FEF794FB40
:108B90004CF26860C2F2000009F000FF4EF2B8101B
:108BA00021460122C2F2000009F0E6FD42F238132C
:108BB00042F2FC102A46C0F202030121C2F2000078
:108BC000FEF72AFC012242F2481342F2C820114665
:108BD000C0F20203C2F20000FEF71EFC012241F6C1
:108BE000C86342F294301146C0F20203C2F20000A0
:108BF000FEF712FC012241F6D46342F260401146B6
:108C0000C0F20203C2F20000FEF706FC012242F2AB
:108C10007C0342F22C501146C0F20203C2F2000063
:108C2000FEF7FAFB012240F27C534BF2980011460A
:108C3000C0F20203C2F20000FEF7EEFB012240F296
:108C4000885342F248601146C0F20203C2F20000AB
:108C5000FEF7E2FB012241F60C734BF2FC201146B9
:108C6000C0F20203C2F20000FEF7D6FB012241F679
:108C70001C734BF2C8301146C0F20203C2F200006E
:108C8000FEF7CAFB012241F6747343F21C30114611
:108C9000C0F20203C2F20000FEF7BEFB012242F264
:108CA000181343F2E8301146C0F20203C2F200008A
:108CB000FEF7B2FB012241F684734CF644201146C4
:108CC000C0F20203C2F20000FEF7A6FB012242F24C
:108CD00028134CF650301146C0F20203C2F20000D5
:108CE000FEF79AFB012241F6287343F2C040114679
:108CF000C0F20203C2F20000FEF78EFB012241F631
:108D0000907343F28C501146C0F20203C2F200008D
:108D1000FEF782FB012242F2E80343F2586011465B
:108D2000C0F20203C2F20000FEF776FB012242F21B
:108D3000081343F224701146C0F20203C2F200008D
:108D4000FEF76AFB012241F6A0734CF6B8501146BB
:108D5000C0F20203C2F20000FEF75EFB012241F600
:108D6000A8734BF6B820C0F202031146C2F200000D
:108D7000FEF752FB4BF20C20C1F6FF7009F00EFE1D
:108D80004FF2B80021460122C2F2000009F0F4FCC3
:108D900041F6F4734AF6CC702A46C0F20203012170
:108DA000C2F20000FEF738FB01224BF2641006F11C
:108DB0000D031146C2F20000FEF77EFA4EF6806007
:108DC000C2F2000009F0EAFD4BF614002146012230
:108DD000C2F2000009F0D0FC41F67C634EF2302074
:108DE0002A46C0F202030121C2F20000FEF714FB82
:108DF000012244F2C43006F10E031146C2F2000013
:108E0000FEF75AFA4BF27070C2F2000009F0C6FD8C
:108E10004DF2F47021460122C2F2000009F0ACFCD0
:108E200040F2BC534DF674502A46C0F202030121B1
:108E3000C2F20000FEF7F0FA01224DF6406006F1A2
:108E40000F031146C2F20000FEF736FA42F6486000
:108E5000C2F2000009F0A2FD4CF6103021460122BA
:108E6000C2F2000009F088FC40F298534BF2302027
:108E70002A46C0F202030121C2F20000FEF7CCFA3A
:108E8000012240F26D434BF23060C0F20003114604
:108E9000C1F6FF70FEF786FA4CF28C10C2F20000A9
:108EA00009F07CFD4CF6381021460122C2F2000088
:108EB00009F062FC42F28C034CF238302A46C0F2D0
:108EC00002030121C2F20000FEF7A6FA012240F2DD
:108ED0008D434CF20440C0F200031146C2F2000080
:108EE000FEF760FA4DF20820C2F2000009F056FDCC
:108EF00044F21C0021460122C2F2000009F03CFCB1
:108F000040F2B05343F64C702A46C0F202030121EE
:108F1000C2F20000FEF780FA012240F2AD434DF2AA
:108F20005820C0F200031146C2F20000FEF73AFAE0
:108F30004BF26050C2F2000009F030FD4BF62030D9
:108F400021460122C1F6FF7009F016FC42F2C80367
:108F50004BF204602A46C0F202030121C2F2000073
:108F6000FEF75AFA012240F26D5342F67C40C0F2FD
:108F700000031146C2F20000FEF714FA4DF60C7021
:108F8000C2F2000009F00AFD43F6F8602146012212
:108F9000C2F2000009F0F0FB42F2D8034EF2C840E2
:108FA0002A46C0F202030121C2F20000FEF734FAA1
:108FB000012240F2B9534EF29450C0F20003114620
:108FC000C2F20000FEF7EEF94DF67400C2F20000A6
:108FD00009F0E4FC4AF68C7021460122C2F200003E
:108FE00009F0CAFB40F2A4534DF270002A46C0F2C9
:108FF00002030121C2F20000FEF70EFA012240F244
:10900000FD534DF23C10C0F200031146C2F20000C5
:10901000FEF7C8F94FF20820C2F2000009F0BEFCCA
:109020004BF2CC1021460122C1F6FF7009F0A4FBDF
:1090300040F2C85343F268002A46C0F202030121FD
:10904000C2F20000FEF7E8F901224DF2683006F1A5
:1090500016031146C2F20000FEF72EF94CF66850D6
:10906000C2F2000009F09AFC4EF21C3021460122A7
:10907000C2F2000009F080FB41F6D4734BF24C7051
:109080002A46C0F202030121C1F6FF70FEF7C4F9BF
:1090900001224BF6680006F117031146C1F6FF7076
:1090A000FEF70AF942F26470C2F2000009F076FCA1
:1090B0004DF6340021460122C2F2000009F05CFBAB
:1090C00040F2D8534BF298402A46C0F202030121E5
:1090D000C1F6FF70FEF7A0F901224BF2645006F1D1
:1090E00018031146C1F6FF70FEF7E6F84CF2A8200F
:1090F000C2F2000009F052FC4BF65040214601221A
:10910000C2F2000009F038FB42F20C034DF2344089
:109110002A46C0F202030121C2F20000FEF77CF9E8
:1091200001224DF2005006F119031146C2F200006F
:10913000FEF7C2F84DF62830C2F2000009F02EFC0E
:109140004DF2283021460122C2F2000009F014FB42
:1091500041F644734BF638102A46C0F2020301214F
:10916000C1F6FF70FEF758F901224BF6042006F114
:109170001A031146C1F6FF70FEF79EF84BF2E800A5
:10918000C1F6FF7009F00AFC4EF2E8002146012208
:10919000C2F2000009F0F0FA41F6246342F6F4103E
:1091A0002A46C0F202030121C2F20000FEF734F9A0
:1091B000012242F6C02006F11B031146C2F2000054
:1091C000FEF77AF843F2CC20C2F2000009F0E6FB89
:1091D0004CF6285021460122C2F2000009F0CCFAD8
:1091E00041F640634DF25C602A46C0F20203012161
:1091F000C2F20000FEF710F9012244F25C0006F111
:109200001C031146C2F20000FEF756F84BF2FC6058
:10921000C1F6FF7009F0C2FB4FF2C41021460122D3
:10922000C2F2000009F0A8FA42F2B8034AF68060E0
:109230002A46C0F202030121C2F20000FEF7ECF858
:1092400001224BF6EC1006F11D031146C2F200009C
:10925000FEF732F84EF2AC30C2F2000009F09EFB8D
:109260004DF21C6021460122C2F2000009F084FA8E
:1092700042F274034FF2F8002A46C0F202030121C1
:10928000C2F20000FEF7C8F801224DF65C2006F19C
:109290001E031146C2F20000FEF748F84CF6D80053
:1092A000C2F2000009F07AFB44F23030214601227C
:1092B000C2F2000009F060FA42F2AC0342F6986094
:1092C0002A46C0F202030121C2F20000FEF7A4F810
:1092D00001224DF2287006F11F031146C2F2000070
:1092E000FEF724F84EF26060C2F2000009F056FB6F
:1092F0004AF64C7021460122C2F2000009F03CFA05
:1093000041F634634EF6D0602A46C0F202030121D2
:10931000C2F20000FEF780F801224EF69C703B4638
:109320001146C2F20000FDF7C7FF4CF2B860C2F26E
:10933000000009F033FB4BF6347021460122C2F2E3
:10934000000009F019FA41F6BC634BF684302A4656
:10935000C0F202030121C2F20000FEF75DF8012213
:1093600041F68C634BF690401146C0F20203C2F204
:109370000000FEF751F8012241F69C6344F22810E8
:109380001146C0F20203C2F20000FEF745F80122C6
:1093900042F29C034BF62860C0F202031146C2F26F
:1093A0000000FEF739F84BF2D060C2F2000009F07D
:1093B000F5FA4CF2F82021460122C2F2000009F031
:1093C000DBF941F638734BF6F8402A46C0F2020347
:1093D0000121C1F6FF70FEF71FF801224BF62C4069
:1093E00006F120031146C1F6FF70FDF765FF43F259
:1093F000F070C2F2000009F0D1FA4DF65C7021461F
:109400000122C2F2000009F0B7F941F6FC634CF208
:10941000DC10C0F2020300220121C2F20000FDF7BD
:10942000FBFF012240F275634CF61C40C0F20003C2
:109430001146C2F20000FDF7B5FF4CF61C00C2F267
:10944000000009F0ABFA4DF67C3021460122C2F251
:10945000000009F091F941F6E47343F23410C0F2D0
:10946000020300220121C2F20000FDF7D5FF012214
:1094700040F2D14343F20020C0F200031146C2F291
:109480000000FDF78FFF4BF23810C1F6FF7009F0B6
:1094900085FA4BF28C1021460122C1F6FF7009F0CB
:1094A0006BF942F2F8034BF67470C0F2020300222B
:1094B0000121C2F20000FDF7AFFF01224CF2800053
:1094C00006F123031146C2F20000FDF7F5FE4AF64D
:1094D0002810C2F2000009F061FA4DF6BC302146B6
:1094E0000122C2F2000009F047F9002241F654734C
:1094F0004CF22C701146C0F20203C2F20000FDF7DC
:109500008BFF41F6647342F6B030C0F202030122D1
:109510000021C2F20000FDF77FFF4DF2CC50C2F2F5
:10952000000009F03BFA4CF6E84021460122C2F265
:10953000000009F021F941F658634DF6A470C0F21D
:10954000020300220121C2F20000FDF765FF0122A3
:1095500049F2F3234EF2FC30C1F6FF731146C2F21A
:109560000000FDF7A9FE42F21470C2F2000009F0FB
:1095700015FA4CF2400021460122C2F2000009F027
:10958000FBF841F670634CF6D860C0F2020300228B
:109590000121C2F20000FDF73FFF012240F2195302
:1095A0004CF6A470C0F200031146C2F20000FDF7B1
:1095B000F9FE44F2E020C2F2000009F0EFF94EF2A9
:1095C000281021460122C2F2000044F2F419C2F22E
:1095D000000909F0D1F84DF6FC300121C2F200007B
:1095E00009F0AAFA99F86430012243F0010362F30A
:1095F000470349F2A025002489F8643049F218563F
:109600002B464FF6FF7E214689F8654089F8664073
:1096100089F8674089F8684089F8E940C1F6FF7326
:10962000C1F6FF7609F1690080221D46C9F85CE0A9
:10963000C9F860E0C9F8486089F84C4089F84D40A5
:1096400089F84E40C9F85440C9F858404EF2807627
:1096500013F05AFB40F2695142F67873C2F20006E9
:109660002A46C2F200034846C0F2000140F6580AFA
:109670000195C9F800401D46C9F80440C9F80840E2
:10968000C9F80C40C9F81040C9F81440C9F818408E
:10969000C9F81C40C9F82040C9F82440C9F828403E
:1096A000C9F82C40C9F83040C9F83440C9F83840EE
:1096B000C9F83C40C9F84040C9F84440C0F20F0A1C
:1096C00012F0AEFF06F5A36C06F5AB6E06F5B361BE
:1096D000502306F59B694022C6F818C0C6F81CE066
:1096E000B38574603046B460C6F800A0C6F8149024
:1096F000716272850BF0E6F84CF2F872029240F259
:109700002852C0F202023260214622462846F9F76A
:10971000F1FA029A85F89C4042F6A85BC2F2000B6F
:10972000C2F2000240F2F4684CF20873C2F2000385
:10973000C0F20F0802922146224658460393C5F80C
:10974000984085F89D400695C5F80080F9F7D2FA53
:1097500002998BF89C4044F2DC400A468946054653
:10976000183208460121CBF80080CBF898408BF8DE
:109770009D40F9F7BFFA0399CDF80890C2F20005B1
:109780004BF65C7307950A464BF65C7540F29857AA
:109790008A461832C0F20F0747F6FF764FF40048AA
:1097A000059508461D460121C9F80070A9F81E60FC
:1097B000A9F82080C1F6FF75F9F79CFA4EF2F81966
:1097C0000798CAF80070C2F20009AAF81E60CDF826
:1097D0000CA0AAF8208005F061FD4EF2B00A2846E0
:1097E000C2F2000A059542F6885705F057FD40F28F
:1097F000DC6609F128024846042142F69035F9F763
:1098000079FA4FF48033C2F20007C0F20F060AF172
:10981000280250460421C2F20005C9F80060C9F8C8
:109820001830C9F81C30C9F82030C9F82430089322
:109830000495F9F75FFA089BCAF8006007F11C026B
:10984000384601213D46CAF81830CAF81C30CAF81B
:109850002030CAF82430F9F74DFA049F089BAB6119
:1098600007F11C02089538462F4640F2D065C0F239
:109870000F05012109933D6043F63878F9F73AFA6C
:109880000499099B029A0D60C2F2000840F26966D1
:10989000C0F20006069D8B61404643F6E067C2F2C7
:1098A0000007C8F80420C8F8005088F8084088F875
:1098B0000940C8F80C4088F810400BF06BFD019A85
:1098C000314640464BF2F43812F0AAFEC1F6FF785A
:1098D000039979603846C7F800B03C727C72FC602E
:1098E0003C740BF057FD019A3146384612F098FE51
:1098F0004BF2084740460695C8F80050079DC8F847
:109900000450C1F6FF7788F8084088F80940C8F885
:109910000C4088F810400BF03DFD3146019A40465E
:1099200012F07EFE059AC7F800B038467A603C72A5
:109930007C72FC603C744BF21C480BF02BFD019ACE
:109940003146384612F06CFEC1F6FF78069B88F867
:10995000084040464BF2304788E80802C1F6FF77DE
:1099600088F80940C8F80C4088F810400BF012FD48
:10997000019A3146404612F053FE3846C7F800B00F
:10998000C7F804A03C727C72FC603C740BF002FDD2
:10999000DDF804B04BF24448C1F6FF785A46314630
:1099A000384612F03DFE294640464FF0010588E852
:1099B000020288F8084088F80950C8F80C4088F876
:1099C000104044F270370BF0E5FC5A4631464046F1
:1099D00012F026FEC2F20007059B3C72384642F6A2
:1099E000E018C2F2000887E808047D72FC603C744D
:1099F0000BF0D0FC5A463146384612F011FE4BF6B9
:109A00000007089BC8F804304046C2F20007C8F8B7
:109A1000009088F8084088F80940C8F80C4088F899
:109A200010400BF0B7FC5A463146404612F0F8FDA4
:109A30004EF2FC28049DC7F800A03846C2F2000888
:109A40007D603C727C72FC603C740BF0A3FC5A4657
:109A50003146384612F0E4FD08F118020221404672
:109A6000F9F748F940F2E863C0F20F03404642F6C6
:109A70006479C2F20009C8F8003005F093FF089B32
:109A800089F8084048464AF27C77C2F2000789E824
:109A9000080189F80940C9F80C4089F810400BF01A
:109AA00079FC31465A46484612F0BAFD2A464FF034
:109AB0000103384687E804017B723C72FC603C7409
:109AC0000BF068FC31465A46384612F0A9FD44F2C4
:109AD000D043C2F2000340F2A452C0F20F021A6057
:109AE0000A221A720DF0B0F840F23463C2F2010398
:109AF00043F6F4651A680B92DDF82CE01A680C92B4
:109B00000C9F1B680D93C2F2000543F2BC444FF258
:109B100004214DF6A0724BF28813C2F20004C2F287
:109B20000001C2F200020D9E2860C1F6FF734FF0E3
:109B30007E50C4F800E00F60166018600FB0BDE8FA
:109B4000F08F00BF2DE9F04F4CF62814C2F200044C
:109B50008DB0204608F07CFC204608F021FA204613
:109B600008F016FA204608F0B9F8204608F0FCFA8A
:109B700020460022012108F0E7F941F6BC412046C9
:109B8000C0F202010E220BF0CFFF2046012200217D
:109B900008F0DAF941F6CC411022C0F20201204669
:109BA00043F6400A4FF268040BF0BEFFC2F2000415
:109BB000C2F2000A4FF47A7043F60C190DF06CF8FB
:109BC000C2F200095146204643F6D81808F0EEFECE
:109BD000C2F200084946204643F6A42708F0E6FEF4
:109BE000C2F200074146204643F6703608F0DEFE1A
:109BF000C2F200063946204643F63C4508F0D6FE40
:109C0000C2F200053146204608F0D0FE2946204623
:109C100008F0CCFE2046022108F0FEFE4BF6F46070
:109C20002146C2F2000008F0B3FD42F2C152504694
:109C3000C0F20002012108F01FFC41F2F112484677
:109C4000C0F20002022108F017FC41F2690240460E
:109C5000C0F20002032108F00FFC42F231523846F4
:109C6000C0F20002042108F007FC41F22D12304638
:109C7000C0F20002052108F0FFFB40F61D42C0F2D1
:109C80000002284606214EF2681408F0F5FBC2F2E5
:109C900000044BF65C512046C2F2000108F086FE3B
:109CA0004CF678112046C2F2000108F07FFE2046F3
:109CB000022108F0B1FE4AF640604AF29073214654
:109CC000C2F20003C2F2000000934BF2207408F0CD
:109CD0005FFD009B0193C2F200044AF65C0B19463B
:109CE000C2F2000B20464BF2944A08F05FFEC2F22B
:109CF000000A594620464AF6781908F057FEC2F283
:109D00000009514620464AF6442808F04FFEC2F2A8
:109D10000008494620464AF6103708F047FEC2F2CE
:109D20000007414620464AF6DC3608F03FFEC2F204
:109D300000063946204608F039FE31464AF674538B
:109D4000204600934AF6A84508F030FE009BC2F278
:109D50000005C2F2000329462046009308F026FEC3
:109D60000099204608F022FE2046022108F054FE09
:109D700042F6A0102146C2F2000008F009FD019B46
:109D800041F279721846C0F20002072108F074FB14
:109D900042F225225846C0F20002082108F06CFB6E
:109DA00042F2A5225046C0F20002092108F064FBED
:109DB00041F2F9624846C0F200020A2108F05CFB59
:109DC00041F679024046C0F200020B2108F054FB34
:109DD00042F2A5323846C0F200020C2108F04CFBDA
:109DE00041F67D123046C0F200020D2108F044FB1E
:109DF00041F2F9722846C0F200020E2108F03CFB45
:109E000040F26172C0F2000200980F214BF6D0249C
:109E100008F032FBC1F6FF744BF25C212046C1F61C
:109E2000FF7108F0C3FD4BF228312046C1F6FF71E7
:109E300008F0BCFD2046022108F0EEFD4CF24C106B
:109E40002146C2F2000042F2F85408F0A1FCC2F22E
:109E500000044BF654012046C2F2000108F0A6FDB2
:109E60004BF620112046C2F2000108F09FFD20466B
:109E7000022108F0D1FD42F648502146C2F200000E
:109E80004BF2B05408F084FCC2F200044BF6C4510B
:109E90002046C1F6FF7108F089FD4BF6906120461F
:109EA000C1F6FF7108F082FD2046022108F0B4FDE2
:109EB00044F284302146C2F200004CF6886408F077
:109EC00067FCC2F2000443F648512046C2F200018A
:109ED00008F06CFD43F614612046C2F2000108F060
:109EE00065FD2046022108F097FD4BF2C070214627
:109EF000C2F200004EF25C3408F04AFCC2F20004E8
:109F00004DF6C4012046C2F2000108F04FFD4DF6A7
:109F100090112046C2F2000108F048FD20460221BF
:109F200008F07AFD4CF698002146C2F2000042F695
:109F3000501408F02DFCC2F200044BF21C01204624
:109F4000C1F6FF7108F032FD4BF660312046C1F6D4
:109F5000FF7108F02BFD2046022108F05DFD4EF256
:109F600070002146C2F2000043F2180408F010FC11
:109F7000C2F2000442F2B4712046C2F2000108F0BD
:109F800015FD42F680012046C2F2000108F00EFDE8
:109F90002046022108F040FD4BF258402146C1F610
:109FA000FF704BF6180408F0F3FBC1F6FF744CF297
:109FB000D0412046C2F2000108F0F8FC4CF29C515E
:109FC0002046C2F2000108F0F1FC2046022108F010
:109FD00023FD43F608502146C2F200004CF26864AB
:109FE00008F0D6FBC2F200044DF6A8412046C2F2AA
:109FF000000108F0DBFC4EF2B0612046C2F2000125
:10A0000008F0D4FC2046022108F006FD4EF2B810FC
:10A0100042F2FC132146C2F20003C2F20000009398
:10A020004BF20C2408F0B4FB009B0B93C1F6FF74B9
:10A0300042F2C82B1946C2F2000B204642F2943A73
:10A0400008F0B4FCC2F2000A5946204642F26049C8
:10A0500008F0ACFCC2F200095146204608F0A6FC0C
:10A0600042F22C584946204608F0A0FCC2F20008F3
:10A0700042F2486341461D46204608F097FC2B46B5
:10A08000C2F200034BF298071D46C2F200074BF2E2
:10A09000FC2339461E46204608F088FC3346C2F2AF
:10A0A00000031E464BF2C8330695294620461D463E
:10A0B00008F07CFC2B46C2F200031D4643F21C3321
:10A0C0000796314620461E4608F070FC3346C2F221
:10A0D00000031E4643F2E8330895294620461D46F4
:10A0E00008F064FC2B46C2F200031D464CF64423E4
:10A0F0000996314620461E4608F058FC3346C2F207
:10A100000003294620464CF6503605930A95C2F2C4
:10A11000000608F04BFC0599204608F047FC314644
:10A1200043F28C522046009243F2C04508F03EFCB8
:10A13000009AC2F2000543F25863C2F200022946B7
:10A1400020460193009208F031FC0199C2F200010F
:10A15000019143F2247200990292204608F026FCF5
:10A16000029A0199C2F200024CF6B85320460292BC
:10A17000039308F01BFC039B02994BF6B82EC2F226
:10A1800000032046CDF810E0039308F00FFC04997B
:10A19000C2F2000104912046039908F007FC0499DB
:10A1A000204608F003FC2046022108F035FC4FF25F
:10A1B000B8002146C2F2000008F0EAFA0B9B41F613
:10A1C00009221846C0F20002102108F055F941F6A4
:10A1D00089225846C0F20002112108F04DF941F6DB
:10A1E00009325046C0F20002122108F045F942F24D
:10A1F000A5124846C0F20002132108F03DF941F2D1
:10A20000F9524046C0F20002142108F035F941F637
:10A2100089323846C0F20002152108F02DF941F2CA
:10A2200079620698C0F20002162108F025F942F280
:10A23000B1420798C0F20002172108F01DF941F25F
:10A2400079520898C0F20002182108F015F942F27C
:10A2500031420998C0F20002192108F00DF941F6C7
:10A2600091420A98C0F200021A2108F005F941F65D
:10A270008D620598C0F200021B2108F0FDF841F63E
:10A2800011523046C0F200021C2108F0F5F842F2EB
:10A2900099022846C0F200021D2108F0EDF841F6AF
:10A2A00091520098C0F200021E2108F0E5F841F634
:10A2B00099720198C0F200021F2108F0DDF842F205
:10A2C00025320298C0F20002202108F0D5F842F2AF
:10A2D00019120398C0F20002212108F0CDF841F6CE
:10A2E0000D72C0F20002049822214EF6806408F03C
:10A2F000C3F8C2F200044AF6CC712046C2F2000153
:10A3000008F054FB4BF264112046C2F2000108F041
:10A310004DFB2046022108F07FFB4BF6140021463E
:10A32000C2F200004BF2707408F032FAC2F200047C
:10A330004EF230212046C2F2000108F037FB44F211
:10A34000C4312046C2F2000108F030FB2046022151
:10A3500008F062FB4DF2F4702146C2F2000042F6B2
:10A36000486408F015FAC2F200044DF67451204614
:10A37000C2F2000108F01AFB4DF640612046C2F21D
:10A38000000108F013FB2046022108F045FB4CF6C3
:10A3900010302146C2F200004CF28C1408F0F8F99B
:10A3A000C2F200044BF230212046C2F2000108F054
:10A3B000FDFA4BF230612046C1F6FF7108F0F6FA63
:10A3C0002046022108F028FB4CF638102146C2F244
:10A3D00000004DF2082408F0DBF9C2F200044CF250
:10A3E00038312046C2F2000108F0E0FA4CF2044194
:10A3F0002046C2F2000108F0D9FA2046022108F0F6
:10A400000BFB44F21C002146C2F200004BF26054E8
:10A4100008F0BEF9C2F2000443F64C712046C2F2C5
:10A42000000108F0C3FA4DF258212046C2F20001A3
:10A4300008F0BCFA2046022108F0EEFA4BF6203074
:10A440002146C1F6FF704DF60C7408F0A1F9C2F276
:10A4500000044BF204612046C2F2000108F0A6FAA3
:10A4600042F67C412046C2F2000108F09FFA2046E5
:10A47000022108F0D1FA43F6F8602146C2F200004A
:10A480004DF6740408F084F9C2F200044EF2C8419B
:10A490002046C2F2000108F089FA4EF2945120469B
:10A4A000C2F2000108F082FA2046022108F0B4FA54
:10A4B0004AF68C702146C2F200004FF2082408F0E0
:10A4C00067F9C2F200044DF270012046C2F20001A9
:10A4D00008F06CFA4DF23C112046C2F2000108F07F
:10A4E00065FA2046022108F097FA4BF2CC1021467B
:10A4F000C1F6FF704CF6685408F04AF9C2F2000445
:10A5000043F268012046C2F2000108F04FFA4DF212
:10A5100068312046C2F2000108F048FA20460221C4
:10A5200008F07AFA4EF21C302146C2F2000042F2E4
:10A53000647408F02DF9C2F200044BF24C7120460D
:10A54000C1F6FF7108F032FA4BF668012046C1F6F9
:10A55000FF7108F02BFA2046022108F05DFA4DF653
:10A5600034002146C2F200004CF2A82408F010F991
:10A57000C2F200044BF298412046C1F6FF7108F088
:10A5800015FA4BF264512046C1F6FF7108F00EFA3D
:10A590002046022108F040FA4BF650402146C2F214
:10A5A00000004DF6283408F0F3F8C2F200044DF232
:10A5B00034412046C2F2000108F0F8F94DF2005192
:10A5C0002046C2F2000108F0F1F92046022108F00D
:10A5D00023FA4DF228302146C2F200004BF2E80483
:10A5E00008F0D6F8C1F6FF744BF638112046C1F6D4
:10A5F000FF7108F0DBF94BF604212046C1F6FF712C
:10A6000008F0D4F92046022108F006FA4EF2E800DC
:10A610002146C2F2000043F2CC2408F0B9F8C2F29D
:10A62000000442F6F4112046C2F2000108F0BEF91F
:10A6300042F6C0212046C2F2000108F0B7F92046D8
:10A64000022108F0E9F94CF628502146C2F2000038
:10A650004BF2FC6408F09CF8C1F6FF744DF25C61AB
:10A660002046C2F2000108F0A1F944F25C01204644
:10A67000C2F2000108F09AF92046022108F0CCF954
:10A680004FF2C4102146C2F200004EF2AC3408F082
:10A690007FF8C2F200044AF680612046C2F200014F
:10A6A00008F084F94BF6EC112046C2F2000108F0E4
:10A6B0007DF92046022108F0AFF94DF21C602146D9
:10A6C000C2F200004CF6D80408F062F8C2F20004AE
:10A6D0004FF2F8012046C2F2000108F067F94DF68A
:10A6E0005C212046C2F2000108F060F920460221F8
:10A6F00008F092F944F230302146C2F200004EF2E6
:10A70000606408F045F8C2F2000442F69861204601
:10A71000C2F2000108F04AF94DF228712046C2F257
:10A72000000108F043F92046022108F075F94AF6C5
:10A730004C702146C2F200004CF2B86408F028F8D0
:10A74000C2F200044EF6D0612046C2F2000108F0C9
:10A750002DF94EF69C712046C2F200014BF6347B77
:10A7600008F024F9C2F2000B2046022108F054F947
:10A770004CF6D8662146584608F00AF8C2F20006A0
:10A7800041F20D5244F2E025C0F20002C2F200058F
:10A790003046272107F070FE3146284608F006F9BA
:10A7A0004CF6A4712846C2F200014EF2281A08F0B5
:10A7B000FDF8C2F2000A284602214BF684374BF21C
:10A7C000D06408F029F9C2F20004C2F20007294659
:10A7D00050464BF6904807F0DBFFC2F200083946BE
:10A7E000204644F2281608F0E1F8C2F2000641467D
:10A7F00020464BF6286508F0D9F8C2F2000531462C
:10A80000204608F0D3F84CF2F8292946204608F0F3
:10A81000CDF8C2F200092046022108F0FDF82146D9
:10A82000484607F0B5FF42F219023846C0F200026E
:10A83000232107F021FE41F6FD024046C0F200024E
:10A84000242107F019FE41F611623046C0F20002E1
:10A85000252107F011FE41F60142C0F20002284610
:10A86000262143F2F07407F007FEC2F200044BF613
:10A87000F8412046C1F6FF7108F098F84BF62C41DC
:10A880002046C1F6FF714DF65C7808F08FF8C2F2F1
:10A8900000082046022108F0BFF84CF61C052146AE
:10A8A000404607F075FFC2F200054CF2DC11284665
:10A8B000C2F2000108F07AF84CF61C412846C2F2B8
:10A8C00000014DF67C3708F071F8C2F20007284607
:10A8D000022108F0A1F84BF238142946384607F057
:10A8E00057FFC1F6FF7443F234112046C2F2000153
:10A8F00008F05CF843F200212046C2F200014BF25E
:10A900008C1608F053F8C1F6FF762046022108F0B5
:10A9100083F84AF628152146304607F039FFC2F27F
:10A9200000054BF674712846C2F2000108F03EF8AB
:10A930004DF6BC334CF280011C462846C2F20001A1
:10A9400008F034F82346C2F200032846022100939F
:10A950004DF2CC5408F060F82946009807F018FF33
:10A96000C2F200044CF22C712046C2F2000108F041
:10A970001DF84CF6E84242F6B03115462046C2F2C8
:10A98000000108F013F82A46C2F200022046022114
:10A99000019242F2147508F03FF82146019807F041
:10A9A000F7FEC2F200054DF6A4712846C2F200017E
:10A9B00007F0FCFF4EF2FC312846C2F200014CF2D7
:10A9C000400407F0F3FFC2F200042846022102947B
:10A9D00008F022F84DF6FC3429460298C2F2000431
:10A9E00007F0D6FE4BF6F4612046C2F2000108F0F3
:10A9F000ABF84AF640612046C2F2000108F0A4F824
:10AA00004FF2B80542F6A011C2F200052046C2F28C
:10AA1000000108F099F82946204608F095F84CF214
:10AA20004C112046C2F2000108F08EF842F648515F
:10AA30002046C2F2000108F087F844F28431204633
:10AA4000C2F2000108F080F84BF2C0712046C2F259
:10AA5000000108F079F84CF698012046C2F2000196
:10AA600008F072F84EF270012046C2F2000108F0C0
:10AA70006BF84BF258412046C1F6FF7108F064F8BC
:10AA800043F608512046C2F2000108F05DF84EF28C
:10AA9000B8112046C2F2000108F056F829462046B7
:10AAA00008F052F84BF614012046C2F2000108F0FB
:10AAB0004BF84DF2F4712046C2F2000108F044F860
:10AAC0004CF610312046C2F2000108F03DF84CF679
:10AAD00038112046C2F2000108F036F844F21C0199
:10AAE0002046C2F2000108F02FF84BF62031204634
:10AAF000C1F6FF7108F028F843F6F8612046C2F26B
:10AB0000000108F021F84AF68C712046C2F20001DB
:10AB100008F01AF84BF2CC112046C1F6FF7108F08C
:10AB200013F84EF21C312046C2F2000108F00CF876
:10AB30004DF634012046C2F2000108F005F84BF64C
:10AB400050412046C2F2000107F0FEFF4DF22831CD
:10AB50002046C2F2000107F0F7FF4EF2E80120465E
:10AB6000C2F2000107F0F0FF4CF628512046C2F275
:10AB7000000107F0E9FF4FF2C4112046C2F20001C4
:10AB800007F0E2FF4DF21C612046C2F2000107F01F
:10AB9000DBFF44F230312046C2F2000107F0D4FF5F
:10ABA0004AF64C712046C2F2000107F0CDFF59462B
:10ABB000204607F0C9FF5146204607F0C5FF494629
:10ABC000204607F0C1FF4146204607F0BDFF394649
:10ABD000204607F0B9FF3146204607F0B5FF00993F
:10ABE000204607F0B1FF0199204607F0ADFF02991A
:10ABF000204607F0A9FF2046022107F0DFFF4CF6B0
:10AC00006C062046012107F0D3FFC2F20006204661
:10AC10004EF6606507F0F6FFC2F200052922FF211B
:10AC2000304612F071F800242846347008F016F807
:10AC300005F1100008F012F820460BF03DFA49F239
:10AC4000F32144F29043C2F20003C1F6FF71632284
:10AC500008701C775C619A6172B69042A8BF10467A
:10AC60008000D86062B643F2B442C2F200020878B3
:10AC700083F83C4005215C631060996372B6DC6226
:10AC800062B654600DB0BDE8F08F00BF70B5022110
:10AC900082B004200BF09CFF02211E200BF098FFD5
:10ACA000FEF750FF41F6E040C0F20200F5F746FD26
:10ACB00041F62450C0F20200F5F740FD41F6545031
:10ACC000C0F20200F5F73AFD41F68450C0F20200EE
:10ACD00049F2E865F5F728FDC1F6FF754EF224410B
:10ACE0000A22C0F20C01002328460AF0A3FF41F615
:10ACF0009850C0F20200F5F721FD28460AF088FFBF
:10AD000041F6A050C0F20200F5F718FD40F6E4400D
:10AD10000BF0B2FC044600F02FFC4BF20063C2F2D1
:10AD2000000301261C60FAF729F8FCF7D1F9FAF7BD
:10AD3000E1F94EF28813CEF2000340F2002044F213
:10AD4000D0441E60C2F200048021C1F6FF700AF0F8
:10AD5000C3F9204603F0B8FC204602F071FDB7EEBF
:10AD6000000A204603F08AF9E288242122F010022A
:10AD7000204602F0BDFBF6EE000AB0EE600A204667
:10AD800002F058FEE288204622F48072242102F06C
:10AD9000AFFB1C21204602F0C9FD204603F0EAFA71
:10ADA0000221204602F0D6FC204602F051FC20464B
:10ADB00002F0CCFB41F6B050C0F20200F5F7BEFC49
:10ADC00049F2F323C1F6FF7340F20E641878FAF7E4
:10ADD0002FFB40F20C61C2F2010440F20862C2F2A1
:10ADE000010140F28C53C2F20102C2F2010341F6AA
:10ADF000CC50248809881480C0F202001980F5F72D
:10AE000093FC802128460AF0A5FE41F6E450C0F2EA
:10AE10000200F5F789FC40F65A3128460AF09AFEFE
:10AE200041F6F850C0F20200F5F788FC4EF2081324
:10AE3000CEF2000341F6FC501E60C0F20200F5F7AE
:10AE40007DFC28460AF0E4FEFAF7BEFC40F23462CC
:10AE5000C2F201024DF6A07312680192C2F2000321
:10AE6000019A1A6002B070BD2DE9F04F2DED068BEE
:10AE70004BF28813844683B0C1F6FF7300F6A844F2
:10AE800093ED000AD4ED008ADCF87CEC9FEDA35A28
:10AE9000DFEDA30A0CF6944300F6C44500F6AC4976
:10AEA00000F54B681C4600F6A44001930CF69C4349
:10AEB0000CF5496B90ED008A93ED00AAD5ED004AA0
:10AEC00099ED003AD8ED003ADBED002A94ED004A06
:10AED0000CF54A630CF69840D3ED009A90ED001AF9
:10AEE00002F1FE030239A2F1020A0093F6EE001A03
:10AEF000B7EE002ABFEE009ABEF1000F9FED896AFF
:10AF000040F30881DCF8806CF0EE465A0CF53C709A
:10AF1000002550F8307C50F8343C50F82C2C50F878
:10AF2000284C3B4402EB234201359BB2A2422DB296
:10AF300040F82C2C40F8303C04DD50F8244C121B17
:10AF400040F82C2C06EB420436F91220B4F90270BA
:10AF500010ED087A50ED076ABF1A03FB07F302EB06
:10AF6000234307EE903AF8EEE77A67EE266A67EE3B
:10AF7000877A40ED086A67EE857AF5EEC07AF1EEE1
:10AF800010FA0EDD24EEA77AE7EEC77AB0EE677A04
:10AF9000F1EE667AB4EEE77AF1EE10FA58BFF0EE11
:10AFA000477A50ED036A10ED027A7545E7EEA65A2E
:10AFB00000F13400A7EE876AABDB36EE637A75EEFC
:10AFC000C37AE7EE283A019BA7EEA83AE1EE042AFD
:10AFD00036EE637AA2EEC14AA7EE086A75EEC37A2E
:10AFE00026EE297AE7EE885AA4EE076A65EE8A7A99
:10AFF00026EE216AE4EE275AB4EEC26AF1EE10FAA8
:10B0000089ED003A65EEA15AC8ED003ACBED002A71
:10B0100083ED004A76DDB7EE006AF4EEC25AF1EE37
:10B0200010FA67DDF7EE005A65EE805A26EE006AE8
:10B0300065EEA05A26EE206AFDEEE57A17EE902A1C
:10B04000FDEEC67A2AF8022F17EE903A21F8023F59
:10B05000009B9A457FF450AFDFED337AB0EEC33AF0
:10B06000B4EEE73ADFED307AF1EE10FAF0EEE33AC3
:10B0700048BF0023F4EEE73A48BFC9F80030F1EECC
:10B0800010FA44BF0023C8F80030BEF1000F2CDDD9
:10B0900000239FED267A1E46342706E0DCF87CEC80
:10B0A000013636B2764533461FDA07FB03C3D3EDCC
:10B0B000B47A0EF1FF3EF4EEC77A07FB0EC4F1EE50
:10B0C00010FA04F52F7403F52F75E7D50FCCCCF8E3
:10B0D0007CEC0FC50FCC0FC50FCC0FC5013636B2B7
:10B0E00023682B6076453346DFDB03B0BDEC068B6F
:10B0F000BDE8F08FF4EE495AF1EE10FA48BFF0EED9
:10B10000495A91E7B4EE496AF1EE10FA48BFB0EE41
:10B11000496A82E7F0EE465A4FE700BF0000003868
:10B1200000FEFF4600000000FFE6DB2E17B7D13817
:10B1300041689FED157AD1ED056ADFED147AE6EEF0
:10B14000877A4FF4884243F2C673C4F22C72C3F27A
:10B15000BE7310B58260C360044617EE900A10F00B
:10B160004FFD41EC100B0FF097F851EC100B11F064
:10B1700093F8DFED077A07EE100A67EE277A04F6F8
:10B180009844C4ED007A10BD3D0AC7403D0A27C06F
:10B19000716415392DE9F84307292DED028B4668B6
:10B1A0005DD00FD9402901D0422936D102F04004A8
:10B1B000E4B2C0F88C4C002C64D0BDEC028B0120B2
:10B1C000BDE8F883012928D107EE902ADFED506A07
:10B1D0009FED507AF8EE677A00F6DC4367EEA67AC8
:10B1E000F4EEC77AF1EE10FAC3ED007AE5DD00F671
:10B1F0009C4300F54A60C3ED007AC0ED007AD6EDBD
:10B20000046AB6EE007AF4EEC76AF1EE10FAD4D50D
:10B21000F1EE677AC0ED007ACFE77A29CDD9037CC9
:10B220007BB103EB430203EB820247F2A401C3F6B6
:10B230007D7100EB82020346C3F8D41234339A4284
:10B24000FAD1BDEC028B00F6C8430022C4F22032D2
:10B250000021C0F88C1C01201A60BDE8F88312FBA5
:10B2600002F207EE902ABDEC028BF8EEE77A9FED32
:10B270002A7A67EE877A00F6D840C0ED007A01207E
:10B28000BDE8F883027C002A97D007460546B1EE58
:10B29000048A03E0A24205F134058EDDD5F8EC32D4
:10B2A000802B04F10104F5D1D7F88C3C002BF1D1AF
:10B2B000F86880F0004010F0A3FCD6ED017A67EE4C
:10B2C000887A804617EE900A894610F099FC0B4662
:10B2D00041F6B8610246C4F21D014FF0A04010F0E3
:10B2E0002FFB41EC100B0EF0D7FF404653EC102B18
:10B2F000494610F0D9FC41EC100B0EF0CDFF51EC9B
:10B30000100B10F0C9FFC5F8D4023A7CC2E700BFA9
:10B310002497FF3BCDCC4C3DACC5A73770B54568F5
:10B32000D0ED035A95ED024A95ED036A9FED697AD7
:10B330009FED695AF2EE084AF9EE087AE4EE247AB3
:10B3400000F6A44300F6A846F1EE006A2DED028B4C
:10B3500066EE266ABFEE008AF0EE484AE6EE264A1E
:10B360000446FDEEE77AF6EE008A17EE902AC0F862
:10B37000882CC3ED004AD5ED037AF4EEE87AF1EEBD
:10B3800010FAD4BFF0EE457AF0EE477AC6ED007AB7
:10B3900065EEE77A17EE900A10F032FC41EC100BE4
:10B3A0000EF07AFF51EC100B10F076FF07EE100A4A
:10B3B000F7EE007A77EEC77AB0EE007AC6ED007A43
:10B3C000D5ED047AA7EE878A04F69C4204F54A6319
:10B3D00082ED008A83ED008A95ED047AB4EEE87A76
:10B3E000F1EE10FA03D5F1EE487AC3ED007ADFED05
:10B3F0003B6A95ED056A9FED3A7AD4ED037A9FEDAD
:10B40000398AA6EE267A04F6984627EE888A17EE41
:10B41000100A10F0F5FB41EC100B0EF03DFF51EC63
:10B42000100B10F039FF07EE900A27EE888AF7EE2E
:10B43000007A86ED008A95ED067A77EE277A04F693
:10B44000D44377EE877AF5EE006AC3ED007A95ED86
:10B45000067AB4EEE67AF1EE10FA09D5B0EE086A93
:10B46000F6EE086AE7EE466A77EEE67AC3ED007A12
:10B4700095ED077A9FED1C6ADFED1C7ADFED1C6A03
:10B4800027EE067A04F6844383ED007A95ED097A77
:10B49000B6EE006A37EE467A04F6B84383ED007ADA
:10B4A00095ED0A7A67EE277A04F54C6367EE877AA2
:10B4B00004F6BC410022C1ED007ABDEC028B1A609B
:10B4C000D5ED0B7A67EEA67A04F6C444C4ED007A93
:10B4D00070BD00BF00C05A4600409C453D0AC740B1
:10B4E0003D0A27C0560EC9408FC2F53C2DB29D3D86
:10B4F0006666E63FF0B547F2A4040025C3F67D7406
:10B50000034600F51C61C3F8D052C3F8D44234336B
:10B510008B424FF00002F6D100F6D8454CF6CD47ED
:10B52000C3F64C6700F6C84400262F600023C4F21F
:10B53000203600F69845266000F5496EC0F87C3C40
:10B54000C0F88C3C00F54B6700F6AC4600F694441E
:10B550004CF6CD4100F54E632A60C3F64C714FF0B6
:10B560007E55CEF800203A60326025601960BDE853
:10B57000F040FFF7D3BE00BFF8B54FF4884243F266
:10B58000C67342F26011C0F20201C4F22C72C3F21F
:10B59000BE73044601608260C36030200BF06EF819
:10B5A00003464FF07C571F6060602046FFF7B6FEF1
:10B5B000636820465F60FFF7B1FE636820469F60C6
:10B5C000FFF7ACFE63682046DF60FFF7A7FE636805
:10B5D00020461F61FFF7A2FE636846F26662C3F66B
:10B5E00026725A612046FFF799FE63684FF07A523F
:10B5F0009A612046FFF792FE63682046DF61FFF7FD
:10B600008DFE63680126267420465F62FFF786FE82
:10B61000636848F20612C3F615629A622046FFF785
:10B620007DFE63680025DD622046FFF777FE42F26B
:10B630006C13C0F20203C4F8803C24236361272307
:10B64000A3612B2323652D2363653023C4F88C303D
:10B650003323C4F890303723C4F8C8303923C4F8F2
:10B66000CC303C23C4F804313F23C4F808314323D1
:10B67000C4F840314523C4F844314823C4F87C3130
:10B680004B23C4F880314F23C4F8B8315123C4F898
:10B69000BC315423C4F8F4315723C4F8F8315B2388
:10B6A000C4F830325D23C4F834326023C4F86C32FD
:10B6B00040F2E733C4F870320023E36142F21C1316
:10B6C000236241F23013636242F21D13236343F697
:10B6D0007873636341F22733A36343F6797363643A
:10B6E00048F20573A36441F6FE03E36448F206736F
:10B6F000A3654AF2A813E36540F6627323664AF233
:10B70000A913E3664BF2C023236740F261636367CA
:10B710004BF2C123C4F880304FF6BB63C4F88430C9
:10B7200041F27D43C4F888304FF6BC63C4F89430CE
:10B730004CF2496366F31F43294648F6230040F65E
:10B740009B0566F31F40C4F8B050C4F8D43041F6EE
:10B75000C14242F6D40343F2223E4FF2AD2566F3D6
:10B760001F4266F31F4E66F31F45C4F8C000C4F8BD
:10B77000D8304FF4C75043F2233745F21F5366F3D6
:10B780001F47C4F89820C4F8ACE0C4F8C400C0F265
:10B790000203C4F8E85048F624024CF24A6E43F221
:10B7A000F1204AF2334566F31F4266F31F4EC4F898
:10B7B000BC70C0F20200C0F20205C4F8103141F6BC
:10B7C000C24C41F2BC034FF2AE2766F31F4766F34B
:10B7D0001F4CC4F8D020C4F8E4E0C4F8FC00C4F85E
:10B7E000143140F61B40C4F8245143F2F22240F6D3
:10B7F0004C7545F220564AF2344E41F63673C0F28B
:10B800000202C0F20206C4F8F870C0F2020E41F261
:10B810006147C4F80001C0F20303C4F828514FF295
:10B82000DE0040F67935C4F8EC70C0F20200C4F8CE
:10B830000C21C4F82061C4F89C50C4F8A8C045F29B
:10B840007376C4F834E1C4F84C3141F27C23C0F281
:10B850000306C4F83801C4F8503149F249104CF6D7
:10B86000CB03C0F20300C0F20303C4F8606141F2ED
:10B870007D26C4F86461C4F87401C4F8883140F6C8
:10B88000ED0041F202034FF2DF0241F6377740F656
:10B890004746C0F20202C0F20307C4F83C51C0F2AE
:10B8A0000406C4F87801C4F88C3145F2747544F686
:10B8B0008F6047F69033C0F20305C4F84821C4F8FE
:10B8C0005C71C0F20400C0F20403C4F89C6149F248
:10B8D0004A1241F203064CF6CC07C0F20302C0F252
:10B8E0000307C4F87051C4F8A061C4F8B001C4F8EB
:10B8F000C43140F6196040F68E1340F648454CF2CC
:10B90000F646C0F20405C4F88421C4F89871C0F268
:10B910000406C4F8B401C4F8C83144F6906247F68E
:10B92000913740F6D81045F2D923C0F20402C0F294
:10B930000407C4F8AC51C0F20500C0F20503C4F816
:10B94000D8614CF2F74541F68606C0F20405C4F80A
:10B95000C021C4F8D471C4F8DC61C4F8EC01C4F8A7
:10B96000003240F6EB0040F6812340F6D91245F252
:10B97000DA2749F26B46C0F20502C0F20507C0F2B1
:10B980000506C4F8E851C4F8F001C4F8043249F2DD
:10B990006C454DF6AD2043F21D23C0F20505C0F203
:10B9A0000500C4F8FC21C0F20603C4F810729D2201
:10B9B000C4F8146241F21216C0F2060245F21737BB
:10B9C000C4F81862C4F8245247F208264DF6AE2592
:10B9D000C4F82802C4F8643241F2694041F2AA1363
:10B9E000C0F20505C0F20607C0F20606C4F82C0234
:10B9F000C4F860229C2043F21E22C4F8683245F24B
:10BA00001633C0F20600C0F20603C0F20602C4F804
:10BA10009C7240F6790E40F6FB27C4F8A062C4F889
:10BA2000385240F60216C4F84C5247F2A405C4F846
:10BA30003C02C4F85002C4F87832C4F88C32C4F81E
:10BA4000A4E2C3F67D75C4F84072C4F85472C4F819
:10BA50007422C4F88822C4F87C62C4F89062234639
:10BA600004F51C60C3F8D012C3F8D45234338342B7
:10BA70004FF00002F6D104F6D8464CF6CD4704F656
:10BA8000C840C3F64C6700253760002304F698468B
:10BA9000C4F22035056004F5496EC4F87C3CC4F856
:10BAA0008C3C04F6AC4004F54E6304F54B6704F699
:10BAB00094454CF6CD413260C3F64C714FF07E5642
:10BAC000CEF800203A60026020462E601960FFF731
:10BAD00025FC2046F8BD00BF70B545689FED6C7A27
:10BAE00095ED025A95ED036AF2EE085AF9EE087ADE
:10BAF000E5EE257A00F6A44300F6A846F1EE006ACA
:10BB00002DED028B66EE266ABFEE008AF0EE485AF3
:10BB1000E6EE265A0446FDEEE77A85ED000A17EEBA
:10BB2000902AC0F8882CC3ED005A95ED036ADFED2A
:10BB3000597AD0ED036AF6EE008AB4EEE86AF1EEC7
:10BB400010FAC8BFF0EE477AC6ED007A66EEE77AE3
:10BB500017EE900A10F054F841EC100B0EF09CFB1D
:10BB600051EC100B10F098FB07EE100AF7EE007A7C
:10BB700077EEC77AB0EE007AC6ED007AD5ED047A9A
:10BB8000A7EE878A04F69C4204F54A6382ED008A98
:10BB900083ED008A95ED047AB4EEE87AF1EE10FABE
:10BBA00003D5F1EE487AC3ED007ADFED3B6A95EDFF
:10BBB000056A9FED3A7AD4ED037A9FED398AA6EEB5
:10BBC000267A04F6984627EE888A17EE100A10F0B7
:10BBD00017F841EC100B0EF05FFB51EC100B10F05E
:10BBE0005BFB07EE900A27EE888AF7EE007A86ED77
:10BBF000008A95ED067A77EE277A04F6D44377EE3D
:10BC0000877AF5EE006AC3ED007A95ED067AB4EE18
:10BC1000E67AF1EE10FA09D5B0EE086AF6EE086A97
:10BC2000E7EE466A77EEE67AC3ED007A95ED077A9D
:10BC30009FED1C6ADFED1C7ADFED1C6A27EE067AA9
:10BC400004F6844383ED007A95ED097AB6EE006A36
:10BC500037EE467A04F6B84383ED007A95ED0A7A1A
:10BC600067EE277A04F54C6367EE877A04F6BC41E9
:10BC70000022C1ED007ABDEC028B1A60D5ED0B7A83
:10BC800067EEA67A04F6C444C4ED007A70BD00BF26
:10BC900000C05A4600409C453D0AC7403D0A27C0A7
:10BCA000560EC9408FC2F53C2DB29D3D6666E63FFB
:10BCB00070B545689FED6C7A95ED025A95ED036A73
:10BCC000F2EE085AF9EE087AE5EE257A00F6A4437A
:10BCD00000F6A846F1EE006A2DED028B66EE266AAC
:10BCE000BFEE008AF0EE485AE6EE265A0446FDEE14
:10BCF000E77A85ED010A17EE902AC0F8882CC3ED8B
:10BD0000005A95ED036ADFED597AD0ED036AF6EE3D
:10BD1000008AB4EEE86AF1EE10FAC8BFF0EE477A96
:10BD2000C6ED007A66EEE77A17EE900A0FF068FF2C
:10BD300041EC100B0EF0B0FA51EC100B10F0ACFA15
:10BD400007EE100AF7EE007A77EEC77AB0EE007AC7
:10BD5000C6ED007AD5ED047AA7EE878A04F69C42F8
:10BD600004F54A6382ED008A83ED008A95ED047A3A
:10BD7000B4EEE87AF1EE10FA03D5F1EE487AC3EDAD
:10BD8000007ADFED3B6A95ED056A9FED3A7AD4EDD6
:10BD9000037A9FED398AA6EE267A04F6984627EEB6
:10BDA000888A17EE100A0FF02BFF41EC100B0EF0F3
:10BDB00073FA51EC100B10F06FFA07EE900A27EEB1
:10BDC000888AF7EE007A86ED008A95ED067A77EE9E
:10BDD000277A04F6D44377EE877AF5EE006AC3ED4E
:10BDE000007A95ED067AB4EEE67AF1EE10FA09D50E
:10BDF000B0EE086AF6EE086AE7EE466A77EEE67A93
:10BE0000C3ED007A95ED077A9FED1C6ADFED1C7A91
:10BE1000DFED1C6A27EE067A04F6844383ED007A90
:10BE200095ED097AB6EE006A37EE467A04F6B84325
:10BE300083ED007A95ED0A7A67EE277A04F54C6374
:10BE400067EE877A04F6BC410022C1ED007ABDECB2
:10BE5000028B1A60D5ED0B7A67EEA67A04F6C4441D
:10BE6000C4ED007A70BD00BF00C05A4600409C453A
:10BE70003D0AC7403D0A27C0560EC9408FC2F53C57
:10BE80002DB29D3D6666E63F70B545689FED6B7AC5
:10BE900095ED036AF2EE085AF9EE087AE0EE257A9B
:10BEA00000F6A44300F6A846F1EE006A2DED028BE1
:10BEB00066EE266ABFEE008AF0EE485AE6EE265A93
:10BEC0000446FDEEE77A85ED020A17EE902AC0F8E7
:10BED000882CC3ED005A95ED036ADFED597AD0ED59
:10BEE000036AF6EE008AB4EEE86AF1EE10FAC8BF13
:10BEF000F0EE477AC6ED007A66EEE77A17EE900A22
:10BF00000FF07EFE41EC100B0EF0C6F951EC100B59
:10BF100010F0C2F907EE100AF7EE007A77EEC77A52
:10BF2000B0EE007AC6ED007AD5ED047AA7EE878AE6
:10BF300004F69C4204F54A6382ED008A83ED008A90
:10BF400095ED047AB4EEE87AF1EE10FA03D5F1EE4D
:10BF5000487AC3ED007ADFED3B6A95ED056A9FED07
:10BF60003A7AD4ED037A9FED398AA6EE267A04F662
:10BF7000984627EE888A17EE100A0FF041FE41EC32
:10BF8000100B0EF089F951EC100B10F085F907EE4B
:10BF9000900A27EE888AF7EE007A86ED008A95ED02
:10BFA000067A77EE277A04F6D44377EE877AF5EEB1
:10BFB000006AC3ED007A95ED067AB4EEE67AF1EE0A
:10BFC00010FA09D5B0EE086AF6EE086AE7EE466A9E
:10BFD00077EEE67AC3ED007A95ED077A9FED1C6A5D
:10BFE000DFED1C7ADFED1C6A27EE067A04F6844347
:10BFF00083ED007A95ED097AB6EE006A37EE467A5F
:10C0000004F6B84383ED007A95ED0A7A67EE277A55
:10C0100004F54C6367EE877A04F6BC410022C1ED5B
:10C02000007ABDEC028B1A60D5ED0B7A67EEA67A2A
:10C0300004F6C444C4ED007A70BD00BF00C05A4687
:10C0400000409C453D0AC7403D0A27C0560EC940E6
:10C050008FC2F53C2DB29D3D6666E63F70B54568E2
:10C060009FED6B7AD5ED025AB2EE086AF9EE087AC6
:10C07000E5EE867A00F6A44300F6A846F1EE006AE3
:10C080002DED028B60EE266ABFEE008AB0EE486AA4
:10C09000A0EE266A0446FDEEE77A85ED030A17EE68
:10C0A000902AC0F8882C83ED006A95ED036ADFEDD5
:10C0B000597AD0ED036AF6EE008AB4EEE86AF1EE42
:10C0C00010FAC8BFF0EE477AC6ED007A66EEE77A5E
:10C0D00017EE900A0FF094FD41EC100B0EF0DCF817
:10C0E00051EC100B10F0D8F807EE100AF7EE007ABA
:10C0F00077EEC77AB0EE007AC6ED007AD5ED047A15
:10C10000A7EE878A04F69C4204F54A6382ED008A12
:10C1100083ED008A95ED047AB4EEE87AF1EE10FA38
:10C1200003D5F1EE487AC3ED007ADFED3B6A95ED79
:10C13000056A9FED3A7AD4ED037A9FED398AA6EE2F
:10C14000267A04F6984627EE888A17EE100A0FF032
:10C1500057FD41EC100B0EF09FF851EC100B10F056
:10C160009BF807EE900A27EE888AF7EE007A86EDB4
:10C17000008A95ED067A77EE277A04F6D44377EEB7
:10C18000877AF5EE006AC3ED007A95ED067AB4EE93
:10C19000E67AF1EE10FA09D5B0EE086AF6EE086A12
:10C1A000E7EE466A77EEE67AC3ED007A95ED077A18
:10C1B0009FED1C6ADFED1C7ADFED1C6A27EE067A24
:10C1C00004F6844383ED007A95ED097AB6EE006AB1
:10C1D00037EE467A04F6B84383ED007A95ED0A7A95
:10C1E00067EE277A04F54C6367EE877A04F6BC4164
:10C1F0000022C1ED007ABDEC028B1A60D5ED0B7AFE
:10C2000067EEA67A04F6C444C4ED007A70BD00BFA0
:10C2100000C05A4600409C453D0AC7403D0A27C021
:10C22000560EC9408FC2F53C2DB29D3D6666E63F75
:10C2300070B545689FED6C7A95ED025A95ED036AED
:10C24000F2EE085AF9EE087AE5EE257A00F6A443F4
:10C2500000F6A846F1EE006A2DED028B66EE266A26
:10C26000BFEE008AF0EE485AE6EE265A0446FDEE8E
:10C27000E77A85ED040A17EE902AC0F8882CC3ED02
:10C28000005A95ED036ADFED597AD0ED036AF6EEB8
:10C29000008AB4EEE86AF1EE10FAC8BFF0EE477A11
:10C2A000C6ED007A66EEE77A17EE900A0FF0A8FC6A
:10C2B00041EC100B0DF0F0FF51EC100B0FF0ECFF08
:10C2C00007EE100AF7EE007A77EEC77AB0EE007A42
:10C2D000C6ED007AD5ED047AA7EE878A04F69C4273
:10C2E00004F54A6382ED008A83ED008A95ED047AB5
:10C2F000B4EEE87AF1EE10FA03D5F1EE487AC3ED28
:10C30000007ADFED3B6A95ED056A9FED3A7AD4ED50
:10C31000037A9FED398AA6EE267A04F6984627EE30
:10C32000888A17EE100A0FF06BFC41EC100B0DF031
:10C33000B3FF51EC100B0FF0AFFF07EE900A27EEA2
:10C34000888AF7EE007A86ED008A95ED067A77EE18
:10C35000277A04F6D44377EE877AF5EE006AC3EDC8
:10C36000007A95ED067AB4EEE67AF1EE10FA09D588
:10C37000B0EE086AF6EE086AE7EE466A77EEE67A0D
:10C38000C3ED007A95ED077A9FED1C6ADFED1C7A0C
:10C39000DFED1C6A27EE067A04F6844383ED007A0B
:10C3A00095ED097AB6EE006A37EE467A04F6B843A0
:10C3B00083ED007A95ED0A7A67EE277A04F54C63EF
:10C3C00067EE877A04F6BC410022C1ED007ABDEC2D
:10C3D000028B1A60D5ED0B7A67EEA67A04F6C44498
:10C3E000C4ED007A70BD00BF00C05A4600409C45B5
:10C3F0003D0AC7403D0A27C0560EC9408FC2F53CD2
:10C400002DB29D3D6666E63F70B545689FED6C7A3E
:10C4100095ED025A95ED036AF2EE085AF9EE087AA4
:10C42000E5EE257A00F6A44300F6A846F1EE006A90
:10C430002DED028B66EE266ABFEE008AF0EE485ABA
:10C44000E6EE265A0446FDEEE77A85ED050A17EE7C
:10C45000902AC0F8882CC3ED005A95ED036ADFEDF1
:10C46000597AD0ED036AF6EE008AB4EEE86AF1EE8E
:10C4700010FAC8BFF0EE477AC6ED007A66EEE77AAA
:10C4800017EE900A0FF0BCFB41EC100B0DF004FF0F
:10C4900051EC100B0FF000FF07EE100AF7EE007AD8
:10C4A00077EEC77AB0EE007AC6ED007AD5ED047A61
:10C4B000A7EE878A04F69C4204F54A6382ED008A5F
:10C4C00083ED008A95ED047AB4EEE87AF1EE10FA85
:10C4D00003D5F1EE487AC3ED007ADFED3B6A95EDC6
:10C4E000056A9FED3A7AD4ED037A9FED398AA6EE7C
:10C4F000267A04F6984627EE888A17EE100A0FF07F
:10C500007FFB41EC100B0DF0C7FE51EC100B0FF050
:10C51000C3FE07EE900A27EE888AF7EE007A86EDD2
:10C52000008A95ED067A77EE277A04F6D44377EE03
:10C53000877AF5EE006AC3ED007A95ED067AB4EEDF
:10C54000E67AF1EE10FA09D5B0EE086AF6EE086A5E
:10C55000E7EE466A77EEE67AC3ED007A95ED077A64
:10C560009FED1C6ADFED1C7ADFED1C6A27EE067A70
:10C5700004F6844383ED007A95ED097AB6EE006AFD
:10C5800037EE467A04F6B84383ED007A95ED0A7AE1
:10C5900067EE277A04F54C6367EE877A04F6BC41B0
:10C5A0000022C1ED007ABDEC028B1A60D5ED0B7A4A
:10C5B00067EEA67A04F6C444C4ED007A70BD00BFED
:10C5C00000C05A4600409C453D0AC7403D0A27C06E
:10C5D000560EC9408FC2F53C2DB29D3D6666E63FC2
:10C5E00070B545689FED6C7A95ED025A95ED036A3A
:10C5F000F2EE085AF9EE087AE5EE257A00F6A44341
:10C6000000F6A846F1EE006A2DED028B66EE266A72
:10C61000BFEE008AF0EE485AE6EE265A0446FDEEDA
:10C62000E77A85ED060A17EE902AC0F8882CC3ED4C
:10C63000005A95ED036ADFED597AD0ED036AF6EE04
:10C64000008AB4EEE86AF1EE10FAC8BFF0EE477A5D
:10C65000C6ED007A66EEE77A17EE900A0FF0D0FA90
:10C6600041EC100B0DF018FE51EC100B0FF014FE06
:10C6700007EE100AF7EE007A77EEC77AB0EE007A8E
:10C68000C6ED007AD5ED047AA7EE878A04F69C42BF
:10C6900004F54A6382ED008A83ED008A95ED047A01
:10C6A000B4EEE87AF1EE10FA03D5F1EE487AC3ED74
:10C6B000007ADFED3B6A95ED056A9FED3A7AD4ED9D
:10C6C000037A9FED398AA6EE267A04F6984627EE7D
:10C6D000888A17EE100A0FF093FA41EC100B0DF058
:10C6E000DBFD51EC100B0FF0D7FD07EE900A27EEA3
:10C6F000888AF7EE007A86ED008A95ED067A77EE65
:10C70000277A04F6D44377EE877AF5EE006AC3ED14
:10C71000007A95ED067AB4EEE67AF1EE10FA09D5D4
:10C72000B0EE086AF6EE086AE7EE466A77EEE67A59
:10C73000C3ED007A95ED077A9FED1C6ADFED1C7A58
:10C74000DFED1C6A27EE067A04F6844383ED007A57
:10C7500095ED097AB6EE006A37EE467A04F6B843EC
:10C7600083ED007A95ED0A7A67EE277A04F54C633B
:10C7700067EE877A04F6BC410022C1ED007ABDEC79
:10C78000028B1A60D5ED0B7A67EEA67A04F6C444E4
:10C79000C4ED007A70BD00BF00C05A4600409C4501
:10C7A0003D0AC7403D0A27C0560EC9408FC2F53C1E
:10C7B0002DB29D3D6666E63F70B545689FED6C7A8B
:10C7C00095ED025A95ED036AF2EE085AF9EE087AF1
:10C7D000E5EE257A00F6A44300F6A846F1EE006ADD
:10C7E0002DED028B66EE266ABFEE008AF0EE485A07
:10C7F000E6EE265A0446FDEEE77A85ED070A17EEC7
:10C80000902AC0F8882CC3ED005A95ED036ADFED3D
:10C81000597AD0ED036AF6EE008AB4EEE86AF1EEDA
:10C8200010FAC8BFF0EE477AC6ED007A66EEE77AF6
:10C8300017EE900A0FF0E4F941EC100B0DF02CFD0F
:10C8400051EC100B0FF028FD07EE100AF7EE007AFE
:10C8500077EEC77AB0EE007AC6ED007AD5ED047AAD
:10C86000A7EE878A04F69C4204F54A6382ED008AAB
:10C8700083ED008A95ED047AB4EEE87AF1EE10FAD1
:10C8800003D5F1EE487AC3ED007ADFED3B6A95ED12
:10C89000056A9FED3A7AD4ED037A9FED398AA6EEC8
:10C8A000267A04F6984627EE888A17EE100A0FF0CB
:10C8B000A7F941EC100B0DF0EFFC51EC100B0FF051
:10C8C000EBFC07EE900A27EE888AF7EE007A86EDF9
:10C8D000008A95ED067A77EE277A04F6D44377EE50
:10C8E000877AF5EE006AC3ED007A95ED067AB4EE2C
:10C8F000E67AF1EE10FA09D5B0EE086AF6EE086AAB
:10C90000E7EE466A77EEE67AC3ED007A95ED077AB0
:10C910009FED1C6ADFED1C7ADFED1C6A27EE067ABC
:10C9200004F6844383ED007A95ED097AB6EE006A49
:10C9300037EE467A04F6B84383ED007A95ED0A7A2D
:10C9400067EE277A04F54C6367EE877A04F6BC41FC
:10C950000022C1ED007ABDEC028B1A60D5ED0B7A96
:10C9600067EEA67A04F6C444C4ED007A70BD00BF39
:10C9700000C05A4600409C453D0AC7403D0A27C0BA
:10C98000560EC9408FC2F53C2DB29D3D6666E63F0E
:10C990000174704770B545689FED6C7A95ED025A49
:10C9A00095ED036AF2EE085AF9EE087AE5EE257A7B
:10C9B00000F6A44300F6A846F1EE006A2DED028BC6
:10C9C00066EE266ABFEE008AF0EE485AE6EE265A78
:10C9D0000446FDEEE77A85ED090A17EE902AC0F8C5
:10C9E000882CC3ED005A95ED036ADFED597AD0ED3E
:10C9F000036AF6EE008AB4EEE86AF1EE10FAC8BFF8
:10CA0000F0EE477AC6ED007A66EEE77A17EE900A06
:10CA10000FF0F6F841EC100B0DF03EFC51EC100B52
:10CA20000FF03AFC07EE100AF7EE007A77EEC77ABD
:10CA3000B0EE007AC6ED007AD5ED047AA7EE878ACB
:10CA400004F69C4204F54A6382ED008A83ED008A75
:10CA500095ED047AB4EEE87AF1EE10FA03D5F1EE32
:10CA6000487AC3ED007ADFED3B6A95ED056A9FEDEC
:10CA70003A7AD4ED037A9FED398AA6EE267A04F647
:10CA8000984627EE888A17EE100A0FF0B9F841ECA5
:10CA9000100B0DF001FC51EC100B0FF0FDFB07EE3D
:10CAA000900A27EE888AF7EE007A86ED008A95EDE7
:10CAB000067A77EE277A04F6D44377EE877AF5EE96
:10CAC000006AC3ED007A95ED067AB4EEE67AF1EEEF
:10CAD00010FA09D5B0EE086AF6EE086AE7EE466A83
:10CAE00077EEE67AC3ED007A95ED077A9FED1C6A42
:10CAF000DFED1C7ADFED1C6A27EE067A04F684432C
:10CB000083ED007A95ED097AB6EE006A37EE467A43
:10CB100004F6B84383ED007A95ED0A7A67EE277A3A
:10CB200004F54C6367EE877A04F6BC410022C1ED40
:10CB3000007ABDEC028B1A60D5ED0B7A67EEA67A0F
:10CB400004F6C444C4ED007A70BD00BF00C05A466C
:10CB500000409C453D0AC7403D0A27C0560EC940CB
:10CB60008FC2F53C2DB29D3D6666E63F70B54568C7
:10CB70009FED6C7A95ED025A95ED036AF2EE085A34
:10CB8000F9EE087AE5EE257A00F6A44300F6A84609
:10CB9000F1EE006A2DED028B66EE266ABFEE008A8A
:10CBA000F0EE485AE6EE265A0446FDEEE77A85EDA9
:10CBB0000A0A17EE902AC0F8882CC3ED005A95EDAA
:10CBC000036ADFED597AD0ED036AF6EE008AB4EE1F
:10CBD000E86AF1EE10FAC8BFF0EE477AC6ED007AC7
:10CBE00066EEE77A17EE900A0FF00AF841EC100BA8
:10CBF0000DF052FB51EC100B0FF04EFB07EE100A3C
:10CC0000F7EE007A77EEC77AB0EE007AC6ED007ADA
:10CC1000D5ED047AA7EE878A04F69C4204F54A63B0
:10CC200082ED008A83ED008A95ED047AB4EEE87A0D
:10CC3000F1EE10FA03D5F1EE487AC3ED007ADFED9C
:10CC40003B6A95ED056A9FED3A7AD4ED037A9FED44
:10CC5000398AA6EE267A04F6984627EE888A17EED9
:10CC6000100A0EF0CDFF41EC100B0DF015FB51EC4E
:10CC7000100B0FF011FB07EE900A27EE888AF7EEF3
:10CC8000007A86ED008A95ED067A77EE277A04F62B
:10CC9000D44377EE877AF5EE006AC3ED007A95ED1E
:10CCA000067AB4EEE67AF1EE10FA09D5B0EE086A2B
:10CCB000F6EE086AE7EE466A77EEE67AC3ED007AAA
:10CCC00095ED077A9FED1C6ADFED1C7ADFED1C6A9B
:10CCD00027EE067A04F6844383ED007A95ED097A0F
:10CCE000B6EE006A37EE467A04F6B84383ED007A72
:10CCF00095ED0A7A67EE277A04F54C6367EE877A3A
:10CD000004F6BC410022C1ED007ABDEC028B1A6032
:10CD1000D5ED0B7A67EEA67A04F6C444C4ED007A2A
:10CD200070BD00BF00C05A4600409C453D0AC74048
:10CD30003D0A27C0560EC9408FC2F53C2DB29D3D1D
:10CD40006666E63F70B545689FED6C7A95ED025AD0
:10CD500095ED036AF2EE085AF9EE087AE5EE257AC7
:10CD600000F6A44300F6A846F1EE006A2DED028B12
:10CD700066EE266ABFEE008AF0EE485AE6EE265AC4
:10CD80000446FDEEE77A85ED0B0A17EE902AC0F80F
:10CD9000882CC3ED005A95ED036ADFED597AD0ED8A
:10CDA000036AF6EE008AB4EEE86AF1EE10FAC8BF44
:10CDB000F0EE477AC6ED007A66EEE77A17EE900A53
:10CDC0000EF01EFF41EC100B0DF066FA51EC100B4B
:10CDD0000FF062FA07EE100AF7EE007A77EEC77AE4
:10CDE000B0EE007AC6ED007AD5ED047AA7EE878A18
:10CDF00004F69C4204F54A6382ED008A83ED008AC2
:10CE000095ED047AB4EEE87AF1EE10FA03D5F1EE7E
:10CE1000487AC3ED007ADFED3B6A95ED056A9FED38
:10CE20003A7AD4ED037A9FED398AA6EE267A04F693
:10CE3000984627EE888A17EE100A0EF0E1FE41ECC4
:10CE4000100B0DF029FA51EC100B0FF025FA07EE3C
:10CE5000900A27EE888AF7EE007A86ED008A95ED33
:10CE6000067A77EE277A04F6D44377EE877AF5EEE2
:10CE7000006AC3ED007A95ED067AB4EEE67AF1EE3B
:10CE800010FA09D5B0EE086AF6EE086AE7EE466ACF
:10CE900077EEE67AC3ED007A95ED077A9FED1C6A8E
:10CEA000DFED1C7ADFED1C6A27EE067A04F6844378
:10CEB00083ED007A95ED097AB6EE006A37EE467A90
:10CEC00004F6B84383ED007A95ED0A7A67EE277A87
:10CED00004F54C6367EE877A04F6BC410022C1ED8D
:10CEE000007ABDEC028B1A60D5ED0B7A67EEA67A5C
:10CEF00004F6C444C4ED007A70BD00BF00C05A46B9
:10CF000000409C453D0AC7403D0A27C0560EC94017
:10CF10008FC2F53C2DB29D3D6666E63FD0F87C0C95
:10CF2000704700BF2DE9F04F2DED028B151E83B029
:10CF300006460F46D0F804A040F3D181D0F87C4CCF
:10CF4000017C8C4280F29A81342303FB040300228B
:10CF5000611CC0F87C1CC3F8DC22C3F8D822A7F1FE
:10CF60003C094EF64F4309FB09F2C4F6C46383FB48
:10CF70000231D317C3EBA10303EB430103EB81039E
:10CF8000D31A07EE903AF8EEE77AB1EE0A7A06F68F
:10CF9000BC4106F6B84377EEC77AD3ED006A91ED4F
:10CFA000007A3C2FE7EE276A09DD07EE102A06F526
:10CFB0004C63D3ED007AB8EEC77AE7EE876AD6F80D
:10CFC000883CB2691A44974240F30082726D1A4459
:10CFD000974240F32F82D6F890201A44974240F3AC
:10CFE0002682D6F8CC201A44974240F31D82D6F808
:10CFF00008211A44974240F3FB81D6F844211A4491
:10D00000974240F3F281D6F880211A44974240F3C8
:10D01000E981D6F8BC211A44974240F3E081D6F862
:10D02000F8211A44974240F3D781D6F834221A44A3
:10D03000974240F3CE81D6F8702213449F42CCBF72
:10D040004FF021084FF01E084FEA880B0BEB080346
:10D0500006EB8303D6ED037A5B699FEDE78A9FEDCC
:10D06000E76AFB1A07EE103AB8EEC77A27EE888A0D
:10D0700077EE267A67EE867A17EE900A0EF0C0FDFC
:10D0800041EC100B0DF008F9342303FB046351EC61
:10D09000100B00930FF000F907EE900A27EE888A34
:10D0A000009BBEEEC88A0022302DC3F8C02283ED5B
:10D0B000AF8A07DD502DD4BF08F1010808F102083E
:10D0C0004FEA880BD84406EB88084FF0340E06F67A
:10D0D000D442D8F82030D2ED008AD8F81C00D8F815
:10D0E00024100EFB0468013BC8F8C832C8F8C4021B
:10D0F000C8F8CC1218EE900A0EF082FD07EE905A96
:10D100009FEDBF7AF8EEE77ACDE9000167EE877A06
:10D11000B0EE088A17EE900A0EF072FD9DED001B2E
:10D1200041EC100B0DF03CF9F0EE007A51EC100BD5
:10D13000A8EEA78A0FF0B0F807EE900A28EE278A2B
:10D140003C2F88EDB48A00F32281DAED046A9FED6A
:10D15000AD7ADFEDAD5ADFEDAD7A9FEDAD6A96EDBC
:10D16000038A06F6C84393ED005A66EEA66A403D70
:10D17000A6EE857A06F6CC4306F6D84105EE107A7F
:10D18000F0EE476A07EE105AD3ED004AB8EEC77AC0
:10D19000B8EEC55AE4EE876A342303FB0463E5EE78
:10D1A000257AC3F8EC7206F68442F4EEE76AF1EEF3
:10D1B00010FA58BFF0EE667AF4EEC67AF1EE10FA85
:10D1C000D4BF67EEA77ADFED937A68EE277A0B2F4C
:10D1D000C3EDB87A6CDD6C2F40F33181D1ED007A6C
:10D1E00092ED007A9FED8C6A27EE877AF0EE675A0F
:10D1F000E7EE065A4EF685394FF0A858F0EE006A71
:10D20000B0EE657AC4F20109B0EE476A97EEA66AFD
:10D2100083EDBA7A83EDB96ADAED007A77EEA77A10
:10D2200017EE900A0EF0ECFC02460B4640464946CB
:10D230000EF086FB41EC100B0DF02EF8F1EE487A63
:10D2400053EC102B17EE900ACDE900230EF0D8FC1A
:10D25000DDE900230EF028FD41EC100B0DF01CF869
:10D26000342351EC100B03FB04660FF015F8C6F8DD
:10D27000D40203B0BDEC028BBDE8F08F002900F0B2
:10D28000DC800024DFED657A2346024692EDB47A15
:10D29000B4EEE77AF1EE10FA48BF1C4603F1010341
:10D2A00048BFF0EE477A994202F13402EED156E6D9
:10D2B000D1ED007A92ED007A9FED596A27EE877AD8
:10D2C000F0EE675AE7EE065A47F6E1294FF020588C
:10D2D000F0EE006AB0EE657AC3F6D47994E7027C8A
:10D2E000002AC6D0044600254FF0800B04E001352B
:10D2F000AA4204F13404BCDDD4F8EC329F42F6D1EA
:10D30000D6F88C3C1BB1C4F8ECB2327CEFE7F06885
:10D3100080F000400EF074FCCDE9000138460EF0BC
:10D320005DFC47F6E1234FF08042C3F684730EF0B4
:10D33000BBFC00230022C4F218030EF003FB9AED9D
:10D34000017AF1EE047A67EE277A804617EE900AAA
:10D3500089460EF055FC02460B46404649460EF003
:10D36000EFFA41EC100B0CF097FFDDE9000153ECF4
:10D37000102B0EF099FC41EC100B0CF08DFF51ECD2
:10D38000100B0EF089FFC4F8D402327CAFE7C7F16E
:10D390003C0307EE903A9FED237AF8EEE77A67EECA
:10D3A000877A17EE900A0EF02BFC41EC100B0CF074
:10D3B00073FF51EC100B0EF06FFFD8EDB47A07EE4F
:10D3C000100A67EE877AC8EDB47ABEE64FF000081F
:10D3D0003AE64FF01B0837E64FF0180834E64FF0F6
:10D3E000150831E64FF012082EE64FF00F082BE635
:10D3F0004FF00C0828E600BF0000FA4620986C3D6C
:10D400002497FF3B00004842CDCCCC3E00005C425C
:10D410000000524300442C47000040420000C64236
:10D42000000040C20AD7233C4FF009080CE64FF039
:10D43000060809E64FF0030806E60C468FE591ED75
:10D44000007AD2ED006A07EE909A67EE266AF8EE4F
:10D45000E77AF0EE475AE6EEA75A2B2FB0EE006AB5
:10D46000F0EE656AD7EE066AC3EDBA5AC3EDB96A43
:10D4700006DC47F6E1294FF02058C3F6D479CBE615
:10D4800038460EF0ABFB4BF651034FF06042C3F64B
:10D490009E730EF009FC00230022C3F6F0730EF019
:10D4A0004FFA80468946B7E670B50021064607F078
:10D4B000EDFEC0B1B6F91E40B6F92010031D00F50F
:10D4C000827533F9022B9442A8BF14469142B8BF2B
:10D4D00011469D42F5D80123F48331843377BDE8AA
:10D4E000704007F08BBE70BD002070470020704771
:10D4F000F8B549F22444037AC1F6FF74242908BF21
:10D50000C2805B0001250E462046C1F30721174665
:10D5100084F83B3084F85E5084F85D5003F05CFF83
:10D52000F1B2204603F058FFC7F30721204603F06D
:10D5300053FFF9B2204603F04FFF2946204604F07E
:10D5400023F8B0FA80F04009F8BD00BF2DE9F84398
:10D5500049F22444037AC1F6FF740125AB40294601
:10D560000746204684F83B3084F85E5084F85D50CE
:10D5700003F032FF0421204603F02EFF2046002155
:10D5800004F002F8B8B34FF0010846464FF0000926
:10D590003B7A012549F22440AB402946C1F6FF7091
:10D5A00084F83B3084F85E5084F85D5003F014FF3B
:10D5B00049F224400421C1F6FF7003F00DFF49F247
:10D5C00024404946C1F6FF7003F006FF49F22440AB
:10D5D0004146C1F6FF7003F0FFFE49F224402946A0
:10D5E000C1F6FF7003F0D0FF10B10020BDE8F88352
:10D5F000B0B2BDE8F8832B460222397A204604F007
:10D600004FF80128BFD994F8381094F83950A9423E
:10D6100018D263184A1CD2B2187E84F8382095427A
:10D620004FEA00230ED922440231107E84F83810CC
:10D63000184320F0010040F001064FEA16295FFA76
:10D6400086F8A5E74FF0FF08C1464FF0FF369FE789
:10D650002DE9F84349F22444037AC1F6FF74012509
:10D66000AB4029460746204684F83B3084F85E509C
:10D6700084F85D5003F0B0FE2421204603F0ACFE98
:10D680002046002103F080FFB8B34FF00108464662
:10D690004FF000093B7A012549F22440AB4029466E
:10D6A000C1F6FF7084F83B3084F85E5084F85D501A
:10D6B00003F092FE49F224402421C1F6FF7003F0EA
:10D6C0008BFE49F224404946C1F6FF7003F084FE08
:10D6D00049F224404146C1F6FF7003F07DFE49F255
:10D6E00024402946C1F6FF7003F04EFF10B1002020
:10D6F000BDE8F883B0B2BDE8F8832B460222397A40
:10D70000204603F0CDFF0128BFD994F8381094F8D3
:10D710003950A94218D263184A1CD2B2187E84F834
:10D72000382095424FEA00230ED922440231107E60
:10D7300084F83810184320F0010040F001064FEA49
:10D7400016295FFA86F8A5E74FF0FF08C1464FF0AB
:10D75000FF369FE7F8B549F22444037AC1F6FF7417
:10D760000126B340074601F003052046314684F800
:10D770003B3084F85E6084F85D6003F02DFE082184
:10D78000204603F029FE2046002103F0FDFE98B359
:10D7900000233A7A012649F22440B2403146C1F6CC
:10D7A000FF701D4384F83B2084F85E6084F85D6060
:10D7B00003F012FE49F224400821C1F6FF7003F085
:10D7C0000BFE49F22440C5F30721C1F6FF7003F0B8
:10D7D00003FE49F22440E9B2C1F6FF7003F0FCFDFC
:10D7E00049F224403146C1F6FF7003F0CDFE08B186
:10D7F0000020F8BDA8B2F8BD33460222397A20468F
:10D8000003F04EFF0128C3D994F8381094F839007A
:10D81000814212D263184A1CD2B21B7E84F838208F
:10D8200090424FEA032308D922440231127E84F841
:10D830003810134323F00303ABE76FF00303A8E7AB
:10D84000F8B549F22444027AC1F6FF745200012669
:10D8500000210546204684F83B2084F85E6084F869
:10D860005D6003F0B9FD0E21204603F0B5FD2046B2
:10D87000002103F089FE88B3002603272B7A49F2A2
:10D8800024405B0001250021C1F6FF7084F83B3085
:10D8900084F85E5084F85D5003F09EFD49F2244008
:10D8A0000E21C1F6FF7003F097FD49F2244039467E
:10D8B000C1F6FF7003F090FD49F224403146C1F6F5
:10D8C000FF7003F089FD49F224402946C1F6FF703C
:10D8D00003F05AFEB0FA80F04009F8BD3346022248
:10D8E000297A204603F0DCFE0128C5D994F83810C7
:10D8F00094F83900814216D263184A1CD2B21E7EB7
:10D9000084F8382090424FEA06230CD92244023191
:10D91000167E84F838101E4326F4407646F440768E
:10D92000370AF6B2AAE7FF263746A7E71F29F8B558
:10D93000064652D80C294DD840F60D55327A49F298
:10D940002444C1F6FF74520001270021204684F8C8
:10D950003B2084F85E7084F85D7003F03DFD2E215D
:10D96000204603F039FD2046002103F00DFEC8B328
:10D970000023327A49F22440520001260021C1F6E8
:10D98000FF701D4384F83B2084F85E6084F85D607E
:10D9900003F022FD49F224402E21C1F6FF7003F06E
:10D9A0001BFD49F22440C5F30721C1F6FF7003F0C7
:10D9B00013FD49F22440E9B2C1F6FF7003F00CFDFB
:10D9C00049F224403146C1F6FF7003F0DDFD38B165
:10D9D0000020F8BD41EA0125B0E741F61F75ADE72B
:10D9E000A8B2F8BD3B460222317A204603F058FE29
:10D9F0000128BDD994F8381094F83900814214D226
:10DA000063184A1CD2B21B7E84F8382090424FEA39
:10DA100003230AD922440231127E84F838101343BA
:10DA200023F4F85323F01F03A3E74EF2E003CFF6ED
:10DA3000FF739EE70023C4F2FE2307EE103A47F679
:10DA4000EE43C3F6FF6307EE903A70B5E0EE877AD7
:10DA50000023C4F2FE2307EE103AFCEEE77A47F605
:10DA6000EE4382B0C3F6FF63CDED017A07EE903A44
:10DA7000E0EE077A9DF80450027AFCEEE77A7F2DFB
:10DA8000CDED017A9DF804309CBFC5F17F052D02D4
:10DA900049F22444C1F6FF7494BF2DB200257F2BB8
:10DAA00094BFC3F17F0300235200012620460021CA
:10DAB0001D4384F83B2084F85E6084F85D6003F0C9
:10DAC0008BFC2046222103F087FCC5F3072120466A
:10DAD00003F082FCE9B2204603F07EFC314620468A
:10DAE00003F052FDB0FA80F0400902B070BD00BFF3
:10DAF0000023C4F27C2307EE103A47F6EE43C3F648
:10DB0000FF6307EE903AF0B5E0EE077A0023C4F227
:10DB1000FE2307EE103AFCEEE77A47F6EE4383B0B9
:10DB2000C3F6FF63CDED017A07EE903AE0EE877A17
:10DB30009DF804500646FCEEE77A3F2DCDED017AC4
:10DB40009DF80400337A98BFC5F13F0549F224449B
:10DB5000C1F6FF744FF0010794BF2D0200257F2806
:10DB600094BFC0F17F020022BB40394620461543D6
:10DB700084F83B3084F85E7084F85D7003F02CFC10
:10DB80000621204603F028FC2046002103F0FCFC7F
:10DB9000A8B30023327A49F224400126B24031462C
:10DBA000C1F6FF701D4384F83B2084F85E6084F862
:10DBB0005D6003F011FC49F224400621C1F6FF70BC
:10DBC00003F00AFC49F22440C5F30721C1F6FF70B7
:10DBD00003F002FC49F22440E9B2C1F6FF7003F001
:10DBE000FBFB49F224403146C1F6FF7003F0CCFC48
:10DBF00010B1002003B0F0BDA8B203B0F0BD3B46A9
:10DC00000222317A204603F04BFD0128C1D994F855
:10DC1000381094F83900814214D263184A1CD2B2E9
:10DC20001B7E84F8382090424FEA03230AD922440D
:10DC30000231127E84F83810134323F47D5323F00D
:10DC40003F03A7E74CF28003CFF6FF73A2E700BFC4
:10DC50002DE9F84F49F2244490F808E0C1F6FF742A
:10DC60000E46C1F307294FEA4E0E4FF0010A49460E
:10DC700007465FFA86F8204693461D4684F83BE047
:10DC800084F85EA084F85DA003F0A6FB4146204620
:10DC900003F0A2FB2046002103F076FCC0B3002570
:10DCA0003B7A242E4BEA050549F2244008BFFD804B
:10DCB0005B0001264946C1F6FF7084F83B3084F8CA
:10DCC0005E6084F85D6003F087FB49F224404146C2
:10DCD000C1F6FF7003F080FB49F22440C5F3072131
:10DCE000C1F6FF7003F078FB49F22440E9B2C1F6B7
:10DCF000FF7003F071FB49F224403146C1F6FF701A
:10DD000003F042FC00280CBF28460020BDE8F88F35
:10DD100053460222397A204603F0C2FC0128BED9BC
:10DD200094F8381094F83900814204D34FF0FF334F
:10DD300023EA0505B4E763184A1CD2B21B7E84F8B7
:10DD4000382090424FEA0323F0D922440231127E58
:10DD500084F838101343EBE72DE9F041437A2DEDB9
:10DD6000028B0646B0EE408AF0EE608A49F2244407
:10DD7000002B40F0E580C1F6FF740023C4F240237D
:10DD800007EE103A47F6EE43C3F6FF6307EE903A0C
:10DD90000023E8EE077ACCF23C2306EE903AF4EE4C
:10DDA000E67AF1EE10FA00F1C780F4EEC77AF1EEF0
:10DDB00010FAC8BF5F2740F35681337A49F22445F1
:10DDC0004FF00108C1F6FF7503FA08F341462846F3
:10DDD00084F83B3084F85E8084F85D8003F0FCFAC0
:10DDE0001621284603F0F8FA2846002103F0CCFB60
:10DDF000002800F0E8800023327A4FF0010849F251
:10DE0000244002FA08F24146C1F6FF7047EA0305D2
:10DE100084F83B2084F85E8084F85D8003F0DCFAAF
:10DE200049F224401621C1F6FF7003F0D5FA49F2F9
:10DE30002440C5F30721C1F6FF7003F0CDFA49F283
:10DE40002440E9B2C1F6FF7003F0C6FA49F224405B
:10DE50004146C1F6FF7003F097FB0023C4F2402354
:10DE600007EE103A47F6EE43C3F6FF6307EE903A2B
:10DE70000023E8EE877ACCF23C2306EE903AF4EEEB
:10DE8000E67AF1EE10FA59D4F4EEC77AF1EE10FA10
:10DE9000C8BF5F2740F3DE80337A49F224454FF054
:10DEA0000108C1F6FF7503FA08F34146284684F8D5
:10DEB0003B3084F85E8084F85D8003F08DFA1E218B
:10DEC000284603F089FA2846002103F05DFB00286C
:10DED00057D00025337A49F224400126B340314619
:10DEE000C1F6FF7084F83B3084F85E6084F85D60B2
:10DEF00003F072FA49F224401E21C1F6FF7003F0CC
:10DF00006BFA3D4349F22440C5F30721C1F6FF7087
:10DF100003F062FA49F22440E9B2C1F6FF7003F05F
:10DF20005BFABDEC028B49F224403146C1F6FF702A
:10DF3000BDE8F04103F028BB00273EE70027ABE730
:10DF4000037AC1F6FF740125AB402946204684F8C8
:10DF50003B3084F85E5084F85D5003F03DFA0821B0
:10DF6000204603F039FA2046002103F00DFB00287B
:10DF700051D0032302224FF484713046FFF768FE2C
:10DF8000FBE643460222317A284603F089FB01284A
:10DF90009FD995F8381095F83900814238D26B181E
:10DFA0004A1CD2B21B7E85F8382090424FEA0323E8
:10DFB0002ED92A440231127E85F8381042EA030530
:10DFC00025F07F0586E743460222317A284603F092
:10DFD00067FB01287FF60FAF95F8381095F83900E8
:10DFE000814212D26B184A1CD2B21B7E85F83820AF
:10DFF00090424FEA032308D92A440231127E85F861
:10E000003810134323F07F03F6E66FF07F03F3E647
:10E010006FF07F055EE72B460222317A204603F03F
:10E020003FFBA842A5D994F8383094F839108B42B8
:10E030009FD25A19D2B2914284F8382099D92244F9
:10E040000233127E84F8383002F00303022B3FF4CF
:10E0500094AE8EE79FED087A77EE877AFCEEE77A4A
:10E0600017EE907A18E79FED047A77EE877AFCEE48
:10E07000E77A17EE907AA0E600003C422DE9F04FD7
:10E080002DED028B49F22444027AC1F6FF7483B06D
:10E0900052000125002180462046B0EE408A84F8D7
:10E0A0003B2084F85E5084F85D5003F095F90E2112
:10E0B000204603F091F92046002103F065FA00287C
:10E0C00000F0D580B5EEC08AF1EE10FA56DCB5EE60
:10E0D000C08AF1EE10FA00F344810C26B1464FF0ED
:10E0E000FF0A98F8082049F22445C1F6FF7552004E
:10E0F0004FF0010B0021284684F83B2084F85EB0E5
:10E1000084F85DB003F068F90E21284603F064F945
:10E110002846002103F038FA0746002800F0F18075
:10E12000002798F8083049F224405B0001250021BF
:10E13000C1F6FF7084F83B3084F85E5084F85D507F
:10E1400003F04AF949F224400E21C1F6FF7003F0B2
:10E1500043F949F224403946C1F6FF7003F03CF917
:10E1600049F224403146C1F6FF7003F035F949F217
:10E1700024402946C1F6FF7003F006FA0023C4F2DA
:10E18000403307EE103A47F6EE43C3F6FF6307EE5F
:10E19000903AE8EE077A98F8082049F22447FCEE16
:10E1A000E77AC1F6FF77CDED017A9DF80450C02DD6
:10E1B00098BFC5F1FC054FEA42024FF001094FF04C
:10E1C0000001384694BF45EA052543F63C4584F8EE
:10E1D0003B2084F85E9084F85D9003F0FDF81021F8
:10E1E000384603F0F9F83846002103F0CDF9064629
:10E1F00000285BD0002698F8083049F224405B00E4
:10E2000001270021C1F6FF7084F83B3084F85E706E
:10E2100084F85D7003F0E0F849F224401021C1F663
:10E22000FF7003F0D9F8354349F22440C5F30721C4
:10E23000C1F6FF7003F0D0F849F22440E9B2C1F60C
:10E24000FF7003F0C9F849F224403946C1F6FF7067
:10E2500003F09AF928B1002003B0BDEC028BBDE8B1
:10E26000F08FA8B203B0BDEC028BBDE8F08F06467C
:10E270002B46022298F80810204603F011FA0128D4
:10E280007FF620AF94F8383094F839108B422AD3B7
:10E290000C23B5EEC08AF1EE10FA67DD002B3FF4D7
:10E2A0006DAF4FF0F30A4FF000091AE74B46022218
:10E2B00098F80810384603F0F3F901289AD997F82E
:10E2C000383097F83920934209D2591CC9B28A4292
:10E2D00087F8381003D9023387F838308BE70026E7
:10E2E000CFF6FF7687E75A1CD2B2914284F83820E5
:10E2F000CED922440233127E84F8383002F00C0367
:10E30000C7E75B46022298F80810284603F0C8F9D0
:10E3100058457FF606AF95F8382095F839008242C7
:10E320001CD2A91802EB0B03DBB2097E85F838304A
:10E3300098424FEA012111D92B44023293F818A0D8
:10E3400085F838204AEA010A2AF00C0A4AEA090943
:10E350005FFA89FA4FEA19275646E2E6FF27564642
:10E36000DFE60026B1464FF0F30ABAE60C2B3FF485
:10E3700005AFACE6F8B549F22444037AC1F6FF7460
:10E380000125AB4029460746204684F83B3084F8F7
:10E390005E5084F85D5003F01FF80021204603F022
:10E3A0001BF80021204603F017F82946204603F009
:10E3B00013F82946204603F0E7F808B10020F8BD1D
:10E3C0003B7A84F85E505B0006460146204684F89E
:10E3D0003B3084F85D5002F0FFFF0A21204602F036
:10E3E000FBFF3146204602F0F7FF7021204602F085
:10E3F000F3FF2946204603F0C7F8B0FA80F0400941
:10E40000F8BD00BFFFFFFFFFF3EE047A80EE277A2E
:10E410002DE9F04F98464FF4AA43C4F65713074628
:10E4200091460E4649F22444C1F6FF742DED068B49
:10E4300017EE100A83B008EE103AB0EE60AAF0EEC4
:10E44000418A0DF0DDFB9FED9E0B41EC110B0BF0B3
:10E45000A7FFCAEE087AB0EE409AF0EE609A012566
:10E4600008EA0508F1EE677A17EE900A0DF0C8FB8E
:10E470009FED930B41EC110B0BF092FFC8EE887AE5
:10E480005BEC10ABF1EE677A17EE900A0DF0B8FB7B
:10E490009FED8B0B41EC110B0BF082FF3B7A84F864
:10E4A0005E50AB40294620468DED000B84F83B3092
:10E4B00084F85D5002F090FF2621204602F08CFF88
:10E4C0000021204602F088FF45F61C234FF0204231
:10E4D000C3F6E47351EC190B0DF0E6FB00230022A8
:10E4E000C4F2E0030DF0E0FB0DF0B6FEC1B2204631
:10E4F00002F072FF2946204603F046F83B7A84F882
:10E500005E50AB402946204684F83B3084F85D508D
:10E5100002F062FF2821204602F05EFF0021204623
:10E5200002F05AFF002152465B460020C3F6F0710C
:10E530000DF006FA00230022C4F220130DF0B4FB04
:10E540000DF08AFEC1B2204602F046FF2946204661
:10E5500003F01AF83B7A84F85E50AB402946204617
:10E5600084F83B3084F85D5002F036FF2A212046C3
:10E5700002F032FF0021204602F02EFF9DED000B3D
:10E58000002153EC102B0020C3F6F0710DF0D8F9E8
:10E5900000230022C4F260130DF086FB0DF05CFE38
:10E5A000C1B2204602F018FF2946204602F0ECFFD7
:10E5B0003A7A84F85E504FEA481309F00308022EB5
:10E5C00043EA0828294602FA05F3204628BF022616
:10E5D00084F83B3084F85D5002F0FEFE2421204692
:10E5E00002F0FAFE2046002148EA063602F0CCFF8F
:10E5F00000283BD000233A7A012549F22440AA4062
:10E600002946C1F6FF701E4384F83B2084F85E5013
:10E6100084F85D5002F0E0FE49F224402421C1F666
:10E62000FF7002F0D9FE49F22440C6F30721C1F67B
:10E63000FF7002F0D1FE49F22440F1B2C1F6FF7042
:10E6400002F0CAFE49F224402946C1F6FF7002F0EA
:10E650009BFF28B1002003B0BDEC068BBDE8F08F16
:10E66000B0B203B0BDEC068BBDE8F08F2B460222A2
:10E67000397A204603F014F80128BBD994F83810F1
:10E6800094F83900814214D263184A1CD2B21B7E1E
:10E6900084F8382090424FEA03230AD922440231F9
:10E6A000127E84F83810134323F44C5323F02003D4
:10E6B000A1E74CF6DF43CFF6FF739CE7AFF3008092
:10E6C00000000000000024402DE9F041074649F217
:10E6D0002444C1F6FF74012520463D7102F090FEEE
:10E6E000052008F0D9FA3B7A84F85E50AB4000214F
:10E6F000204684F83B3084F85D5002F06DFE3021F6
:10E70000204602F069FE4021204602F065FE6021AD
:10E71000204602F061FE2946204602F035FF10B186
:10E720000020BDE8F0813B7A84F85E5006465B002D
:10E730000146204684F83B3084F85D5002F04CFEE0
:10E740002621204602F048FE3146204602F044FED3
:10E750006C21204602F040FE2946204602F014FFBC
:10E760003B7A84F85E505B003146204684F83B30AB
:10E7700084F85D5002F030FE2821204602F02CFE85
:10E780002946204602F028FEF221204602F024FE0F
:10E790002946204602F0F8FE3B7A84F85E505B0082
:10E7A0003146204684F83B3084F85D5002F014FE78
:10E7B0002C21204602F010FE0F21204602F00CFE14
:10E7C0002221204602F008FE2946204602F0DCFE07
:10E7D0003B7A84F85E505B003146204684F83B303B
:10E7E00084F85D5002F0F8FD3C21204602F0F4FD73
:10E7F0004421204602F0F0FD4621204602F0ECFDC7
:10E800002946204602F0C0FE3B7A40F23712FA80D9
:10E810005B003146204684F83B3084F85E5084F833
:10E820005D5002F0D9FD2421204602F0D5FD294695
:10E83000204602F0D1FD3721204602F0CDFD2946C9
:10E84000204602F0A1FE3B7A84F85E505B00314620
:10E85000204684F83B3084F85D5002F0BDFD302145
:10E86000204602F0B9FD4021204602F0B5FDFF210F
:10E87000204602F0B1FD2946204602F085FE3B7A93
:10E8800084F85E505B003146204684F83B3084F8C3
:10E890005D5002F0A1FD0221204602F09DFD3146AF
:10E8A000204602F099FD7321204602F095FD29468D
:10E8B000204602F069FE4FF4C87008F0EDF93B7A8B
:10E8C00084F85E505B003146204684F83B3084F883
:10E8D0005D5002F081FD2E21204602F07DFD1D21BC
:10E8E000204602F079FD1D21204602F075FD2946E3
:10E8F000204602F049FE3B7A84F85E505B003146C8
:10E90000204684F83B3084F85D5002F065FD042118
:10E91000204602F061FD3146204602F05DFD0421F3
:10E92000204602F059FD2946204602F02DFE3B7A92
:10E9300084F85E505B003146204684F83B3084F812
:10E940005D5002F049FD0621204602F045FD2946B2
:10E95000204602F041FD3021204602F03DFD2946CF
:10E96000204602F011FE3B7A84F85E505B0031468F
:10E97000204684F83B3084F85D5002F02DFD0A21DA
:10E98000204602F029FD3146204602F025FD1021E7
:10E99000204602F021FD2946204602F0F5FD3B7A93
:10E9A00084F85E505B003146204684F83B3084F8A2
:10E9B0005D5002F011FD0E21204602F00DFD3146A2
:10E9C000204602F009FD3146204602F005FD2946A9
:10E9D000204602F0D9FD3B7A84F85E505B00314658
:10E9E000204684F83B3084F85D5002F0F5FC10219D
:10E9F000204602F0F1FC3C21204602F0EDFC3C21D7
:10EA0000204602F0E9FC2946204602F0BDFD3B7A93
:10EA100084F85E505B003146204684F83B3084F831
:10EA20005D5002F0D9FC2221204602F0D5FC7F2166
:10EA3000204602F0D1FC7F21204602F0CDFC294681
:10EA4000204602F0A1FD3B7A4FF036085B00A7F8A4
:10EA500006803146204684F83B3084F85E5084F8C6
:10EA60005D5002F0B9FC2421204602F0B5FC31468D
:10EA7000204602F0B1FC4146204602F0ADFC29469A
:10EA8000204602F081FD7D722846BDE8F08100BF7E
:10EA90002DE9F8430023C4F2013307EE103A47F69C
:10EAA000EE43C3F6FF6307EE903AE0EE077A0646C0
:10EAB000FCEEE77A17EE904A002C71D0802C39D901
:10EAC000337900242746002B3ED149F22445C1F674
:10EAD000FF75337A49F224405B0001260021C1F61C
:10EAE000FF7085F83B3085F85E6085F85D6002F068
:10EAF00073FC49F224402221C1F6FF7002F06CFC45
:10EB000049F224403946C1F6FF7002F065FC49F233
:10EB100024402146C1F6FF7002F05EFC49F2244019
:10EB20003146C1F6FF7002F02FFDB0FA80F04009C7
:10EB3000BDE8F883C4F18004337944EA0424C4F3C3
:10EB40000727E4B2002BC0D0B6F80680337A49F22A
:10EB50002445C1F6FF7528F0100800215B003171D3
:10EB6000A6F806804FF00109284685F83B3085F865
:10EB70005E9085F85D9002F02FFC2846242102F07B
:10EB80002BFC4FEA1821284602F026FC08F0EF0182
:10EB9000284602F021FC4946284602F0F5FC98E799
:10EBA000037A49F22445C1F6FF75012717EE901A42
:10EBB000BB400771284685F83B3085F85E7085F8C4
:10EBC0005D7002F009FC2846222102F005FC28466F
:10EBD0007F2102F001FC28467F2102F0FDFB39462F
:10EBE000284602F0D1FCB6F80680337A48F01008C7
:10EBF0001FFA88F8BB40A6F806802146284685F80B
:10EC00003B3085F85E7085F85D7002F0E5FB2846C4
:10EC1000242102F0E1FB4FEA1821284602F0DCFB38
:10EC20005FFA88F1284602F0D7FB3946284602F001
:10EC3000ABFCB0FA80F04009BDE8F883F8B50646B1
:10EC40000D4619B1012948D00020F8BD037A49F2D8
:10EC50002444C1F6FF745B000127204684F83B3052
:10EC600084F85E7084F85D7002F0B6FB20212046C7
:10EC700002F0B2FB2946204602F0AEFB55212046A9
:10EC800002F0AAFB3946204602F07EFC0028DBD1C8
:10EC9000F588337A45F00405ADB25B00F580014696
:10ECA000204684F83B3084F85E7084F85D7002F092
:10ECB00093FB2421204602F08FFB290A204602F014
:10ECC0008BFBE9B2204602F087FB3946204602F072
:10ECD0005BFCB0FA80F04009F8BD037A49F22444A5
:10ECE000C1F6FF745B000021204684F83B3084F8B5
:10ECF0005E5084F85D5002F06FFB2A21204602F03E
:10ED00006BFB2946204602F067FB7321204602F088
:10ED100063FB2946204602F037FC0746002893D1C2
:10ED2000337A84F85E505B000146204684F83B301D
:10ED300084F85D5002F050FB2021204602F04CFB8D
:10ED40003946204602F048FB8821204602F044FB69
:10ED50002946204602F018FC00287FF475AFF7889A
:10ED6000337A27F004075B00F7800146204684F8D9
:10ED70003B3084F85E5084F85D5002F02DFB242176
:10ED8000204602F029FB390A204602F025FB07F055
:10ED9000FB01204602F020FB2946204602F0F4FB4E
:10EDA000B0FA80F04009F8BD2DE9F04F9BB0044661
:10EDB00006F0CCF91690002800F05F820021204672
:10EDC00006F064FA1790002800F0608240F2B85311
:10EDD000C0F20F03199345F24C6945F24E6734F9BE
:10EDE0000930049345F25266E35F099345F254609B
:10EDF000A35F089345F25661235E189345F258626B
:10EE0000635E059345F25A6AA35E079334F90A30AC
:10EE1000069304F5AC431A4604F5C5491E46CDF8E1
:10EE2000449002F13C093E320B9206F140020C92F2
:10EE300006F142020D9206F144020E9206F14602DC
:10EE40000F9206F14802119B109232464A32039209
:10EE50001A46183211921A461A3245F25065129229
:10EE600045F25E681A4645F25C6C45F2606E1C32F3
:10EE70001E3334F905B0139234F9088034F90CC00C
:10EE800034F90EE0CDF808901493179B18989A1C4B
:10EE90000192169A03F5817302321593019B0A922F
:10EEA0004FF0000A5D4633F9022F019302EB021284
:10EEB00002EB0222520022F34F42029B04991E8869
:10EEC00004EB460701FB0CF9B7F91C3003FB08996A
:10EED00029F3CF390FFA89F1049112B201FB0EF92F
:10EEE00029F3CF39914409F30F090136A7F81C9093
:10EEF0000299B6B240F25B47BE4294BF0E80A1F8C1
:10EF000000A00B99099F0E8804EB460907FB0CFB38
:10EF1000B9F9D4783B4407FB08BB2BF3CF3B0FFA7E
:10EF20008BF7099707FB0EF727F3CF37174407F343
:10EF30000F070136A9F8D4780B99B6B240F2A3476F
:10EF4000BE4294BF0E80A1F800A00C990E8804EB7D
:10EF5000460707F590571C37B7F9009005FB0CF5ED
:10EF60004B4409FB085525F3CF352DB205FB0EF9AF
:10EF700029F3CF39914409F30F090136A7F800901E
:10EF8000B6B240F2FC47BE4294BF0E80A1F800A08A
:10EF90000D990E88089904EB460707F5E0571637D8
:10EFA000B7F9009001FB0CFB4B4409FB08BB2BF3AA
:10EFB000CF3B0FFA8BF9CDF8209009FB0EF929F31E
:10EFC000CF39914409F30F090136A7F800900D9944
:10EFD000B6B240F24B57BE4294BF0E80A1F800A0DB
:10EFE0000E990E8804EB460707F51A572E37B7F926
:10EFF000009000FB0CF04B4409FB080020F3CF30DD
:10F0000000B200FB0EF929F3CF39914409F30F093F
:10F010000136A7F80090B6B240F28D57BE4294BFB9
:10F020000E80A1F800A00F990E88059904EB460701
:10F0300007F547570A37B7F9009001FB0CFB4B4423
:10F0400009FB08BB2BF3CF3B0FFA8BF9CDF81490DB
:10F0500009FB0EF929F3CF39914409F30F09013661
:10F06000A7F800900F99B6B240F2D257BE4294BFB3
:10F070000E80A1F800A010990E88079904EB4607AE
:10F0800007F575573037B7F9009001FB0CFB4B447F
:10F0900009FB08BB2BF3CF3B0FFA8BF9CDF81C9083
:10F0A00009FB0EF929F3CF39914409F30F09013611
:10F0B000A7F800901099B6B240F21467BE4294BF10
:10F0C0000E80A1F800A003990E88069904EB46076C
:10F0D00007F593471A37B7F9009001FB0CF14B4441
:10F0E00009FB081121F3CF3109B2069101FB0EF99A
:10F0F00029F3CF394A4402F30F020136B6B2B6F50E
:10F10000CA6F3A808ABF039A0399A2F800A047F613
:10F11000E12298BF0E8002FB03F323F34F431199C2
:10F120000E8804EB460707F5AC470FFA83F9B7F9E9
:10F13000622003EB6203A7F86230C9EB020222F3FC
:10F140004F020136B6B2B6F50B7F34BF0E80A1F880
:10F1500000A012990E8804EB460707F5B5470FFA91
:10F1600082F9B7F93A3002EB63027A87C9EB0303FD
:10F1700023F34F030136B6B2B6F5DC7F94BF0E80A1
:10F18000A1F800A013990E8804EB460707F5BC47C9
:10F190000FFA83F9B7F92C2003EB6203BB85C9EBA7
:10F1A000020222F34F020136B6B2B6F5AA7F94BF2F
:10F1B0000E80A1F800A014990E8804EB460707F50D
:10F1C000C1470FFA82F9B7F9563002EB6302A7F88C
:10F1D0005620C9EB030323F34F030136B6B21BB22B
:10F1E000E02EC3EB031394BF0E80A1F800A05B00D8
:10F1F00003F30F030A9A22F8023F019B0A92159A21
:10F2000093427FF450AE0499002213461E4661F3E8
:10F210000F02079965F30F03354661F30F0509994E
:10F2200061F31F42089961F31F43059960F30F06CC
:10F2300061F31F46069945F2546E45F2586C45F24B
:10F24000506045F24C6761F31F45E251235044F88A
:10F250000E60204644F80C50169C0022214605F012
:10F26000FBFF204605F0CAFF1798199A90420AD072
:10F270001BB0BDE8F04F05F0C1BF0146204606F0C7
:10F2800005F80028F4D11BB0BDE8F08F40F2B85368
:10F29000C0F20F03199317939DE500BFF8B540F234
:10F2A0001C530446C0F2020303600021012004F154
:10F2B00018020B46607222612172E16000E022694F
:10F2C00042F82310627A01339A42F8DC40F2885304
:10F2D000C2F201031A680AB9B9E01A465369002B51
:10F2E000FBD15461204640F2C4630025C0F20F03F5
:10F2F0006561A580E580A572294640F81C3B40F673
:10F30000B8020DF001FD294640F6481204F6D4007B
:10F310000DF0FAFC04F59050294640F6FA121C3024
:10F320000DF0F2FC04F5E050294640F69822163024
:10F330000DF0EAFC04F51A50294640F61C322E3036
:10F340000DF0E2FC04F54750294640F6A6320A309B
:10F350000DF0DAFC04F57550294640F62A423030AB
:10F360000DF0D2FC04F59340294640F6A2421A3033
:10F370000DF0CAFC45F23C6345F23E6045F2406741
:10F3800045F2426145F24462E55245F24666255235
:10F3900045F2486345F24A60E553655245F24C67D1
:10F3A000A55245F24E6145F25062A553E55245F231
:10F3B0005266255245F2546345F25660E553655254
:10F3C00045F25867A55245F25A6145F25C62A55371
:10F3D000E55245F25E66255245F2606341F69910AA
:10F3E000E553655246F26767A05246F6843204F54B
:10F3F000AC402946A7536230E2524FF48B620DF0C5
:10F4000083FC04F5B540294640F272323A300DF0E3
:10F410007BFC04F5BC40294640F2AA222C300DF0BA
:10F4200073FC04F5C14029464FF4E17256300DF0EB
:10F430006BFC46F2982046F29A2146F29C2246F254
:10F440009E23255265522046A552E552F8BD1C6008
:10F4500048E700BF10B5044606F03EF9204610BD4F
:10F4600049F2A0224FF255414FF25820C1F6FF72E7
:10F47000C0F20001C2F200000DF0D2B838B549F276
:10F48000A0254FF25544C1F6FF75C0F200044FF2BB
:10F4900060202A462146C2F200000DF0C1F84FF26A
:10F4A00068202A462146C2F20000BDE838400DF02F
:10F4B000B7B800BF49F2A0224FF255414FF2702079
:10F4C000C1F6FF72C0F20001C2F200000DF0A8B850
:10F4D00049F2A0224FF255414FF27820C1F6FF7257
:10F4E000C0F20001C2F200000DF09AB849F2A02269
:10F4F0004FF255414FF28020C1F6FF72C0F2000179
:10F50000C2F200000DF08CB849F2A0224FF2554132
:10F510004FF28820C1F6FF72C0F20001C2F2000073
:10F520000DF07EB82DE9F04F00F5807EB1E8A00A1D
:10F53000B2E84015C5EA0643C6EA2544C7EA0845CD
:10F54000C8EA2746C9EA0A47CAEA2948CBEA0C4969
:10F55000CCEA2B4AA0E8F8078645E7D1BDE8F04F92
:10F5600070474FF000022DE9F00F00F5807C00BFDE
:10F57000B1E8A00AC5EA0203C2EA2544C7EA0205C7
:10F58000C2EA2746C9EA0207C2EA2948CBEA0209C9
:10F59000C2EA2B4AA0E8F8078445E9D1BDE8F00F9C
:10F5A00070474FF000022DE9F00F00F5807C00BF9E
:10F5B000B1E8A00AC2EA0543C2EA0504C2EA074567
:10F5C000C2EA0706C2EA0947C2EA0908C2EA0B49C9
:10F5D000C2EA0B0AA0E8F8078445E9D1BDE8F00FBC
:10F5E00070472DE9F00F089C00F5007B51F8045B93
:10F5F00053F8046BC5EA0647C6EA254952F8045B8E
:10F6000054F8046BC5EA0648C6EA254AA0E8800714
:10F610008345EBD1BDE8F00F704700BF2DE9F843FB
:10F620004FF00008064600F11805474641463046AF
:10F63000002F4FD005F02AFEF0B12C68B4F5803FC2
:10F6400007F1040100F1040E07F5827C27D05EF873
:10F65000042B34FB02F334FB12F903F30F0209F31A
:10F660000F03C2EA03430A6893FA12F341F8043B1A
:10F670008C45ECD805F0C2FD08F10108B8F1040F83
:10F6800005F10405D2D1002F40D030463946002282
:10F6900005F0E2FD3846BDE8F84305F0AFBD07F1DF
:10F6A0000C0100F10C0451F8083C54F8082C93FAB2
:10F6B00012F341F8083C54F8042C51F8043C93FA36
:10F6C00012F38C4541F8043C04F1080401F10801EF
:10F6D000E9D8CFE705F0E6FD07460028CCD028683A
:10F6E000B0F5803FC8D0391D07F582740B6830FB38
:10F6F00003F230FB13F302F30F0203F30F03C2EA2A
:10F70000034341F8043B8C42F0D8B5E7BDE8F883E9
:10F7100070B584692CB3B4F5803F06464FF0000104
:10F7200025D005F0BFFD054600B3011D00F5827030
:10F730000B6834FB03F234FB13F302F30F0203F301
:10F740000F03C2EA034341F8043B8842F0D8304635
:10F750000022294605F080FD2846BDE8704005F0EE
:10F760004DBD214605F092FD0028F6D170BD05F093
:10F770008DFD04460028F9D030462146002205F0D0
:10F780006BFD2046BDE8704005F038BD49F2A0226F
:10F790004FF255414FF29020C1F6FF72C0F20001C6
:10F7A000C2F200000CF03CBF49F2A0224FF25541DA
:10F7B0004FF29820C1F6FF72C0F20001C2F20000C1
:10F7C0000CF02EBF49F2A0224FF255414FF2A0207B
:10F7D000C1F6FF72C0F20001C2F200000CF020BFBF
:10F7E0002DE9F84F4FF2AC23C2F2000348F21F029A
:10F7F00019681B79096848F20050C1F6FF70C4F21D
:10F8000000028142137035D24FF2C423C2F20003CA
:10F810001B7893BB4FF2BC29C2F200094FF2B42807
:10F820004FF2A8254FF2B826C2F20008C2F2000536
:10F83000C2F20006D9F800A0D8F800B02C883788AA
:10F84000BAF1000F45D0BBF1000F3AD00BF1040222
:10F850000AF1040102EB470201EB4401FFF762FEEB
:10F86000403740347F2C1ED82C807F2F0CD8378017
:10F87000BDE8F88FA0F58070CCE74EF20823CEF2F9
:10F88000000301221A60C5E700245846348005F0C1
:10F89000B5FC4FF2C023C2F200031A68C8F800207A
:10F8A0001C60BDE8F88F002450462C8005F0A6FCB3
:10F8B0004FF2C823C2F200031A68C9F800201C6086
:10F8C000D3E70AF1040101EB4401FFF74AFE40349B
:10F8D000C8E7BBF1000F07D00BF1040101EB4701B2
:10F8E000FFF75FFE4037BDE74FF4807259460DF0D9
:10F8F0000BFAB7E7F8B50021054605F0C7FCC8B11B
:10F9000072B64FF2BC23C2F200031968002938D046
:10F910004FF2C822C2F20002166866B34FF2A82462
:10F92000C2F2000400271E601060278062B60846FD
:10F9300005F064FC2846012105F0A8FCD0B172B6A0
:10F940004FF2B423C2F200031C6814B34FF2C0227A
:10F95000C2F2000215688DB14FF2B821C2F2000167
:10F9600000261D6010600E8062B62046BDE8F8409B
:10F9700005F044BCF8BD106062B6DBE7106062B60B
:10F98000F8BD4FF2A822C2F200021860118062B6E0
:10F99000D0E74FF2B822C2F200021860148062B6BB
:10F9A000F8BD00BF4FF2AC20F8B5C2F20000012153
:10F9B00005F0ECFD48F23C03C4F204034FF2BC2412
:10F9C00019684FF2B420C2F20004C2F2000048F2FB
:10F9D00040020025C4F2040241F4004125600560A4
:10F9E0001960116841F0020111601A684FF470410A
:10F9F00042F00202C4F202011A600B68AB427DDBE6
:10FA00004FF28003C4F202031B68AB4276DB4FF473
:10FA10007142C4F202024FF0804313601368002B5E
:10FA2000FCDB4FF20410C4F202004FF26003C4F298
:10FA300002034FF2FE054FF2040E0560C4F2020EFF
:10FA400000251D604FF2080101234FF20C07CEF88C
:10FA50000030C4F20201C4F202079E46C0F2007EEA
:10FA60004FF4803C4FF21002C1F800E0C4F20202F1
:10FA7000C7F800C041F61B7763F31F474FF2140627
:10FA80004FF2E0044FF284001760C4F20206C4F2A1
:10FA90000204C4F202004FF288014FF4F852C4F29B
:10FAA0000201C1F61F7241F61B77326063F31F47F4
:10FAB00025600360C4F200730B604FF28C0E4FF2AE
:10FAC00090064FF294054BF208044BF20C004BF2F7
:10FAD0001801C4F2020EC4F20206C4F20205C4F216
:10FAE0000404C4F20400C4F204014FF4C063CEF86D
:10FAF00000C037602A60236003600B604FF2AC24C3
:10FB0000C2F200044BF204002368C4F2040048F27D
:10FB1000004202214FF4C065C1F6FF7205601A6011
:10FB200099802279996002F180424FF2220102F518
:10FB30000432C4F2020140F201164FF47E4519610D
:10FB4000DE8000214FF48070CFF6FF7506278D26EA
:10FB5000D882DD609982D88399619F831170167075
:10FB600005F0B0FC22794FF2C4215311C2F200011A
:10FB700048F21B06C4F200069B00087003F16043C4
:10FB800002F01F004FF4704548F20064012132700A
:10FB9000C4F2020502F11007814003F56143C1F68A
:10FBA000FF7401204FF2E172C9F200004FF080763D
:10FBB000C0F200022E60286044F827201960F8BDCA
:10FBC00049F2A0224FF255414FF2AC20C1F6FF722C
:10FBD000C0F20001C2F200000CF022BD49F2A022E6
:10FBE0004FF255414FF2CC20C1F6FF72C0F2000136
:10FBF000C2F200000CF014BD49F2A0224FF25541B0
:10FC00004FF2D420C1F6FF72C0F20001C2F2000030
:10FC10000CF006BD49F2A0224FF255414FF2DC2014
:10FC2000C1F6FF72C0F20001C2F200000CF0F8BC95
:10FC300049F2A0224FF255414FF2E420C1F6FF7283
:10FC4000C0F20001C2F200000CF0EABC49F2A022AE
:10FC50004FF255414FF2EC20C1F6FF72C0F20001A5
:10FC6000C2F200000CF0DCBC90F89D3090F89C20B3
:10FC7000DBB2934215D001331F2B84BF00210B460A
:10FC800010B598BFD9B20633002250F8234080F84F
:10FC90009D10214605F0E0FA2046BDE8104005F031
:10FCA000ADBA7047D0F898300BB10120704710B54D
:10FCB000044605F04BFAC4F89800003018BF012044
:10FCC00010BD00BF10B50446D0F8980018B104303C
:10FCD00010BD09F0C9FC05F039FAC4F898000028F5
:10FCE000F7D0043010BD00BFD0F89810B1B190F833
:10FCF0009C2001321F2A10B4CABF0024D4B222466D
:10FD000090F89D309342FBD00632002340F8221039
:10FD100080F89C405DF8044BC0F89830704700BFF5
:10FD200010B4047F4160022CC26003D05DF8044B24
:10FD300005F0F0BC83685DF8044B1847F0B449F255
:10FD40007433C1F6FF7348F21F02996BC4F20002CC
:10FD500008791070586B48F21C02C4F20002047952
:10FD60001470097911701A6B002A4FD05968C9684C
:10FD70008A4247D80168CC8B240402F1FF3073D447
:10FD8000C0F30E00C883C88B80B2C882996B096823
:10FD9000C88B000460D4C2F30E00C883C88B002453
:10FDA00080B212F1FF32C88218BF01221C63596B66
:10FDB000086849F274310568C1F6FF7101F12C043D
:10FDC000A54241D00968CC6814F0804F04680568EA
:10FDD00015BF248824780235013544F000440560BD
:10FDE0004C63996B48F21B03C4F200030979197044
:10FDF00049F27431C1F6FF7112B14A6B12791A706F
:10FE0000F0BC7047521A1A630122D0E71968D86B08
:10FE10000A630024CFF60F74CC620468CD682668AC
:10FE20004FF62154C0F2000425F080450327A64276
:10FE3000CD6083F82D701FD1037F4260022BC2601A
:10FE40001ED0F0BC05F066BC086891F82C10C468A0
:10FE500041F000414163C4E7CC8BC2F3080004F4D5
:10FE60007E442043C88399E7CC8BC0F3080004F498
:10FE70007E442043C88386E733461146F0BC1847CA
:10FE80008368F0BC184700BF00207047704700BF70
:10FE90004FF2F423C2F20003022240F29471C0F246
:10FEA0000F015A600022D9629A7083F8242083F8E7
:10FEB000302083F83220704741F23801C4F20B0140
:10FEC00041F230020B6823F0805323F00A030B60E9
:10FED000C4F20B0213689907FCD541F22C03C4F25B
:10FEE0000B031A68920703D51A6822F002021A60FF
:10FEF00041F22803C4F20B034FF24832196821F093
:10FF0000080119601968C2F2000241F008010120DD
:10FF100019601060704700BF830769D1F0B54FF2D8
:10FF20004C34C2F2000423780BB10320F0BD41F23F
:10FF30002402C4F20B0215461368DE07FCD42B68BA
:10FF40009B07F9D4637803B9490241F23003C4F244
:10FF50000B0341F234021C681C60C4F20B0241F234
:10FF60003804136823F4081323F0310343F080535B
:10FF700041F22C05C4F20B0543F00A03C4F20B0452
:10FF8000136023682E684FF2483246F002064FF4A1
:10FF9000805EC2F200022E60C4F20B0E002541F218
:10FFA00008071560C4F20B0741F2040641F20C0584
:10FFB000CEF8000043F08053C4F20B06C4F20B05E8
:10FFC0001120396043F00A03C1F222104FF481314D
:10FFD0003160236028601368002BFCD041F23003AD
:10FFE000C4F20B0300201A6802F003021A60F0BD8D
:10FFF0004FF0FF30704700BF830740F0AD802DE920
:020000021000EC
:10000000F0414FF24C35C2F200052B7813B10320BA
:10001000BDE8F08141F22402C4F20B0214461368D9
:10002000DF07FCD423689E07F9D46B7803B9490233
:1000300041F23003C4F20B0341F234021C681C602D
:10004000C4F20B0241F23804136823F4081323F0BE
:10005000310343F0805341F22C06C4F20B0643F007
:100060000A03C4F20B041360236837684FF2483266
:1000700047F002074FF4805E3760C2F20002C4F21C
:100080000B0E41F20807C4F20B0700261660CEF8EB
:10009000000041F2040641F20C00396043F0805345
:1000A000C4F20B06C4F20B00012143F00A034FF423
:1000B0008137C1F622013760236001601368002B8D
:1000C000FCD041F23003C4F20B0341F22402196860
:1000D00001F003011960C4F20B0213685907FCD444
:1000E00041F2240141F23002C4F20B01C4F20B02CE
:1000F00041F2340741F2080841F20C0C41F21006BB
:100100008E461446C4F20B07C4F20B08C4F20B0C63
:10011000C4F20B060B68DB07FCD4DEF8003098074E
:10012000F8D43B6843F001033B6013681360002080
:100130006B68C8F80030C0F60250CCF800001368B5
:10014000DB07FCD5236803F001032360306810F45B
:100150000070DFD1BDE8F0814FF0FF30704700BF85
:10016000F0B540F23466C2F2010683B03368019301
:100170004FF44044C4F20204019F0546A4464FF0E8
:10018000004EFF20236843F480632360C4F82CE012
:100190006063E36A002BFCDADCF83830DBB2FF2B5B
:1001A00006D033680093009BDB1BB3F5967FE9D341
:1001B0004FF44043C4F202034FF00046186841F088
:1001C000400440F480601860DE6218465C63C36AD5
:1001D000002BFCDA4FF44044C4F2020418204FF024
:1001E0000047266822FA00F346F48066DBB22660F8
:1001F000E7626363E36A002BFCDA083810F1080F4A
:10020000EFD1002932D008290CBF8721FF214FF4FC
:100210004043C4F202034FF000401A6842F4806287
:100220001A60D8621A465963D36A002BFCDA4FF47D
:100230004042C4F20202164600274FF00044FF215C
:10024000136843F480631360D4625163D36A002B54
:10025000FCDAB36BD8B21B06687001D403B0F0BDF2
:100260000137B7F5807FEBD103B0F0BD9521CEE724
:100270002DE9F0414FF260358378C2F20005032B7F
:100280002B780F4682B00446164618BF4F02002B4B
:100290006AD00021207806F067FC3A4611212046FA
:1002A000FFF75EFF60BB40F23460C2F201004FF422
:1002B000404103680093C4F20201DDF800808C46DF
:1002C0004FF0004EFF270B6843F480630B60C1F8CA
:1002D0002CE04F63CA6A4FF44043002AC4F2020381
:1002E000F8DADCF83820D2B2FF2A627040F0918050
:1002F00003680193019BC8EB0303B3F5967FE2D932
:100300002078012106F030FC2B784FF26032C2F2E7
:1003100000022BB349F27433C1F6FF730020D97A7F
:1003200010700A46E1B1CC0706D54FF46142CEF217
:100330000002D86910600A46880706D54EF20412FA
:10034000CEF20002196A1160DA7A510700F1EE80EC
:10035000120705D54EF20C12CEF200029B6A136012
:10036000002002B0BDE8F08149F27433C1F6FF739A
:100370004FF25C32C2F20002D97A12680120287072
:10038000002933D072B6D97A11F0010F08460DD08A
:100390004EF2801CCEF2000CD868DCF800E00EEAC9
:1003A000000EC3F81CE00846CCF800E089070BD526
:1003B0004EF2841ECEF2000E1869DEF800100140E5
:1003C0001962CEF80010D87A41070BD54EF2881E7C
:1003D000CEF2000E5869DEF8001001405962CEF8E6
:1003E0000010D87A010700F1A98062B61B68D968AD
:1003F00091423FF44EAF44F20100C0F23F000021B1
:100400001860C8F23F0142F08040DA60186119605C
:100410003FE7FE2A7FF474AF4FF480604FF6FF7120
:10042000C9F20001C8F21F0018608E4659631A46CF
:1004300059631846596306F5FE77B11CD36A13F069
:10044000F00FFBD0C0F834E0836B01F8013C1B12C5
:1004500001F8023C02318F42F0D106F5FD7106F53C
:100460000076B14210D24FF44042C4F20202174665
:10047000D36A13F0F00FFBD0BB6B181201F8020B1C
:10048000B14201F8013CF3D34FF44043C4F20203FC
:100490004FF480614FF6FF72C8F21F01C9F20002EB
:1004A000196019465A63CA6A4FF4404312F0F00FBC
:1004B000C4F20203F7D020789B6B012106F054FBB5
:1004C0002B784FF26032C2F200025BB349F2743310
:1004D000C1F6FF730020D97A10700A4611B3C8071D
:1004E00006D54FF46142CEF20002D86910600A4688
:1004F0008F0706D54EF20412CEF20002196A11607F
:10050000DA7A560706D54EF20812CEF20002596A80
:100510001160DA7A150705D54EF20C12CEF2000200
:100520009B6A1360012002B0BDE8F0814EF2081210
:10053000CEF20002596A1160DA7A09E74EF28C1E97
:10054000CEF2000E9869DEF8001001409962CEF8F4
:1005500000104AE7F0B44FF44046C4F202064FF0F0
:100560000047336843F4806333603D46F7623446A6
:1005700071633346511C02F20127E26A002AFCDA59
:100580001A6811F8016C42F480621A60DD625E63E1
:10059000E26A002AFCDA1A6811F8026B42F48062FF
:1005A000B9421A60DD625E63E7D14FF44041C4F2A4
:1005B0000201CA6A4FF44043002AC4F20203F8DA87
:1005C0001A684FF0004542F48062FF241A60194611
:1005D000DD625C63CA6A4FF44043002AC4F202033E
:1005E000F8DA1A684FF0004542F48062FF241A607E
:1005F0001946DD625C63CA6A4FF44043002AC4F2C4
:100600000203F8DA1A684FF0004542F48062FF24D2
:100610001A601946DD625C63CA6A4FF44043002ADF
:10062000C4F20203F8DA9B6BDBB203F01F024370E3
:10063000A2F10500B0FA80F04009F0BC704700BF9D
:100640002DE9F041064682B0002900F0AC804FF25F
:1006500060358378C2F20005032B2B780C461746D1
:1006600018BF4C02002B3FD00021307806F07CFAF6
:10067000224618213046FFF773FD002800F09880CD
:100680003078012106F070FA2B784FF26032C2F216
:1006900000022BB349F27433C1F6FF730020D97AFC
:1006A00010700A46E1B1CC0706D54FF46142CEF294
:1006B0000002D86910600A46880706D54EF2041277
:1006C000CEF20002196A1160DA7A510700F1A480B3
:1006D000120705D54EF20C12CEF200029B6A13608F
:1006E000002002B0BDE8F08149F27433C1F6FF7317
:1006F0004FF25C32C2F20002D97A126801202870EF
:1007000000293DD072B6D87A10F0010F01460DD005
:100710004EF2801CCEF2000CD968DCF800E00EEA44
:10072000010EC3F81CE00146CCF800E080070BD5B1
:100730004EF2841ECEF2000E1869DEF80010014061
:100740001962CEF80010D97A48070BD54EF2881EF0
:10075000CEF2000E5869DEF8001001405962CEF862
:100760000010D97A09070AD54EF28C1ECEF2000E7F
:100770009869DEF8001001409962CEF8001062B668
:100780001B68D96891423FF46FAF44F20100C0F298
:100790003F0000211860C8F23F0142F08040DA605B
:1007A0001861196060E74FF26035C2F2000567E733
:1007B0003A46FE213046FFF7CDFE00283FF460AFF9
:1007C00040F23461C2F201014FF440420B680193E0
:1007D000C4F20202DDF8048094464FF0004EFF2080
:1007E000136843F480631360C2F82CE05063D36A4B
:1007F0004FF44044002BC4F20204F8DADCF83870FD
:10080000FFB2FF2F10D00B680093009BC8EB0303CF
:10081000B3F5167FE4D333E74EF20812CEF20002AE
:10082000596A1160DA7A53E700220D213046FFF74A
:1008300097FC00287FF424AF23684FF0004243F474
:10084000806323602146E2626763CA6A4FF44043D3
:10085000002AC4F20203F8DA9B6B13F0FF047FF462
:100860000FAF3078012106F07FF92B784FF260321C
:10087000C2F2000253B349F27433C1F6FF7314702D
:10088000D97A0A4611B3C80706D54FF46142CEF2B1
:100890000002D86910600A468F0706D54EF204128E
:1008A000CEF20002196A1160DA7A560706D54EF2C6
:1008B0000812CEF20002596A1160DA7A150705D5DE
:1008C0004EF20C12CEF200029B6A1360012008E780
:1008D0004FF25C33C2F2000342F20302C3F600029D
:1008E0001A6070472DE9F04F837987B0012B0546D8
:1008F000029205D001232B71002007B0BDE8F08FD4
:1009000042799007F6D553070E4626D5EB68AF69B6
:10091000BB4200F03781002F00F058812A6A147C16
:10092000591E09347A1EE14022FA04F4A14200F271
:100930005181002B00F04E81641A05F1080806E091
:10094000A968286A00F062FC013C0028D2D0424627
:10095000002CF5D1EF603B4600E0EB68029A002ADC
:1009600000F09C8049F2B4324FF270514FF2703B6C
:10097000C1F6FF72C2F20001029F0192C2F2000BA7
:100980000391286A0279013A02EA532212F0FF0920
:10099000C3F3080840F08B80B8F1000F40F0878067
:1009A000A968002940F0BE80EB69002B00F0D080E0
:1009B000AB60C8F50074017C4269A4B2023B8B4075
:1009C0004A44BC4203EB020973D9BCB2B8F1000F30
:1009D00004D1A869EB68834280F0868048460121F3
:1009E00000F030FA002885D008EB0B031819834279
:1009F0004ED008F10408321DD844934238BF464512
:100A000043EA060E2CBF01220022591C1EF0030FE0
:100A100002F00102C1EB000E18BF00220EF1010925
:100A20009C46002A6ED0B9F1090F6BD9AEF10302D2
:100A3000920801324FEA820AA6F104084FF0000E34
:100A400000940EF1010E58F8044F4CF8044B9645F3
:100A5000F7D3CA45009C06EB0A0C03EB0A0E13D031
:100A600016F8228003F822800EF1010398420BD081
:100A70009CF801308EF801300EF10203984203D049
:100A80009CF802308EF80230C1F10101084406449E
:100A9000EB683F1B2344EB607FF473AFAA699A4273
:100AA00075D26A79AB6142F080026A717BE0AB6813
:100AB0007FE7B4F5007F89D1019B1B6899452CD055
:100AC0004FF26C33C2F20003494618680378FE2BDC
:100AD00051D03246FFF7B4FD00283FF40BAF06F5C6
:100AE00000764FF40074D3E700F05EF900283FF47D
:100AF00001AF039A01991378C1F8009043F0010304
:100B0000137071E7013B721E00F1FF3C12F801EF18
:100B100003F801EF9C45F9D1B6E7019A4FF0FF3396
:100B20001360CDE705AA00F071FB00283FF4E5AEA5
:100B3000286A059B90F820404FF6F872C0F6FF72C5
:100B40004FF6F871102C08BF0A469342FFF430AFFD
:100B500005F10802012100F0EDF900283FF4CAAECA
:100B6000EB69002B30D16A79AB68EB6162F07F02F0
:100B70006A71286A1DE73046FFF73EFAB0FA80F046
:100B80004009A9E7029900297FF4ECAE0BE04FF28F
:100B90006433C2F200036A791B6823B1029B13B16C
:100BA00042F080026A7111070AD5AB79002B3FF43D
:100BB000A1AE120611D400F0F7F800283FF49AAE67
:100BC000029807B0BDE8F08FAB68D2E7AF60EF6086
:100BD0003B46C3E6EB69AB60AFE60121286900F054
:100BE00031F900283FF486AE4FF270332C7DC2F20B
:100BF000000313EB44143FF47DAEAB794FF2643243
:100C0000012B9CBFAB69E361C2F20002EB69126881
:100C100063831B0CA38232B104F1160104F11800A6
:100C20009047238B63826B7903F07F036B71C2E77C
:100C300000B583B002AB012203F8011D1946FFF78E
:100C400051FE03B05DF804FB2DE9F84F90F8203019
:100C5000C66949F2B438102B05460F469146C1F6D5
:100C6000FF7822D006EBD116D8F800108E422FD193
:100C70004FF27054C2F200044FF2703307F07F0756
:100C8000C2F2000343F8279023782A7E43F0010341
:100C9000012A237054D9AA684FF26833C2F20003C4
:100CA000114419600120BDE8F88F06EB1126D8F831
:100CB0000010B1420CD14FF27054C2F200044FF256
:100CC0007033FFB2C2F20003314623F81790DBE71E
:100CD0004FF27054C2F200044FF26C3A2378C2F221
:100CE000000AA3B9DAF800000378FE2B2BD04FF2EC
:100CF0007032C2F200023146FFF7BAFAE8B195F855
:100D00002030C8F80060102BD9D03146B4E7DAF8AB
:100D100000000378FE2B32D04FF27032C2F2000294
:100D2000FFF78EFC48B14FF2683BC2F2000BDBF8D4
:100D3000001099B900232370D4E70020BDE8F88F94
:100D40000120BDE8F88F4FF27030C2F2000031464A
:100D5000FFF7E2F8B0FA80F04009CFE7DAF80000D8
:100D60000378FE2B15D04FF27032C2F20002FFF76B
:100D700067FC0028E1D00023CBF80030DAE74FF21F
:100D80007030C2F20000FFF737F9B0FA80F0400986
:100D9000C8E74FF27030C2F20000FFF72DF9B0FA49
:100DA00080F04009E5E700BF70B54FF27054C2F221
:100DB000000423780BB9012070BD4FF26C35C2F2EC
:100DC000000549F2B43328680278C1F6FF73FE2AA1
:100DD000196820D04FF27032C2F20002FFF730FCE7
:100DE000B8B14FF26836C2F20006316819B9002373
:100DF0002370012070BD28680378FE2B15D04FF2B8
:100E00007032C2F20002FFF71BFC10B10023336006
:100E1000EDE7002070BD4FF27030C2F20000FFF726
:100E2000EBF8B0FA80F04009DAE74FF27030C2F226
:100E30000000FFF7E1F8B0FA80F040090028E5D1A2
:100E4000E7E700BF2DE9F84349F2B435C1F6FF7575
:100E500088462B68834218D04FF27054C2F20004C7
:100E60004FF26C3722780646C2F20007C2B93868E2
:100E70000378FE2B38D04FF27032C2F200023146B6
:100E8000FFF7F6F910B32E6003E04FF27054C2F290
:100E90000004217848EA010121700120BDE8F883AF
:100EA00038680278FE2A14D04FF270321946C2F226
:100EB0000002FFF7C5FB48B14FF26839C2F20009E2
:100EC000D9F80010D9B900232370D0E70020BDE87D
:100ED000F8834FF270301946C2F20000FFF78CF829
:100EE000B0FA80F04009E6E74FF27030C2F200003D
:100EF0003146FFF711F8B0FA80F04009C2E73868D0
:100F00000378FE2B0BD04FF27032C2F20002FFF7D3
:100F100097FB0028DAD00023C9F80030D3E74FF25E
:100F20007030C2F20000FFF767F8B0FA80F04009B5
:100F3000EFE700BF2DE9F04F136889B0002B00F0F8
:100F4000AF8003F1010A00230693C3685E1CB0461C
:100F5000002B44D05446A04538BF0224019105928D
:100F60004FF270334FF270524FF26C31C2F2000305
:100F7000C2F20002C2F2000138BFA246B4420546E6
:100F8000029203914FF00007994628D895F8203037
:100F9000EE6949F2B43B102BC1F6FF7B2BD0DBF896
:100FA000001006EBD416B1422BD104F07F034FF2B0
:100FB000703659F82330C2F2000623F0704393B123
:100FC0000134A246EE680137BE4208D9A04538BFB9
:100FD000022406F1010638BFA246B442D6D9002049
:100FE00009B0BDE8F08F631C0199CAEB030291427E
:100FF00073D01C46E6E7DBF8001006EB1426B1427E
:1010000019D0029B1B78F3B94FF26C33C2F2000384
:1010100018680378FE2B38D04FF27032C2F200020B
:101020003146FFF725F90028D9D095F82030CBF8C4
:101030000060102BB9D1E3B24FF2703639F813309B
:10104000C2F20006BBE7039B186802784FF26C33CC
:10105000C2F20003FE2A049300F0A6804FF2703221
:10106000C2F20002FFF7ECFA049B0028B7D04FF25F
:101070006832C2F2000204921168D1B9029918686C
:1010800000220A700378FE2BC6D14FF27030C2F2F4
:1010900000003146FEF740FFB0FA80F04009C2E799
:1010A000A1F10103B3FA83F35B09D0F800A0069322
:1010B0004BE7039A079310680278FE2A00F09B80A2
:1010C0004FF27032C2F20002FFF7BAFA079B002813
:1010D00085D0049900220A60D0E7012C7FF67FAF0B
:1010E000EB6801339C423FF67AAF6FF070422146C5
:1010F0002846FFF7A9FD00283FF471AFA2455ED254
:1011000004F1FF38B8F1010F7FF669AFEB680133E6
:101110004345FFF464AF4FF268334FF27059C2F2A7
:101120000003C2F2000901932EE007EBD817BA4280
:101130000AD000213846FFF785FE00283FF44FAF64
:1011400095F82020102A2AD008F07F0246F8224085
:1011500099F80020297E42F00102012989F8002037
:1011600003D9AA68019B17441F60C24527D008F124
:10117000FF38B8F1010F3FF432AFEA680132904511
:1011800004F1FF343FF62BAF95F82020EF69102AC9
:10119000DBF80020C9D107EB1827BA42C9D15FFAA2
:1011A00088F226F81240D3E74FF27030C2F2000006
:1011B000FEF722FFB0FA80F04009049B55E7059B3B
:1011C000196871B101297FF60AAFEB6801339942C2
:1011D0003FF605AF52462846FFF736FD00283FF49C
:1011E000FEAE059BC3F800A0069B13B10AF10103F4
:1011F0002B600120F4E64FF27030C2F20000FEF7DF
:10120000FBFEB0FA80F04009079B60E72DE9F84F3C
:10121000C36801338B423DD390F82030C46949F252
:10122000B438102B17460E460546C1F6FF7813D08A
:1012300004EBD114D8F800108C4213D14FF2703364
:1012400006F07F01C2F20003012053F8213023F0A1
:1012500070433B60BDE8F88F04EB1124D8F8001010
:10126000A14220D04FF2705AC2F2000A4FF26C39FC
:101270009AF80030C2F2000903BBD9F800000378E5
:10128000FE2B3FD04FF27032C2F200022146FEF731
:10129000EFFF10B90020BDE8F88F95F82030C8F8AE
:1012A0000040102BCAD14FF27033F1B2C2F20003EA
:1012B000012033F811303B60BDE8F88FD9F8000009
:1012C0000378FE2B12D04FF27032C2F20002FFF709
:1012D000B7F90028DED04FF2683BC2F2000BDBF812
:1012E0000010E1B900238AF80030C6E74FF27030F1
:1012F000C2F20000FEF780FEB0FA80F0400900283C
:10130000E9D1C7E74FF27030C2F200002146FEF784
:1013100003FEB0FA80F040090028BED1BAE7D9F840
:1013200000000378FE2B0BD04FF27032C2F20002A5
:10133000FFF786F90028ADD00023CBF80030D1E7C5
:101340004FF27030C2F20000FEF756FEB0FA80F0A5
:101350004009EFE790F8392090F83800101A7047EC
:1013600090F8383090F839209A4205D95A1C034435
:1013700080F83820187E70474FF0FF30704700BF6C
:1013800090F8383090F839209A4286BF1B18187EA2
:101390004FF0FF30704700BF704700BF38B50546BB
:1013A000B0F85E0090B195F85D301446C3F12102AB
:1013B00094420CD805F13B001844224604F0CEFEBE
:1013C00095F85D30234485F85D30204638BD012016
:1013D00014462871EEE700BFB0F85E306BB190F8AC
:1013E0005D30202B07D8C218013380F85D30012012
:1013F00082F83B107047012303710020704700BF43
:101400000023426980F8383080F8393080F85C3049
:1014100080F85D3080F85E3080F85F3006CA30B406
:101420000D68046943662A4383660A60A3704169B4
:1014300090F861300C680B4440F6EC021D7A5B7B3F
:10144000C0F20F0202EBC5051B026D6803F4E063F6
:1014500043F064032B6090F862300B449D7CDB7D8D
:1014600002EBC5021B02526803F4E06343F064031D
:10147000136022684B681A4205D003692C225A7007
:10148000036904229A71036920225A710369802238
:101490009A7030BC704700BF2DE9F04740F23467C6
:1014A000C2F2010782B03B68009340F6EC09DDF818
:1014B000008002690646C0F20F0900214FF49675BC
:1014C000D3789B065BD53B680193019BC8EB030374
:1014D0000F2BF5D949B1102BF2D000209070336951
:1014E00080229A7002B0BDE8F087726996F8613088
:1014F00013440521187A05F06BFB726996F8613088
:101500001344012193F812A0504605F061FB092411
:101510000021504605F028FB2B46013BFDD101215F
:10152000504605F021FB2B46013BFDD1013CEFD19C
:10153000706996F8611001444FF416720C7A4B7B77
:1015400009EBC4011B02496803F4E06343F0640340
:101550000B6096F862300344997CDB7D09EBC10196
:101560001B02496803F4E06343F064030B60013A33
:10157000FDD13269D3789B064FF00101A3D401203D
:1015800002B0BDE8F08700BFF0B503691222DA703F
:101590000269937803F0200385B004460D46002BC2
:1015A00061D0B423937040F23461C2F20101226928
:1015B0000B680093009E05E00B680193019B9B1B49
:1015C000042B42D8D37803F0200303F0FF00002B54
:1015D000F2D094F85D30002B31D04FF0000E4FF078
:1015E000020C04EB0E0393F83B3013710B6803936A
:1015F000039F206907E09B060DD50B680293029BB1
:10160000DB1B052B28D8C378DBB203F0020202F003
:10161000FF06002AEFD080F803C02669F378DBB21A
:10162000DF0632462DD49F062BD5DB0731D40EF1D1
:10163000010E94F85D305FFA8EFE7345D1D800201C
:101640001DBB002384F85E3004E090702369802283
:101650009A70042005B0F0BD8670236980220420B2
:101660009A7005B0F0BD03F0FF06FFF715FF10B943
:10167000042005B0F0BD236984F85F60B0229A7041
:1016800091E78023B3700420DAE726698023B370E2
:10169000D7E7BEF1000F0CBF02200320F6E700BF22
:1016A0002DE9F04306690024122780F8384080F8BD
:1016B0003940F770D0F810E09EF8024004F02004A2
:1016C00089B00546884616461F46002C48D0B423EC
:1016D0008EF8023040F23464C2F201042A692368B1
:1016E0000093009905E0236801930198401A0428AB
:1016F0002DD8D07800F0200000F0FF090028F2D0AB
:101700004FEA480343F00103DBB2137123680293ED
:1017100002982A6905E0236803930399091A0529A9
:1017200015D8D17801F0020101F0FF090029F2D0AB
:101730000220D0702B6993F8039019F011091BD186
:10174000FEB9002F0CBFA02280229A7004E082F81C
:1017500002902B6980229A70484609B0BDE8F08358
:1017600004F0FF09FFF798FE0028F5D02B6985F8F3
:101770005F90B0229A70ADE780229A704FF0000916
:10178000EAE7012E76D0A0229A7029690B79CE461D
:101790004FF0A80C23680493049A05E0236805938E
:1017A000059B9B1A052B4CD8CB7803F0020303F062
:1017B000FF08002BF2D0C8702969CB78DBB213F098
:1017C000100F0A465CD19B065AD5013EF6B2012E97
:1017D0004BD0BEF11F0F3DD90B79012EDAD1236812
:1017E0000693069805E023680793079B1B1A052BB1
:1017F00055D8D37803F0020303F0FF01002BF2D099
:101800000223D3702A69D378DBB2D9063AD49B0677
:1018100036D5B0239370BEF11F0F2B6941D805EB6D
:101820000E02197911760EF1010E5FFA8EFE00BFDD
:1018300000BF00BF0FB180229A7085F839E0F146F1
:101840008AE781F802802B6980229A70F14685F838
:1018500039E081E705EB0E0391F8048083F81880E6
:101860000EF1010E5FFA8EFEB7E781F802C029691A
:101870000A46AEE7A8229A702A69CE461379AEE7E7
:10188000F14669E710214FF49673D170013BFDD109
:101890002A69937803F0F703F14693705CE791703F
:1018A000D1E71A79C3E700BF38B549F22444C1F63D
:1018B000FF742269D578EDB2E9062BD51023D370D9
:1018C0006B0626D505F0040505F0FF03002D6CD04E
:1018D0004FF27153C2F20003616E002249F22445B7
:1018E0001A7084F85D20C1F6FF75002974D088470E
:1018F00095F85D30002B6FD02369D0229A70236950
:1019000094F83B201A712369012284F85C2002229A
:10191000DA7038BD05F0400303F0FF00002BD1D191
:101920009379DBB203F0600160295CD0937803F017
:10193000100303F0FF01D3B115F0010545D194F870
:101940005C1094F85D0049F224438842C1F6FF73AD
:1019500055D95818013190F83B0083F85C1010718C
:101960002369D0229A7023690222DA70D1E784F8C1
:101970006010937943F020039371236994F8390040
:10198000197949F224421F28C9B2C1F6FF72BED8A4
:101990004FF27154C2F200042478002CB7D014180E
:1019A0000130217682F83900B1E7226984F83930B4
:1019B000C023937023694FF27152C2F20002197969
:1019C000012111700222DA70A3E7C023937023690A
:1019D0001A790222DA709CE70122002384F85D2044
:1019E00084F83B3088E703F0DF039371A36E23B1E3
:1019F00084F8380094F839009847226996E7157101
:101A0000AEE700BF38B549F29044C1F6FF742269D1
:101A1000D578EDB2E9062BD51023D3706B0626D509
:101A200005F0040505F0FF03002D6CD04FF2715353
:101A3000C2F20003616E002249F290451A7084F8E8
:101A40005D20C1F6FF75002974D0884795F85D3098
:101A5000002B6FD02369D0229A70236994F83B2021
:101A60001A712369012284F85C200222DA7038BDE1
:101A700005F0400303F0FF00002BD1D19379DBB2D6
:101A800003F0600160295CD0937803F0100303F049
:101A9000FF01D3B115F0010545D194F85C1094F81D
:101AA0005D0049F290438842C1F6FF7355D958183A
:101AB000013190F83B0083F85C1010712369D0224B
:101AC0009A7023690222DA70D1E784F86010937962
:101AD00043F020039371236994F83900197949F28E
:101AE00090421F28C9B2C1F6FF72BED84FF271549E
:101AF000C2F200042478002CB7D0141801302176EB
:101B000082F83900B1E7226984F83930C023937034
:101B100023694FF27152C2F200021979012111704A
:101B20000222DA70A3E7C023937023691A79022294
:101B3000DA709CE70122002384F85D2084F83B30B2
:101B400088E703F0DF039371A36E23B184F83800B4
:101B500094F839009847226996E71571AEE700BFFF
:101B600038B549F2B834C1F6FF742269D578EDB2C0
:101B7000E9062BD51023D3706B0626D505F0040596
:101B800005F0FF03002D6CD04FF27153C2F2000339
:101B9000616E002249F2B8351A7084F85D20C1F6F2
:101BA000FF75002974D0884795F85D30002B6FD001
:101BB0002369D0229A70236994F83B201A71236913
:101BC000012284F85C200222DA7038BD05F040035F
:101BD00003F0FF00002BD1D19379DBB203F0600159
:101BE00060295CD0937803F0100303F0FF01D3B1B8
:101BF00015F0010545D194F85C1094F85D0049F2A8
:101C0000B8338842C1F6FF7355D95818013190F89E
:101C10003B0083F85C1010712369D0229A7023690D
:101C20000222DA70D1E784F86010937943F0200340
:101C30009371236994F83900197949F2B8321F2851
:101C4000C9B2C1F6FF72BED84FF27154C2F200049D
:101C50002478002CB7D014180130217682F839008E
:101C6000B1E7226984F83930C023937023694FF2B9
:101C70007152C2F200021979012111700222DA7048
:101C8000A3E7C023937023691A790222DA709CE7D4
:101C90000122002384F85D2084F83B3088E703F0BC
:101CA000DF039371A36E23B184F8380094F83900F0
:101CB0009847226996E71571AEE700BF30B440F649
:101CC0003005C0F20F05417100210560C272037337
:101CD00001718172417330BC704700BF38B549F261
:101CE00024444379C1F6FF7401255B000822427346
:101CF00084F83B3084F85E5084F85D50417B204688
:101D0000FFF76AFB29462046BDE83840FFF73CBC98
:101D10002DE9F84349F224444379C1F6FF740125C3
:101D20005B0084F83B3084F85E5084F85D50437B60
:101D300001F0F00949EA050806460F01204648EA85
:101D40000301FFF749FB29462046FFF71DFC737985
:101D500084F85E50AB4084F83B3084F85D50717B72
:101D600041F0050149EA01012046FFF735FB4FF03C
:101D70003C0929462046FFF707FCFFB24B46013BD2
:101D8000FDD1737984F85E50AB4084F83B3084F821
:101D90005D50717B204648EA0101FFF71DFB40F6CC
:101DA000B83829462046FFF7EFFB4346013BFDD1FB
:101DB000737984F85E50AB4084F83B3084F85D5012
:101DC000717B294339432046FFF706FB294620460D
:101DD000FFF7DAFB737984F85E50AB4084F83B3050
:101DE00084F85D50717B41F0050139432046FFF7CF
:101DF000F3FA29462046FFF7C7FBB9F10109FCD1E8
:101E0000737984F85E50AB4084F83B3084F85D50C1
:101E1000717B294339432046FFF7DEFA29462046E5
:101E2000FFF7B2FBB8F10108FCD12846BDE8F88302
